:0800000C322E342E302E363066
:1000000A9BB6BC9EE2D7BD98DDE9EDCCA7E7C5AAB1
:1000000AC8CBADEDDAC9CCB2D7DDB5DFE3B8BFC630
:1000000ABFC2C1C8C3C8C30AFEF0BB10030DF2CAFF
:1000000A0AF5F9CEDDD9D7D9D9DADFDFE3DEDBE0CD
:1000000AE2E2E4E4E5EAEAEEE9E609EB0DDE1403EE
:0F00000A06EC1111EF090DF23B2F21EC2211141E
:020000040800F2
:4080000038EC0020A98B0308BB8B0308EDBA0308BF8B0308C18B0308C38B03080000000000000000000000000000000021830008C78B030800000000E58300085984000857
:40804000CD8B0308CD8B0308CD8B0308CD8B0308CD8B0308CD8B0308CD8B0308CD8B0308CD8B0308CD8B0308CD8B0308CD8B0308CD8B0308CD8B0308CD8B0308CD8B0308D0
:40808000CD8B0308CD8B03086D240308CB290308DF2A0308CD8B0308CD8B0308CD8B0308098B0308158B0308218B0308AF8A0308BB8A0308C98A0308D58A0308D95403088D
:4080C000E9540308F954030803550308CD8B03080D5E030809350308133503081D350308CD8B0308CD8B0308CD8B03082D8B0308398B0308458B0308FD8A0308CD8B030820
:40810000CD8B0308CD8B0308DF8A0308CD8B0308CD8B0308CD8B0308EB8A0308F58A0308CD8B0308CD8B0308CD8B0308CD8B0308CD8B0308CD8B0308CD8B0308852A030863
:40814000532B0308C92B0308CD8B0308CD8B0308CD8B0308CD8B0308CD8B03083B3503080D5503081D550308CD8B0308CD8B0308CD8B0308CD8B0308CD8B03080000000034
:40818000CD8B0308CD8B0308453503084F350308CD8B0308CD8B0308175E0308CD8B03080000000000000000CD8B030800F002F800F073F80AA090E8000C82448344AAF13E
:4081C0000107DA4501D100F068F8AFF2090EBAE80F0013F0010F18BFFB1A43F00103184778BA030098BA03000A444FF0000C10F8013B13F0070408BF10F8014B1D1108BFB3
:4082000010F8015B641E05D010F8016B641E01F8016BF9D113F0080F1EBF10F8014BAD1C0C1B09D16D1E58BF01F801CBFAD505E014F8016B01F8016B6D1EF9D59142D6D37C
:40824000704700000023002400250026103A28BF78C1FBD8520728BF30C148BF0B607047632933F0E482732933F0E982002070471FB537F0E0FF9DE8030033F06DFA33F0F9
:40828000E6F833F0BBFB04000020002137F004F9401C60601FBD10B510BD33F08AFB1146FFF7E6FF10F0B7FD33F0BBFB03B4FFF7F2FF03BC33F0ECFB80F309887047EFF3A9
:4082C00009807047684680F3098804480078C00714BF0220032080F3148870479C2B0408DFF818C0EFF305831B0618BF6047EFF31483DB0708BF604700DF70471FE6030829
:40830000DFF818C0EFF305831B0618BF6047EFF31483DB0708BF604700DF704725E80308EFF30980816911F8021C01B142E010B590E80F10E047BDE81040EFF3098C254B5F
:4083400093E80600914232D041B91EF0100F16D12149086820F00100086010E00CB41EF0100F06BF2CED108A0323012381F826302CE9F00FC1F82CC036F0EAFD0CBC1A60D0
:40838000D2F82CC0BCE8F00F92F8263013F0020F1ABFBCEC108A6FF0120E6FF0020E8CF3098813F0010F08BF704792F82500CCF80000704710B5094A1268914209D8084C02
:4083C00054F8214090E80F10A047EFF3098C8CE80F0010BD8C07002034EF00E0DCBA0308DCBA030810B536F067FCBDE81040194B93E80600914208BF70470CB4EFF3098CE3
:408400001EF0100F06BF2CED108A0223002381F826302CE9F00FC1F82CC036F099FD0CBC1A60D2F82CC0BCE8F00F92F8263013F0020F1ABFBCEC108A6FF0120E6FF0020E73
:408440008CF3098813F0010F1CBF92F82530CCF8003070478C07002010B536F049FEC4E710B536F0DBF836F043FEBEE70B49D1F800C04A685CF8043B1068184442F8040BDB
:408480008C4528BFA1F1DC0C8A4228BFA1F1DC02C1F800C04A6020F00040704730E600200146F948B0F8AA0000EE100AB8EE400A81ED080AF44890ED800A81ED010A90ED7C
:4084C000810A81ED020A90ED820A81ED030A90F8AF0000EE100AB8EE400A81ED050AEA4890F8AE000877E84890ED7D0A81ED000A90F8B00000EE100AB8EE400A81ED060A06
:40850000B7EE000A81ED040A012070474FF6FF76DFF878C300DF074639460120DFF870C300DF0421DB4880F8D01100BF002231460120DFF864C300DF0446012C17D100BFA2
:40854000D44890F8D10140F00101D24880F8D111B0F8DC014FF6FF71884207DACD48B0F8DC01401C81B2CB48A0F8DC11DEE7022CDCD1DFF828C300DF054605F0010000288F
:40858000D4D0C748FFF78CFFD0E7C54880ED0C0ADFEDC40AC0ED0D0ADFEDC20AC0ED0F0ADFEDC00AC0ED0E0A80ED0A0A704710B52DED0C8BB0EE409AB0EE608AF0EE419AC2
:4085C0009FEDB80AF0EE408A2022B549243101F1200032F0DCFF9FEDB40AC9EE000AB048C0ED090AB5EEC08AF1EE10FA04D1B0EE480AFFF7CAFF10E1B5EEC08AF1EE10FAFD
:4086000007DDA74890ED120AB5EEC00AF1EE10FA0CD9B5EEC08AF1EE10FA0FD2A04890ED120AB5EEC00AF1EE10FA07DBB0EE480AFFF7ABFF2DF0ADFC99498866984A92ED9C
:40864000080ABCEEC00A10EE101A906E2DF0A7FC50BBB5EEC08AF1EE10FA0ADD9FED930A8F4880ED0A0A9FED8F0A914880ED000A11E09FED900A8A4880ED0A0AD0ED050A9A
:40868000B7EE001A81EE200AF0EE000A80EE201A874880ED001A824890ED0A0A80ED0C0A012085490870B8E09FED800AB4EEC08AF1EE10FA07DB9FED810A794880ED0A0A79
:4086C000F0EE488A80E09FED7B0AB4EEC08AF1EE10FA07D89FED7A0A714880ED0A0AF0EE488A71E0724890ED000A30EE290A80ED000A6B4890ED050ADFED720A20EE200A92
:408700006B48D0ED000A20EE200A10EE101A084637F020FD41EC1D0BB0EE4D0AF0EE6D0A34F0B2FFB0EE40BAF0EE60BA5C4890ED060A10EE101A084637F00CFD41EC1C0B9E
:4087400053EC1B2B37F010FA41EC1A0B36F0C6FE08EE900AF5EEC08AF1EE10FA05DD504890ED060AF0EE408A06E04D4890ED060AB1EE400AF0EE408A38EE880AF0EE408AB9
:40878000B5EEC08AF1EE10FA09DDF5EEC08AF1EE10FA04D89FED4C0AF0EE408A0DE0B5EEC08AF1EE10FA08D2F5EEC08AF1EE10FA03DB9FED460AF0EE408A394890ED000A64
:4087C00020EE280A80ED0A0A3B48007870B13448C0ED0C8A90ED0A0AD0ED090A30EE600A80ED0D0A00203449087016E09FED2D0A2B49243101F1200014F01EF928493431D6
:40880000A1F1300013F0ACFFF0EE408A244890ED0C0A30EE280A80ED0C0A214890ED0A0AB5EEC00AF1EE10FA0BDD90ED0C0AB5EEC00AF1EE10FA04D29FED1A0A80ED0C0A24
:4088400054E0174890ED0A0AB5EEC00AF1EE10FA0BD290ED0C0AB5EEC00AF1EE10FA04DD9FED100A80ED0C0A40E00D4890ED0C0ADFED0E0AB4EEE00AF1EE10FA28DD9FEDBC
:408880000B0A80ED0C0A31E0081F0020C9F3030889E70308D03F0020E9E7030831E70308EC1400200000000000007A440000C842440300200000C8C24003002066662640EB
:4088C000666626C0DB0FC9400AD7233C0AD723BCF64890ED0C0A5FED090AB4EEE00AF1EE10FA03D21FED0D0A80ED0C0AEF4890ED0C0ABDEC0C8B10BD01B500BF0122694695
:40890000EB480068B03010F03BFD20B99DF80000E84981F8B00000BFE748D0F8CC110120DFF898C300DF08BD10B52DED020B00BF04226946DE48006800F5FA7010F020FDA8
:4089400020B99DED000ADB4880ED7D0A00BFDA48D0F8CC110120DFF864C300DF1CBD01B500BF01226946D2480068AE3010F008FD20B99DF80000CF4981F8AE0000BFCE48E8
:40898000D0F8CC110120DFF834C300DF08BD01B500BF01226946C6480068AF3010F0F0FC20B99DF80000C34981F8AF0000BFC248D0F8CC110120DFF804C300DF08BD10B5BF
:4089C0002DED020B00BF04226946B948006800F5027010F0D5FC20B99DED000AB54880ED820A00BFB448D0F8CC110120DFF8CCC200DF1CBD10B52DED020B00BF042269469A
:408A0000AB48006800F5017010F0BAFC20B99DED000AA84880ED810A00BFA748D0F8CC110120DFF898C200DF1CBD10B52DED020B00BF042269469E48006800F5007010F0DA
:408A40009FFC20B99DED000A9A4880ED800A00BF9948D0F8CC110120DFF860C200DF1CBD01B500BF0222694691480068AA3010F087FC20B9BDF800008E49A1F8AA0000BFB1
:408A80008D48D0F8CC110120DFF830C200DF2F2004F038FB08BD10B58AB00446022C1FD1B2EE040A8DED090A9FED850A8DED020A1FED840A8DED030A9FED810A8DED040A35
:408AC0009FED800A8DED060A01208DF820009FED7E0A8DED010AB1EE080A8DED070AA6E0042C1FD1B3EE080A8DED090A1FED910A8DED020A1FED950A8DED030A1FED950A4B
:408B00008DED040A1FED970A8DED060A01208DF820009FED6E0A8DED010AB1EE040A8DED070A84E0052C1FD1B3EE080A8DED090A1FEDA20A8DED020A1FEDA60A8DED030AA9
:408B40009FED630A8DED040A9FED620A8DED060A01208DF820009FED600A8DED010AB1EE040A8DED070A62E00E2C1FD1B2EE040A8DED090A9FED520A8DED020A1FEDB70A97
:408B80008DED030A9FED520A8DED040A9FED4D0A8DED060A01208DF820009FED500A8DED010AB2EE040A8DED070A40E0152C1FD1B2EE040A8DED090A9FED460A8DED020AF9
:408BC0001FEDC80A8DED030A9FED420A8DED040A9FED3C0A8DED060A01208DF820009FED3A0A8DED010AB1EE080A8DED070A1EE01FEDD40A8DED090A1FEDD60A8DED020A16
:408C00001FEDD80A8DED030A1FEDDA0A8DED040A1FEDDC0A8DED060A00208DF820001FEDDF0A8DED010A1FEDE10A8DED070A9DED090ABDEEC00A10EE101A08B2FFF710FF11
:408C4000DDED020AB0EE600AFFF7EFFEDDED030AB0EE600AFFF7CEFEDDED040AB0EE600AFFF7ADFE9DED060ABCEEC00A10EE101AC8B2FFF78CFE9DF82000FFF770FEDDEDFE
:408C8000010AB0EE600AFFF74FFE9DED070ABCEEC00A10EE101AC8B2FFF72EFE2F2004F031FA532004F02EFA0AB010BDEC140020A4030020081F0020D03F002089E703082F
:408CC000000048420000A042F3FDD43CA69B443C000048430000F042BC74933C96438B3C204890ED0A0ABDEEC00A10EE100A00B270471C4890ED090ABDEEC00A10EE100A7B
:408D000000B2704780220270164A92ED010ADFED160A20EE200ABCEEC00A10EE102A91B241700A0A82700F4A92ED020ADFED0E0A20EE200ABCEEC00A10EE102A91B2C170E2
:408D40000A0A0271074A92ED030ADFED070A20EE200ABCEEC00A10EE102A91B241710A0A82717047EC1400200000C84270B5054601249048DFF840C200DF204670BD8F4961
:408D8000097801708E49416001218160002181764176704700B5A1B06846FFF7F0FF01208DF8180006219DF81920501CC0B28DF819000DF14B00815400208DF8190068466E
:408DC00001992CF0B7FD002021B000BD00B5A1B06846FFF7D4FF02208DF8180005219DF81920501CC0B28DF819000DF14B00815400208DF81900684601992CF09BFD9DF842
:408E00001800401E0DF11B01085C21B000BD2DE9F74F814615464FF000081FFA89F7E8191FFA80FBBBF5005F02DD4FF0080854E02D2D02DD4FF040084FE04FF47A615D489A
:408E4000DFF880C100DF012802D14FF0100844E0842032F098F9044654B3FFF79BFFFFF7B5FF82462046FFF78AFFE81C20760221627E501C607604F14B008154390A627EDE
:408E8000501C607604F14B008154627E501C607604F14B008754627E014650182A46019932F030FB00206076204661682CF042FD94F8800001280BD1FFF788FF06460AF0E4
:408EC000020010B106F0020020B14FF0800801E04FF02008204632F091F93648DFF8E8C000DFB8F1000F05D03848007840EA0800364908704046BDE8FE8F2DE9F043A1B0E9
:408F000080460F4614460026BDB260191FFA80F9B9F5005F01DD082642E02D2C01DD40263EE06846FFF72BFFE01CC0B28DF8180003219DF81920501CC0B28DF819000DF1E1
:408F40004B008154290A9DF81920501CC0B28DF819000DF14B0081549DF81920501CC0B28DF819000DF14B0085549DF81920014650185522214632F03CFB00208DF8190058
:408F8000684601992CF0D6FC9DF88000012806D122460DF11E01404632F0B4FA00E0202626B10A480078304308490870304621B0BDE8F083184400205DEB0308C206002072
:408FC0000038004051EC03086DEB0308A103002088B0016807914168069181680591C1680491016903914169029181690191C169009108B070477047FFFFFFFFFFFFFFFF44
:40900000FE4890ED0A0A704710B52DED048BB0EE408A0446F94890ED720ADFEDF90A80EE201AB0EE419AF74890F8AE0058B1FFF7E7FFF0EE409A9FEDF41AF0EE480AFFF786
:40904000B6FAB0EE408AEF4890F89C00012803D1B1EE480AB0EE408A9FEDEC0AB4EEC08AF1EE10FA04D29FEDE90AB0EE408A0AE09FEDE70AB4EEC08AF1EE10FA03DD9FED6B
:40908000E40AB0EE408A062C4DD008DC022C12D0032C12D0042C0DD0052C5ED10CE00E2C06D0122C40D0132C08D0152C55D100E000BF00BF00BF00BF00BF00BFB5EEC08A8A
:4090C000F1EE10FA0ED2B1EE480AB0EE408A0021D04800782AF0E2FB0121CF4800782AF0DDFB19E0B5EEC08AF1EE10FA0ADD0121C84800782AF0D2FB0021C74800782AF0FA
:40910000CDFB09E00021C34800782AF0C7FB0021C14800782AF0C2FBB0EE480ABF4800782EF0FEFE1AE000BFF0EE000A89EE200A9FEDB71AC8EE010A60EE890AB1EE001A02
:40914000C0EE811A70EE218ADFEDB50AB0EE680AB44800782AF01CFC00E000BF00BFBDEC048B10BD70B52DED048B04460D46AE48007848B1012020700121AC4880F82910AF
:409180002CF007FFA9490862207830B101283BD002284DD003286CD157E0A44890F8290001280ED1A148016A28462CF029FFFA2807D2012020709D4890ED090A84ED010A56
:4091C00021E014F0EEFC30B10220207014F0E5FC84ED010A17E0954890F8410001280ED19248816B28462CF00BFFFA2807D2032020708E4890ED0F0A84ED010A03E09FED88
:409200008C0A84ED010A37E0884890F8290030B18648016A28462CF0F3FEFA2802D90020207004E0814890ED090A84ED010A23E014F0B7FC30B10220207014F0AEFC84ED1D
:40924000010A01E00020207016E0784890F8410030B17648816B28462CF0D2FEFA2802D90020207004E0714890ED0F0A84ED010A02E00020207000BF00BF94ED020A84ED84
:40928000030A2078F0B394ED050AB5EEC00AF1EE10FA5AD094ED010A10EE101A084636F059FF41EC190BB0EE490AF0EE690A33F02BFBB0EE408AF0EE608A9FED5E0B53EC96
:4092C000102B51EC180B36F013FC3ED894ED010AB5EEC00AF1EE10FA04D19FED550A84ED020A36E094ED010AD4ED050A30EE600AD4ED020AB4EEE00AF1EE10FA0ADD94EDC5
:40930000020A00E02EE0D4ED050A30EE200A84ED020A1EE094ED010AD4ED050A30EE200AD4ED020AB4EEE00AF1EE10FA08D294ED020AD4ED050A30EE600A84ED020A08E096
:4093400094ED010A84ED020A03E094ED010A84ED020A94ED020A84ED040A0120334981F8480013E09FED320A84ED020A9FED300A84ED010A9FED2E0A84ED030A9FED2C0A10
:4093800084ED040A0020294981F8480094ED040A264880ED110ABDEC048B70BD10B52DED088B044603F00DFEB0EE408A94ED090AD4ED0B0A30EE200AF0EE000A80EE201A8D
:4093C000F0EE418A94ED080AD4ED0A0A30EE200AF0EE000A80EE201AB0EE419A94ED020AB4EEE80AF1EE10FA4CDD94F8440002283ED1B2EE040A03F027F81FE07008002078
:4094000000007A44081F00206F12833A0000C8C20000C842B5060020B60600201407002003005841DB0600202D000020C4070020000000000000000000005940A0B994ED1B
:40944000120A38EE400AF0EE040AB4EEE00AF1EE10FA09D24FF47A71E06C2CF0A0FD30B101215020015502E000215020015508E0022084F8440084ED128A2CF08AFDE064A1
:4094800000BF56E094ED020AB4EEC90AF1EE10FA2BD294F8440001281DD1B2EE040A02F072FFA0B994ED120A38EE400AF8EE040AB4EEE00AF1EE10FA09DD4FF47A71E06CA8
:4094C0002CF06DFD30B101215020015502E000215020015508E0012084F8440084ED128A2CF057FDE06400BF23E0002084F8440094ED120A30EE480A10EE101A084636F07F
:4095000029FE41EC1B0BB0EE4B0AF0EE6B0A33F0FBF9B0EE40AAF0EE60AA9FEDF70B53EC102B51EC1A0B36F01DFC02D2002150200155BDEC088B10BD70B52DED0C8B044657
:409540000D4694ED0A0AF2EE040AB4EEE00AF1EE10FA0CD294ED0A0AFAEE040AB4EEE00AF1EE10FA03DD1FED4E0A84ED0A0A94ED0A0A5FED5D0AC0EE208A95ED020AD5ED09
:40958000080AB4EEE00AF1EE10FA18D895ED0C0AD5ED020A20EE200A1FED631AC0EE010A94ED780A20EE800A1FED6B1AC0EE010A95ED0D0A30EEC00A84ED620A25E095ED8A
:4095C000020AD5ED090AB4EEE00AF1EE10FA18DB95ED0C0AD5ED020A60EE200A1FED741A80EE810AD4ED780A60EE200A1FED7C1A80EE810AD5ED0D0A30EE200A84ED620A5D
:4096000003E01FED750A84ED620A95ED020AB5EEC00AF1EE10FA02D11FED878A18E094ED620A10EE101A084636F094FD41EC1B0BB0EE4B0AF0EE6B0A33F066F9B0EE40AA56
:40964000F0EE60AA51EC1A0B35F048FF08EE100A94ED620A10EE101A084636F07BFD41EC1D0BB0EE4D0AF0EE6D0A33F04DF9B0EE40BAF0EE60BA18EE900A36F06BFD41EC30
:409680001D0BB0EE4D0AF0EE6D0A33F03DF9B0EE40CAF0EE60CA53EC1B2B51EC1C0B36F06FFC41EC1A0B35F019FF09EE100A89EE080AB0EE409A1E219148B0EE490A1AF001
:4096C0005BFEBDEC0C8B70BD2DE9F0412DED028B04460D468B4890F8BD010A287DD14FF432700159001D0151001FD4F8C4120151854800782EF0E2FBC4F8C4024FF4327018
:409700000059D4F8C412081A00EE100AB8EEC00ADFED7E0A80EE201A84EDB41A94EDB40AB2EE041AC0EE010A9FED790A20EE800A84EDC40A95ED020AD5ED080AB4EEE00ACF
:40974000F1EE10FA23D895ED0E0AD5ED020A20EE200A1FEDD11AC0EE010A94ED780A20EE800A1FEDD91AC0EE010A95ED0F0A30EEC00A84EDDA0A94EDDA0AB5EEC00AF1EED9
:4097800010FA37DD1FEDD60A84EDDA0A32E095ED020AD5ED090AB4EEE00AF1EE10FA25DB95ED0E0AD5ED020A20EE200A1FEDE81AC0EE010A94ED780A20EE800A1FEDF01A48
:4097C000C0EE010A95ED0F0A30EE800A84EDDA0A94EDDA0AB5EEC00A00E07DE0F1EE10FA08D21FEDED0A84EDDA0A03E01FEDF00A84EDDA0A434890F830000A2803D132270E
:409800004FF0480802E032274FF04108D4EDC40AB0EE600A394604F53E701AF0ADFDD4EDDA0AB0EE600A414604F554701AF0A4FD94EDD40AD4EDBE0A30EE600AF2EE040A6B
:4098400020EE208A9FED330AB4EEC08AF1EE10FA04DD9FED300AB0EE408A0AE09FED2E0AB4EEC08AF1EE10FA03D29FED2B0AB0EE408A012104F53970B0EE480A1AF07CFDCB
:4098800094EDD40A84EDDD0A94EDBE0A84EDC70A04261AE0711E04F55D7000EB810090ED000A04F55D7000EB860080ED000A04F5477000EB810090ED000A04F5477000EB0E
:4098C000860080ED000A701EC6B2002EE2DC94EDB90A124880ED150ABDEC028BBDE8F081084991F84A10062904D0064991F84A10122915D1012014E0000000000000F83F2D
:40990000B0070020081F0020D80600208DED244800606A4700007A4400007AC4C40700200020704710B52DED020B00BF04226946FE48006800F558700FF022FD20B99DEDEA
:40994000000AFB4880EDD80A00BF1CBD10B52DED020B00BF04226946F448006800F557700FF00EFD20B99DED000AF14880EDD70A00BF1CBD10B52DED020B00BF04226946BD
:40998000EA48006800F556700FF0FAFC20B99DED000AE74880EDD60A00BF1CBD10B52DED020B00BF04226946E048006800F555700FF0E6FC20B99DED000ADD4880EDD50A53
:4099C00000BF1CBDDA4991F84A10032901D1012000E00020704710B52DED020B00BF04226946D248006800F55C700FF0C9FC20B99DED000ACE4880EDDC0A00BF1CBD10B539
:409A00002DED020B00BF04226946C848006800F55B700FF0B5FC20B99DED000AC44880EDDB0A00BF1CBD10B52DED020B00BF04226946BE48006800F55A700FF0A1FC20B9FE
:409A40009DED000ABA4880EDDA0A00BF1CBD10B52DED020B00BF04226946B448006800F559700FF08DFC20B99DED000AB04880EDD90A00BF1CBDAE4991F84A10042918D001
:409A8000AB4991F84A10022913D0A94991F84A1005290ED0A64991F84A100E2909D0A44991F84A10152904D0A14991F84A10132901D1012000E00020704710B52DED028BFD
:409AC00084B00446FFF77EFF10B1B2EE048A01E0B7EE008A964890ED280A20EE080A84ED000AB0F8A80000EE100AB8EE400A84ED020A9FED900A84ED010A8D4890F89C00EE
:409B000084F82C008A4890F842106C3000EB810090ED000A84ED030A854890F84210743000EB810090ED000A84ED040A804890F842107C3000EB810090ED000A84ED050A46
:409B40007B4890F84210843000EB810090ED000A84ED060A764890ED700A84ED070A90ED710A84ED080A90ED720A84ED090A90ED730A84ED0A0A29F067FE002874D0FFF792
:409B8000AFFE78B301216C48007829F087FE00216A48007829F082FE00216948007829F07DFEB2EE040AFFF7F9FE9FED660AFFF7E1FEB7EE000AFFF7C9FE9FED5E0AFFF75D
:409BC000B1FE9FED610AFFF742FF9FED600AFFF72AFF9FED5F0AFFF712FF1FEDB20AFFF7FAFE96E0FFE7FFF746FFE0B35948009094ED020AF0EE400A9FED570A01231A4640
:409C00005649574800782DF05DFE00214A48007829F044FE01214948007829F03FFE01214748007829F03AFE9FED4E0AFFF7B6FE9FED460AFFF79EFE9FED450AFFF786FE24
:409C40001FEDCC0AFFF76EFE9FED470AFFF7FFFE9FED3E0AFFF7E7FE9FED3D0AFFF7CFFE1FEDD40A01E003E044E0FFF7B4FE50E0FFF7A8FE70B33748009094ED020AF0EEA8
:409C8000400A9FED350A01231A463449344800782DF018FE00212848007829F0FFFD01212648007829F0FAFD01212548007829F0F5FD9FED2C0AFFF771FE9FED240AFFF748
:409CC00059FE9FED230AFFF741FE1FEDEE0AFFF729FE1EE000211848007829F0DFFD01211648007829F0DAFD01211548007829F0D5FD0EE01748009094ED020AF0EE400AB6
:409D00009FED150A012300221849154800782DF0D9FD94F82C0068BB00200090019002900346032212490390552024E0A4030020081F002000000000F00600201207002029
:409D4000110700206F12833A00401C45000048420000FA4340D80020A037A04B0018004014070020000048450080544500000140260700200DE029F068FE00200090019097
:409D8000029003460322FE490390562029F05DFE15E0002000900190029003460322F8490390552029F051FE002000900190029003460322F3490390562029F046FE0120F4
:409DC00004B0BDEC028B10BD2DED028B5421EE4831F039FC4FF46771EC4831F034FC5821EB4831F030FCE848EA490860E8484830E9490860E548E949086000F5F070E84911
:409E00000860A0F5DC70E749086000F5B070E649086000F59E70E54908604C30E4490860DB485430E3490860E348E4490860D6481430E34908609FEDE30A143880ED030ABB
:409E40009FEDE00AD24880ED130A9FEDDF0A80ED140AFFF7B7FD40B1DFF870C300DF06460A2202212CF09FF90AE029F0EDFC38B1DFF858C300DF0646012202212CF093F915
:409E8000DFF848C300DF064602212CF0BBF9DFF83CC300DF064631460120DFF834C300DF0321CC4880F8541000BF00224FF6FF710320DFF824C300DF044604F0010000288B
:409EC000F3D104F002000028EFD0DFF810C300DF054605F0010030B1AB481430FFF7EDFD182023F049FF05F002000028DDD0BC48007815F051FBA54880ED780AD0ED780AB8
:409F0000B0EE600A142100F5E4701AF035FA29F083FC78B1B348007815F0FBFC9B4880ED0A0AD0ED0A0AB0EE600A1E2110301AF023FA87E029F088FC002823D0FFF7D0FC6E
:409F400008B3A948007815F0E4FC904880ED8E0AA648007815F020FB8C4880EDA40AD0EDA40AB0EE600A142100F51E701AF004FA8648D0ED8E0AB0EE600A142100F5087086
:409F80001AF0FAF95EE09748007815F0C2FC7F4880ED0A0AD0ED0A0AB0EE600A1E2110301AF0EAF9794890ED0A0AD0ED040A30EE600A20EE000AB0EE408A1E212030B0EE6D
:409FC000480A1AF0D9F98A48007815F0A2FC6F4880ED200AD0ED200AB0EE600A1E2168301AF0CAF9694890ED200AD0ED1A0A30EE600A20EE000AB0EE408A1E217830B0EE9F
:40A00000480A1AF0B9F95F48007815F082FC5F4880ED360AD0ED360AB0EE600A1E21C0301AF0AAF95648007815F073FC574880ED4C0AD0ED4C0AB0EE600A1E2100F58C7004
:40A040001AF09AF950495148FFF73EFB4E494F48FFF772FA4C48FFF7A1F92BF09AFF064631464948FFF77EF84748007820B1484890F84800002845D129F0CEFB90B11FED15
:40A08000D30A414880ED020A00204049087000215848007829F002FC00215748007829F0FDFBBCE029F0D0FB00282AD01FEDDF0A354880ED020A00203449087000214E48AE
:40A0C000007829F0EBFB00214C48007829F0E6FB00214848007829F0E1FB00214848007829F0DCFB00214748007829F0D7FB00214548007829F0D2FB00214448007829F02E
:40A10000CDFB8CE0224890F84800012836D11F48007898BB29F080FB68B101201B49087001213548007829F0B9FB01213148007829F0B4FB73E029F087FBF8B101201349D2
:40A14000087001212C48007829F0A8FB01212B48007829F0A3FB01212648007829F09EFB01212748007829F099FB01212548007829F094FB01212448007849E04FE000005C
:40A1800027070020260700201C08002070080020C40700200000002004000020080000200C000020100000201400002018000020200000201C000020D80B00202400002046
:40A1C000280000200000C8420000C8C2C9F3030889E70308D03F0020E9E7030831E7030893060020E4060020DC060020E1060020E7060020F5060020F60600200B070020D2
:40A20000F40600200D07002015070020F706002029F044FB0121FE48007829F03FFBFD4991F84A00FC49D1ED020AB0EE600AFEF7EBFE3AE601B50BF05FFD70B900BF0122A6
:40A240006946F64800689C300FF09AF820B99DF80000F04981F89C0000BFF148016D0120DFF8C0C300DF132002F04CFF08BD10B52DED020B00249DED000AF2EE040AB4EE47
:40A28000E00AF1EE10FA05DDB2EE040A8DED000A02240BE09DED000AB5EEC00AF1EE10FA04D29FEDE10A8DED000A032400BF04226946DA480068A0300FF062F820B99DED1A
:40A2C000000AD44880ED280A00BFD548016D0120DFF850C300DF182002F014FF20461CBD01B500BF02226946CC480068A8300FF047F820B9BDF80000C649A1F8A80000BF72
:40A30000C748016D0120DFF81CC300DF08BD10B5FFF758FB58B144F62060FFF7E1FFB6EE000AFFF7A4FF0020FFF784FF1BE0FFF7D7FA50B12820FFF7D3FF9FEDBB0AFFF784
:40A3400096FF0020FFF776FF0DE0FFF794FB50B144F62060FFF7C4FF9FEDB30AFFF787FF0020FFF767FFAB4991F84A00FEF793FB012010BD70B52DED028BB0EE408A0446E0
:40A380000D460026012C04D0022C03D0032C4AD101E000BF00BFA54890ED140AB4EEC80AF1EE10FA05DD90ED140AB0EE408A03260CE09E4890ED130AB4EEC80AF1EE10FABD
:40A3C00004D290ED130AB0EE408A022610219748DFF85CC200DF012823D004EB44019348143000EB810080ED018A2BF0D2FD04EB44028E49143141F82200012104EB4402B9
:40A400008A48143000EB8200017204EB44018748143000EB810045728448DFF818C200DF00E0062601E0062600BF00BF3046BDEC028B70BD7D4890ED110A7047764890F896
:40A440005000012800D170470020FCE7774890ED150A70470020754991F84810012904D175490978012900D10120704701B500BF01226946694800684A300EF081FF20B9C5
:40A480009DF80000634981F84A0000BFFFF73FFF6348016D0120DFF88CC100DF262002F031FE08BD644890ED780A7047624890ED8E0A7047604890ED040A70475E4890ED57
:40A4C0001A0A70475C4890ED080A70475A4890ED300A7047584890ED460A704700B5FFF771FA30B15548007808B1012000BD0020FCE70020FAE700207047504800780228AB
:40A5000004D14F48007D012800D170470020FCE710B5FFF7E5F930B14A48007829F0C0FD08B1012010BD0020FCE770B52DED068B0024FFF78FFF70B329F0A2F958B300BF61
:40A54000FFF799FA38B3334890EDD50A10EE101A084635F0FFFD41EC180BFEF751FD10EE105A284635F0F6FD41EC1A0BB0EE4A0AF0EE6A0A32F0C8F9B0EE409AF0EE609AAF
:40A5800053EC182B51EC190B35F0ECFB01D2012000E0002004462046BDEC068B70BD00201D4991ED020A1B4991F84220743101EB8201D1ED000AB4EEE00AF1EE10FA10DB06
:40A5C000154991ED020A134991F84220843101EB8201D1ED000AB4EEE00AF1EE10FA00D80120704700200C4991ED020A094991F842206C3101EB8201D1ED000AB4EEE00A7F
:40A60000F1EE10FA2DD8044991ED020A01491BE0F7060020081F00201C080020A4030020D03F002089E7030800000000C407002051EC03086DEB0308700800202C0000207D
:40A64000402800201907002091F842207C3101EB8201D1ED000AB4EEE00AF1EE10FA00DB0120704700B50023FFF7BCFF10B9FFF796FF00B10123184600BD70B52DED068B7E
:40A680000024FFF7E7FE78B329F0FAF860B3FFF7E9FF48B300BFFFF7EEF928B3FE4890EDD60A10EE101A084635F054FD41EC180BFEF7A6FC10EE105A284635F04BFD41EC1C
:40A6C0001A0BB0EE4A0AF0EE6A0A32F01DF9B0EE409AF0EE609A53EC182B51EC190B35F007FA02D2012001E001E0002004462046BDEC068B70BD70B52DED068B0024FFF788
:40A70000A9FE70BB29F0BCF858B300BFFFF7B3F938B3E14890EDD70A10EE101A084635F019FD41EC180BFEF76BFC10EE105A284635F010FD41EC1A0BB0EE4A0AF0EE6A0AA1
:40A7400032F0E2F8B0EE409AF0EE609A53EC182B51EC190B35F006FB01D2012000E0002004462046BDEC068B70BD70B52DED068B0024FFF780F970B3FFF76CFE58B329F06F
:40A780007FF840B300BFC44890EDD50A10EE101A084635F0DFFC41EC180BFFF797FE10EE105A284635F0D6FC41EC1A0BB0EE4A0AF0EE6A0A32F0A8F8B0EE409AF0EE609A42
:40A7C00053EC182B51EC190B35F0CCFA01D2012000E0002004462046BDEC068B70BD70B52DED068B0024FFF746F978B3FFF732FE60B3FFF7F7FE48B329F042F830B300BF18
:40A80000A54890EDD60A10EE101A084635F0A2FC41EC180BFFF75AFE10EE105A284635F099FC41EC1A0BB0EE4A0AF0EE6A0A32F06BF8B0EE409AF0EE609A53EC182B51EC3D
:40A84000190B35F055F902D2012001E001E0002004462046BDEC068B70BD70B52DED068B0024FFF708F970B3FFF7F4FD58BB29F007F840B300BF884890EDD70A10EE101A2B
:40A88000084635F067FC41EC180BFFF71FFE10EE105A284635F05EFC41EC1A0BB0EE4A0AF0EE6A0A32F030F8B0EE409AF0EE609A53EC182B51EC190B35F054FA01D2012090
:40A8C00000E0002004462046BDEC068B70BD70B52DED068B0024FFF7CEF870B3FFF7BAFD58B328F0CDFF40B300BF6B4890EDD50A10EE101A084635F02DFC41EC180BFFF707
:40A90000E9FD10EE105A284635F024FC41EC1A0BB0EE4A0AF0EE6A0A31F0F6FFB0EE409AF0EE609A53EC182B51EC190B35F01AFA01D2012000E0002004462046BDEC068B20
:40A9400070BD70B52DED068B0024FFF794F878B3FFF780FD60B3FFF722FE48B328F090FF30B300BF4C4890EDD60A10EE101A084635F0F0FB41EC180BFFF7ACFD10EE105A5B
:40A98000284635F0E7FB41EC1A0BB0EE4A0AF0EE6A0A31F0B9FFB0EE409AF0EE609A53EC182B51EC190B35F0A3F802D2012001E001E0002004462046BDEC068B70BD70B5AD
:40A9C0002DED068B0024FFF756F870B3FFF742FD58BB28F055FF40B300BF2F4890EDD70A10EE101A084635F0B5FB41EC180BFFF771FD10EE105A284635F0ACFB41EC1A0BF3
:40AA0000B0EE4A0AF0EE6A0A31F07EFFB0EE409AF0EE609A53EC182B51EC190B35F0A2F901D2012000E0002004462046BDEC068B70BD70B52DED088B0024FFF71CF868B31B
:40AA400028F01EFF50B300BFFFF740FDF0EE400AFFF740FD30EE800AB0EE408A0E4890EDD80A10EE101A084635F074FB41EC190BFFF720FD30EE480A10EE105A284635F0B3
:40AA800069FB41EC1B0BB0EE4B0AF0EE6B0A31F03BFFB0EE40AA02E0081F00200DE0F0EE60AA53EC192B51EC1A0B35F05BF901D2012000E00020044600BF2046BDEC088BBB
:40AAC00070BDD24890ED030A704710B50124D04890F84A000E2811D0CD4890F84A0002280CD0CB4890F84A00152807D0C84890F84A00032803D128F0A7FE00B100240CB1CD
:40AB0000012010BD0020FCE710B50024FFF7A2FCA0B128F0B5FE88B1FFF7D7FF70B100BFFFF7CFFFBA48D0EDD90AB4EEE00AF1EE10FA01DD012000E000200446204610BD4F
:40AB400010B50024FFF786FC98B128F099FE80B1FFF7BBFF68B1FFF7B4FFAD48D0EDDA0AB4EEE00AF1EE10FA01D2012000E000200446204610BD10B50024FFF76BFC98B9C6
:40AB800028F07EFE80B1FFF7A0FF68B1FFF799FF9F48D0EDDB0AB4EEE00AF1EE10FA01DD012000E000200446204610BD994890ED030A704710B50024FFF74CFCA0B128F068
:40ABC0005FFE88B1FFF781FF70B100BFFFF7EEFF8F48D0EDD90AB4EEE00AF1EE10FA01DD012000E000200446204610BD10B50024FFF730FCA0B128F043FE88B1FFF765FFD6
:40AC000070B100BFFFF7D2FF8148D0EDDA0AB4EEE00AF1EE10FA01D2012000E000200446204610BD10B50024FFF714FCA0B928F027FE88B1FFF749FF70B100BFFFF7B6FF96
:40AC40007348D0EDDB0AB4EEE00AF1EE10FA01DD012000E000200446204610BD70B52DED068B002428F00CFE78B3FFF72EFF60B300BF674890EDDC0A10EE101A084635F0A3
:40AC800069FA41EC180BFFF71CFFF0EE400AFFF78DFF30EEC00A10EE105A284635F05AFA41EC1A0BB0EE4A0AF0EE6A0A31F02CFEB0EE409AF0EE609A53EC182B51EC190BDB
:40ACC00035F050F802D2012001E001E0002004462046BDEC068B70BD10B52DED028B9FED4E0AB0EE408A28F097FD28B14B4890ED030AB0EE408A11E028F0A6FD70B1FFF774
:40AD0000E0FEB0EE408AB3EE040AB4EEC08AF1EE10FA03D89FED400AB0EE408AB0EE480ABDEC028B10BD3E4890EDA40A704710B52DED068BFEF7D4FD20B1FFF7C2FEB0EE7A
:40AD4000408A0CE0324890F84A00032803D1354890ED038A03E0FFF7ADFBB0EE408A18EE100A35F0F7F941EC1A0BB0EE4A0AF0EE6A0A31F0C9FDB0EE409AF0EE609A9FEDD4
:40AD80002A0B53EC102B51EC190B34F0B1FE03D89FED210AB0EE408AB0EE480ABDEC068B10BD00B50022FFF755FB90B1FEF798FD78B1FFF7B8FFF0EE400AFFF773FB9FEDE9
:40ADC0001C1A20EE010AF4EEC00AF1EE10FA00DD0122104600BD00B50022FFF73BFB90B1FEF77EFD78B1FFF79EFFF0EE400AFFF759FB9FED101A20EE010AF4EEC00AF1EE20
:40AE000010FA00D20122104600BD00000C0C0020081F0020640C002000000000BC0C002070080020140D002000000000000034406666663FCDCCCC3D10B5044628F0ECFC9A
:40AE400000287DD0092C7CD005DC4CB1032C31D0062C77D158E00B2C75D00C2CF9D1E5E00120FE490870FA208861FA21FB48C1612BF08FF8F94948620121F84880F82810D6
:40AE8000D0ED080AB0EE600AF54800782DF048F80020F24948604FF47A71F0488160416A0161002101759FEDEF0AEF4800782DF037F8F5E00120E9490870FA204860FA21BE
:40AEC000E64881602BF065F8E44908610121E3480175D0ED030AB0EE600AE34800782DF01FF80020DD4988614FF47A71DB48C16101694162002180F828109FEDDA0AD848B9
:40AF000000782DF00DF8CBE00120D44908704FF47A7088610021D148C1612BF03AF8CF4948620121CD4880F82810D0ED080AB0EE600ACB4800782CF0F3FF0020C74903E02B
:40AF4000AFE011E0ABE03AE048604FF47A71C3488160416A0161002101759FEDC20AC24800782CF0DDFF9BE00120BC4908704FF47A7048600021B94881602BF00AF8B74966
:40AF800008610121B5480175D0ED030AB0EE600AB54800782CF0C4FF0020B04988614FF47A71AE48C16101694162002180F828109FEDAC0AAA4800782CF0B2FF70E002205C
:40AFC000A6490870642048600021A44881602AF0E0FFA24908610121A0480175D0ED030AB0EE600AA04800782CF09AFF64209B49886100219948C16101694162002180F801
:40B0000028109FED980A964800782CF089FF0020924981F87C000121904880F87D10022180F88B10002180F88C1039E002208B4908704FF47A7048600146884881602AF0E8
:40B04000A8FF86490861012184480175D0ED030AB0EE600A844800782CF062FF4FF47A707E49886101467D48C16101694162002180F828109FED7B0A794800782CF050FF5C
:40B080000020764981F87C000121744880F87D10022180F88B10002180F88C1000E000BFDDE228F0D1FB0028FAD0102C75D2DFE804F074083E75ABFA74E7E6E5E47474E353
:40B0C000E2E10120654908704FF4FA70C8620146624801632AF05DFF6049886301215F4880F83C106148007828F0D8FB00205B4948604FF47A7159488160816B01610021EC
:40B1000001750020554908644FF47A7153484164816BC164002180F850105348007828F0BDFB00215248007828F0B8FB96E201204A4908704FF4FA700864014647484164DE
:40B140002AF027FF4549C8640121444880F850104748007828F0A2FB0020404948604FF47A713E488160C16C01610021017500203A49C8624FF47A7138480163C16C816397
:40B18000002180F83C103848007828F087FB00213648007828F082FB60E25EE201202F4908704FF4FA70486001462C4881602AF0F0FE2A4908610121284801752A48007812
:40B1C00028F06CFB0020254908644FF47A71234841640169C164002180F8501000201F49C8624FF47A711D48016301698163002180F83C101D48007828F050FB00211C486F
:40B20000007828F04BFB29E20120144908704FF4FA70C8620146114801632AF0BAFE0F49886301210D4880F83C101048007828F035FB4FF4FA70094908640146074841644E
:40B240002AF0A7FE0549C8640121044880F850100748007828F022FB002013E058140020AD06002000000000AE06002005070020FC060020B5E172E129E1EEE0B7E080E007
:40B2800049E010E0F74948600021F64881602AF080FEF44908610021F2480175F248007828F0FCFADAE10120EE4908703220C8623221EC4801632AF06CFEEA4988630121C8
:40B2C000E84880F83C10E948007828F0E7FA3220E44908643221E34841642AF05AFEE149C8640121DF4880F85010E148007828F0D5FA0020DB4948600021DA4881602AF00F
:40B3000048FED84908610021D6480175D648007828F0C4FAA2E10120D24908704FF47A70C8620021CF4801632AF033FECD4988630121CC4880F83C10CC48007828F0AEFA60
:40B340000020C84948604FF47A71C6488160816B0161002101750020C24908644FF47A71C0484164816BC164002180F85010BE48007828F093FA0021BD48007828F08EFA15
:40B380006CE10120B74908704FF47A7008640021B44841642AF0FDFDB249C8640121B14880F85010B248007828F078FA0020AD4948604FF47A71AB488160C16C01610021B2
:40B3C00001750020A749C8624FF47A71A5480163C16C8163002180F83C10A348007828F05DFA0021A148007828F058FA36E101209C4908704FF47A7048600021994881601D
:40B400002AF0C7FD974908610121964801759648007828F043FA0020924908644FF47A71904841640169C164002180F8501000208C49C8624FF47A718A4801630169816359
:40B44000002180F83C108948007828F027FA00218748007828F022FA00E10120814908704FF47A70C86200217E4801632AF091FD7C49886301217B4880F83C107B480078A7
:40B4800028F00CFA4FF47A70764908640021754841642AF07EFD7349C8640121714880F850107348007828F0F9F900206D49486000216C4881602AF06CFD6A490861002132
:40B4C000684801756848007828F0E8F9C6E00220644908704FF47A7048600021614881602AF057FD5F49086101215E48017500215D48007828F0D2F94FF47A705949C862C1
:40B5000000215848016301698163012180F83C1000215648007828F0C1F94FF47A705149086400214F4841640169C164012180F8501000214E48007828F0B0F900204949EE
:40B5400081F87C000221474880F87D10032180F87E1080F88B10002180F88C107EE00220404908706420486000213E4881602AF010FD3C49086101213A4801753A4800784F
:40B5800028F08CF964203749C86200213548016301698163012180F83C103448007828F07DF964202F49086400212E4841640169C164012180F850102D48007828F06EF96F
:40B5C0000020284981F87C000221264880F87D10032180F87E1080F88B10002180F88C103CE001201F4908704FF47A70486001461C4881602AF0CDFC1A490861002119480E
:40B60000017501211948007828F048F94FF47A701449C8620021134801632AF0BAFC1149886301210F4880F83C101048007828F035F900200B4908644FF47A710948416440
:40B640002AF0A7FC0749C8640021064880F850100748007828F022F900E000BF00BF0548047010BD58140020AE06002005070020FC0600203E03002001B59DF8000000EE1C
:40B68000100AB8EE400AFE4880ED030A9DF8000000EE100AB8EE400AF94880ED080A00BF01226946F748006840300DF069FE20B99DF80000F44981F8400000BF0120F349E7
:40B6C000087008BD08B506464FF4C8774FF000080121EF4880F8A8119421E9482FF0B3FF307818B94620FFF7C7FF11E0E64890F84050642D03DD6420FFF7BEFF08E00A2D61
:40B7000003DA0A20FFF7B8FF02E02846FFF7B4FF0020DB4981F88D0028F07EF8E8B10020FFF78AFBDB48DFEDDC0A9FEDDC0A01230022DB490090DB4800782CF0C3F8D54880
:40B74000DFEDD50A9FEDD50A01230022D6490090D64800782CF0B6F805E028F075F810B10120FFF769FB0321C94880F8A81100BF012239464FF6FF70DFF834C300DF2AF076
:40B7800008FC0446BE4890F88D00002874D101201DF071FA18BB28F03FF868B1C548007818B9BA480078012805D10020FFF744FB0020B64908709EE028F046F80028FAD05E
:40B7C000BC480078052803D1B04800780128F2D10520FFF731FB0020AC4908708BE008F0CFFA20BB28F018F870B1B2480078092803D1A648007801287DD10920FFF71CFBC2
:40B800000020A249087076E028F01EF8002872D0A8480078022803D19C48007801286AD10220FFF709FB00209849087063E027F0F3FF70B19F480078062803D193480078BB
:40B84000012858D10620FFF7F7FA00208F49087051E027F0F9FF28B396480078042803D18A480078012846D10420FFF7E5FA0020864908703FE0FFE7814890F88D00012892
:40B8800023D127F0C9FF70B18A4800780C2803D17E48007801282ED10C20FFF7CDFA00207A49087027E027F0CFFF20B3814800780D2803D17548007801281CD10D20FFF721
:40B8C000BBFA00207149087015E06D4890F88D00022810D127F0B8FF68B1764800780F2803D16A480078012805D10F20FFF7A4FA00206649087062480078012802D00228D5
:40B900007ED115E15E48007D28BB5D48406810B35B48016920462AF073FB5949896888423FD3012156480175046127F075FF48B15348D0ED030AB0EE600A5C4800782CF07E
:40B94000EFFA2EE027F080FF10B301215748007827F0A4FF25E04A48007D012821D148488068A8B14648016920462AF049FB44494968884215D3002141480175046127F03C
:40B980004BFF30B19FED4C0A484800782CF0C8FA07E027F059FF20B100214448007827F07DFF374890F82800C8B935488069B0B13348416A20462AF023FB3149C969884204
:40B9C0002BD301212E4880F828104462D0ED080AB0EE600A334800782CF0A2FA1DE0284890F82800012818D12548C069A8B12448416A20462AF004FB21498969884200E01F
:40BA0000F6E10AD300211E4880F8281044629FED2A0A244800782CF083FA194890F85000A8B91748006C90B11548C16C20462AF0E7FA1349496C884245D30121104880F8C2
:40BA40005010C4641D48007827F028FF3BE00C4890F85000012836D10948406C80B30848C16C20462AF0CCFA0549096C88422AD30021034880F85010C4641048007820E0F3
:40BA800058140020A4030020081F00203F030020D03F002040D800200000FA4300247449001C0040AD06002000200040AE060020E9E703083E03002000000000FC06002044
:40BAC00001E027F0EBFED84890F83C00A8B9D648C06A90B1D448816B20462AF091FAD249096B884223D30121CF4880F83C108463CE48007827F0D2FE19E0CB4890F83C000C
:40BB0000012814D1C848006B88B1C748816B20462AF076FAC449C96A884208D30021C24880F83C108463C148007827F0B7FE5FE1BD4890F88C107C30405C78BBBA48007DED
:40BB400001282CD1B848016920462AF059FAB6494968884221D30021B3480175046127F05BFE30B11FED2C0AB14800782CF0D8F90DE027F069FE50B11FED310AAC480078ED
:40BB80002CF0CEF90021AA48007827F087FEA6488068002801D14FF00108C1E00BE0A248016920462AF02CFA9F498968884201D34FF00108B4E09C4890F88C107C30405C3A
:40BBC00001282BD1984890F8280001281AD19648416A20462AF014FA93498969884210D30021914880F8281044621FED4D0A914800782CF095F98C48C069002801D14FF006
:40BC000001088DE08848416A20462AF0F9F98649C969884201D34FF0010881E0824890F88C107C30405C022836D17F4890F83C00012825D17C48816B20462AF0E1F97A497B
:40BC4000C96A88426CD30021774880F83C1084637648007827F022FE27F0F6FD50B100217248007827F01AFE1FED6D0A6F4800782CF056F96C48006B90BB4FF001084FE005
:40BC80006948816B20462AF0BBF96749096B884246D34FF0010843E0634890F88C107C30405C03283CD1604890F8500001282CD15D48C16C20462AF0A3F95B49096C88427B
:40BCC0002ED30021584880F85010C46427F0A4FD38B11FED870A574800782CF021F90EE01EE027F0B1FD50B11FED8D0A524800782CF016F900215048007827F0CFFD4A48BF
:40BD0000406C68B94FF001080AE04748C16C20462AF076F94449496C884201D34FF00108B8F1010F63D14FF000083F4890F88C00401CC1B23C4880F88C1090F88C1090F84F
:40BD40008B00814203DB0021374880F88C10364890F88C107C30405C022809D10121324880F83C1084633148007827F097FD3EE02D4890F88C107C30405C01280DD10121EA
:40BD8000294880F828104462D0ED080AB0EE600A284800782CF0C4F829E0234890F88C107C30405C032809D101211F4880F85010C4642148007827F071FD18E001211A48D5
:40BDC0000175046127F028FD48B11748D0ED030AB0EE600A164800782CF0A2F807E027F033FD20B101211248007827F057FD00BFBEE42DE9F04106460C4617469846069DF4
:40BE00002078642803DD6420FFF736FC09E020780A2803DA0A20FFF72FFC02E02078FFF72BFCBDE8F08100005814002005070020AE060020AD060020FC0600200000000049
:40BE40000000000000000000000000000000000000000000000000000000000000000000000000000000000000000000526176656E20496E647573747269657320496E6342
:40BE80000000000000000000000000004175672D31382D323031380000000000322E342E302E363000000000000000005374656572696E6720436F6E74726F6C20556E69C3
:40BEC0007400000000000000000000003037373031373135303200000000000000000000000000000000000000000000FFFFFFFFFFFFFFFFFFFFFFFFFFFFFFFFFFFFFFFFE4
:40BF0000FFFFFFFFFFFFFFFFFFFFFFFFFFFFFFFFFFFFFFFFFFFFFFFFFFFFFFFFFFFFFFFFFFFFFFFFFFFFFFFFFFFFFFFFFFFFFFFFFFFFFFFFFFFFFFFFFFFFFFFFFFFFFFFF41
:40BF4000FFFFFFFFFFFFFFFFFFFFFFFFFFFFFFFFFFFFFFFFFFFFFFFFFFFFFFFFFFFFFFFFFFFFFFFFFFFFFFFFFFFFFFFFFFFFFFFFFFFFFFFFFFFFFFFFFFFFFFFFFFFFFFFF01
:40BF8000FFFFFFFFFFFFFFFFFFFFFFFFFFFFFFFFFFFFFFFFFFFFFFFFFFFFFFFFFFFFFFFFFFFFFFFFFFFFFFFFFFFFFFFFFFFFFFFFFFFFFFFFFFFFFFFFFFFFFFFFFFFFFFFFC1
:40BFC000FFFFFFFFFFFFFFFFFFFFFFFFFFFFFFFFFFFFFFFFFFFFFFFFFFFFFFFFFFFFFFFFFFFFFFFFFFFFFFFFFFFFFFFF00C00008FFFF030800800008FBBF0008488DFF95E9
:40C0000001B500BF01226946FE48006800F5D9700DF0B6F920B99DF80000FB4981F8B20100BF022017F0A6F9012009F0E4FB08BD01B500BF01226946F248006800F2B31060
:40C040000DF09EF920B99DF80000EF4981F8B30100BF022017F08EF9012009F0CCFB08BD70B52DED028B05460E460024012D07D1E54890ED610ABDEEC00A10EE104A12E0DB
:40C08000032D07D1E04890ED630ABDEEC00A10EE104A08E0022D06D1DB4890ED620ABDEEC00A10EE104AD84890F8B201032809D1D648844202DC4042844201DA00242CE05D
:40C0C00001242AE0D04890F8B20108280AD142F21070844202DC4042844201DA00241CE001241AE0204633F0D8FC41EC180B9FEDC80B53EC102B33F035FE0BD3204633F0B6
:40C10000CCFC41EC180B9FEDC40B53EC102B33F0EFFC01D2002400E001241CB10120BDEC028B70BD0020FAE701460420704731B52DED020B044600BF04226946B148006848
:40C1400000F5C2700DF01CF920B99DED000AAE4880ED610A00BF0AF062FF10B109F055FB02E0012017F026FA1C2021F005FE01203EBD31B52DED020B2DED088B044694B346
:40C1800000209FEDA70A16F043F810EE105A284633F0E0FF41EC1B0BB0EE4B0AF0EE6B0A30F0B2FBB0EE40AAF0EE60AA51EC1A0B33F094F908EE100A934890EDE20A30EEAF
:40C1C000480AF0EE408A90EDE20A30EE080AB0EE409A9DED080AB4EEC90AF1EE10FA03DD8DED089A09E009E09DED080AB4EEE80AF1EE10FA01D2CDED088A0FE000BF042260
:40C2000008A98048006800F562700DF0B9F820B99DED080A7C4880EDE20A00BF00BF042208A97848006800F5C6700DF0A9F820B99DED080A744880ED630A00BF0AF0EFFE1F
:40C2400010B109F0E2FA02E0022017F0B3F91C2021F092FD0120BDEC088B3EBD31B52DED020B044600BF042269466648006800F5C4700DF085F820B99DED000A624880ED15
:40C28000620A00BF0AF0CBFE10B109F0BEFA02E0032017F08FF91C2021F06EFD01203EBD0146002009292BD2DFE801F02A1F20051D1E2A2A13009FED5B1AC0EE010A9FED12
:40C2C0005A1A70EE810AFCEEE00A10EE902A90B218E0DFED550A70EE200AFCEEE00A10EE902A90B20EE000BF00BF00BFDFED4F0A60EE200AFCEEE00A10EE902A90B201E023
:40C30000002000BF00BF704701460020092923D2DFE801F022171805151622220F00DFED410A80EE201AFDEEC10A10EE902A10B214E0FCEEC00A10EE902A10B20EE000BFD0
:40C3400000BF00BFDFED390A60EE200AFDEEE00A10EE902A10B201E0002000BF00BF7047DFED330AB0EE600A28B93249D1ED360AB0EE600A06E0012804D12E49D1ED590A44
:40C38000B0EE600A704770B52DED0A8BB0EE408A9FED290AC8EE000A10EE905A1A4890ED610AF0EE408A90ED630AB0EE409A0020FFF7D6FFF0EE409A284633F0CBFE41EC9D
:40C3C0001A0B38EEE90A78EEC90A80EE201A11EE106A304633F0BEFE41EC1C0BB0EE4C0AF0EE6C0A30F090FAB0EE40BAF0EE60BA53EC1A2B51EC1B0B33F07AFB1ED20120EA
:40C400001DE00000A4030020081F0020001A0B009A999999999913409A9999999999B93F35FA0E3D0000AF4300401C4500007A44000000006C0D00200000C842002004467B
:40C440002046BDEC0A8B70BD70B52DED0A8BB0EE408A1FED070AC8EE000A10EE905AFE4890ED620AF0EE408A90ED630AB0EE409A0020FFF775FFF0EE409A284633F06AFE76
:40C4800041EC1A0B38EEE90A78EEC90A80EE201A11EE106A304633F05DFE41EC1C0BB0EE4C0AF0EE6C0A30F02FFAB0EE40BAF0EE60BA53EC1A2B51EC1B0B33F019FB01D25D
:40C4C000012000E0002004462046BDEC0A8B70BD70B52DED0C8BF0EE408A1FED290AC8EE800A10EE904ADC4890ED620AF0EE409A90ED610AB0EE40AA90ED630AB0EE408AA4
:40C500000020FFF72DFFB0EE409A204633F022FE41EC1B0B39EE480A7AEE480A80EE201A11EE106A304633F015FE41EC1D0BB0EE4D0AF0EE6D0A30F0E7F9B0EE40CAF0EE20
:40C5400060CA53EC1B2B51EC1C0B33F0D1FA24D2204633F0FFFD41EC1B0B39EE480A79EEC80A80EE201A11EE106A304633F0F2FD41EC1D0BB0EE4D0AF0EE6D0A30F0C4F915
:40C58000B0EE40CAF0EE60CA53EC1B2B51EC1C0B33F0AEFA01D2012000E0002005462846BDEC0C8B70BDAD4890F85000032801D0012070470020FCE710B50124FFF7F3FF87
:40C5C00028B9A649C86A642129F0E9FC00B10024204610BDA14890F82800032801D0012070470020FCE710B50124FFF7F3FF28B99A494868642129F0D2FC00B10024204651
:40C6000010BD10B5FFF7EFFF10B1FFF7D5FF08B9022411E0904890ED6A0AB5EEC00AF1EE10FA08D090ED6B0AB5EEC00AF1EE10FA01D0012400E00024204610BD18B9874914
:40C6400091ED080A04E0012802D1844991ED120A704710B50021824800782BF04FFC0021804800782BF04AFC7B4890F8B201032802D0082820D10FE000209FED7B0AFFF7AA
:40C6800056FD00201FED960AFFF773FD00209FED770AFFF7E3FD1FE000209FED750AFFF746FD00201FED9E0AFFF763FD00209FED710AFFF7D3FD0FE00020B7EE000AFFF7C4
:40C6C00036FD0020B0EE040AFFF753FD0020B1EE000AFFF7C3FD00BF00BF10BD01B55E4890F8410001280FD000BF012269466248006800F2B5100CF043FE20B99DF80000F9
:40C70000554981F8B50100BF1C2021F035FB08BD10B52DED028B044694ED030AD4ED040A30EE600A84ED060A94ED030A84ED040A29F02FFC2060D4E90001401AA06094EDA5
:40C74000020AB8EE400A5FEDC70A80EE201AB0EE418A20686060B5EEC08AF1EE10FA0EDD94ED060AC0EE080AC4ED050AD4ED050AB0EE600A042104F11C0017F0FDFDBDECBD
:40C78000028B10BD10B52DED020B00BF042269463948006800F5D4700CF0F2FD20B99DED000A2D4880ED6A0A00BF1CBD10B52DED020B00BF042269462F48006800F5D6709D
:40C7C0000CF0DEFD20B99DED000A234880ED6B0A00BF1CBD214981F8500070471F4981F82800704710B51D4890F86D01012815D0194890F84B00194981F86C01084690F8E6
:40C800006C11543017F0A8FD144890F86C11E03017F0A2FD0120114981F86D010E4890F8B201092877D2DFE800F0A505487B9697A0A67C000A48007827F0F6F900EE100ADC
:40C84000B8EE400ADFED0D0A20EE200A034880ED040A90ED040A13E0081F00206C0D0020D8060020D706002090ED24C990ED244900803BC500803B45A40300203333533A00
:40C88000F6EE000AB4EEE00AF1EE10FA03D20020FFF7A4FF10E0F94890ED040ADFEDF80AB4EEE00AF1EE10FA03DD0120FFF796FF02E00320FFF792FF66E0F248007827F061
:40C8C000B3F900EE100AB8EE400A5FED140A20EE200ADFEDED0A80EE201AE84880ED041A90ED040ADFEDE90AB4EEE00AF1EE10FA03D20020FFF772FF11E0E04890ED040A0D
:40C90000DFEDE30AB4EEE00AF1EE10FA04DD0120FFF764FF03E02CE00320FFF75FFF33E000BFD84800782BF0C9FA00EE100AB8EEC00AD248D0ED000A30EE200A80ED040AA4
:40C94000FDF7CCFD18B10020FFF748FF02E00320FFF744FF18E000BF9FEDCE0AC74880ED040A0020FFF73AFF0EE00320FFF736FF0AE000BF00BF9FEDC70AC04880ED040A1E
:40C980000020FFF72BFF00BF00BFBC4890F86C11D0ED040AB0EE600A543017F089FCB748001DFFF7B5FEBC4890F8B301092870D2DFE800F08005337065667B727100B7484E
:40C9C000007827F031F900EE100AB8EE400A5FED550A20EE200AA94880ED0E0A90ED0E0AF6EE000AB4EEE00AF1EE10FA03D20020FFF7F0FE10E0A14890ED0E0ADFEDA00A78
:40CA0000B4EEE00AF1EE10FA03DD0120FFF7E2FE02E00320FFF7DEFE55E0A048007827F003F900EE100AB8EE400A5FED6C0A20EE200ADFED950A80EE201A904880ED0E1AB9
:40CA400090ED0E0ADFED910AB4EEE00AF1EE10FA03D20020FFF7BEFE10E0884890ED0E0ADFED8B0AB4EEE00AF1EE10FA03DD0120FFF7B0FE02E00320FFF7ACFE23E000BF67
:40CA80009FED840A7D4880ED0E0A0020FFF7A2FE19E00EE000BF00BF9FED7E0A774880ED0E0A0320FFF796FE0DE00320FFF792FE09E000BF9FED770A704880ED0E0A00204A
:40CAC000FFF788FE00BF00BF6C4890F86C11D0ED0E0AB0EE600AE03017F0EAFB67482C30FFF716FE10BD6C4890ED610AD0ED630A30EE600AB5EEC00AF1EE10FA01DD012025
:40CB000070470020FCE730B589B026F0B0FE40B10021084616F03BFD0121002016F037FD1AE05D4890F8B201032804D05A4890F8B201082808D10021032016F028FD0121EF
:40CB4000032016F024FD07E00021032016F01FFD0121002016F01BFD4F4890F8B25190F8B341092D7BD2DFE805F0A3051729A5A65DA42A0000200090019002900346032242
:40CB8000404903900846007826F05FFF03213D48007827F008FBA0E0002000900190029003460322374903900846007826F04DFF00213448007827F0F6FA8EE000BF00207F
:40CBC000009001900290034602222E4903900846007826F03AFF02212A48007827F0E3FA26F01AFE68B12E48DFED2A0A9FED2D0A042300222C490090224800782AF062FECB
:40CC00000FE026F021FE60B12548DFED220A9FED250A04230022190700901A4800782AF051FE5AE0002000900190029003460222144903900846007826F007FF0621114897
:40CC4000007827F0B0FA002000900190022314220121029004A82AF04DFF04A800E027E0DFED0C0A9FED110A032300224FF080410090044800782AF025FE2EE06C0D00207D
:40CC800066664640D80600200CAC233FCDCCCC3C33339F4000000000081F0020D706002040D80020809FD54A00040140A037A04C00BF00BF00BF0020009001900290034609
:40CCC0000322FA4903900846007826F0BEFE0121F648007827F067FA00BF00BF092C7BD2DFE804F0880517298A8B5D892A00002000900190029003460322ED49039008464C
:40CD0000007826F0A2FE0321E948007827F04BFA85E0002000900190029003460322E44903900846007826F090FE0021E048007827F039FA73E000BF0020009001900290DC
:40CD400003460222DA4903900846007826F07DFE0221D748007827F026FA26F05DFD68B1D4485FED340A1FED310A04230122D2490090CF4800782AF0A5FD0FE026F064FD2C
:40CD800060B1CC485FED3D0A1FED3A0A0423012291070090C64800782AF094FD3FE0002000900190029003460222C14903900846007826F04AFE0621BD48007827F0F3F901
:40CDC000002000900190034614220121029004A82AF090FE04A800E00CE05FED520A1FED4F0A0223012291070090B14800782AF069FD14E000BF00BF00BF00200090019013
:40CE0000029003460322AA4903900846007826F01CFE0121A648007827F0C5F900BF00BF09B030BD10B5A54988684FF4967129F0B6F810BDA24890ED000A7047A14991F8D9
:40CE40004110012901D1012007E09E4991F8B51109B1012100E000210846704710B52DED068BB0EE408A9848007838B91FED770A964880ED000A012093490870FFF7DEFFFA
:40CE8000002868D008F038FF002864D0FFF7D2FF10EE104A204633F05DF941EC1A0BB0EE4A0AF0EE6A0A2FF02FFDB0EE409AF0EE609A9FED870B53EC102B51EC190B32F03D
:40CEC00017FE48D2FFF7AEFFE8BB20F005FADFED820AB4EEE00AF1EE10FA3CDBFFF791FB012838D1774890F830000A2833D0754890F8B201092827D2DFE800F02610110545
:40CF000012132626060000BF704890ED000ADFED730A08EE200A80ED000A1BE000BF00BF00BF6848D0ED630A9FED6C1A48EE410AB0EE600A0120FFF71CF91FEDAA0A634858
:40CF400080ED000A06E006E01FEDAE0A5F4880ED000A00BF00BFBDEC068B10BD5B4890F8280008B9012070470020FCE7574890F82800012800D170470020FCE7534890F8F2
:40CF8000500008B9012070470020FCE74F4890F85000012800D170470020FCE700B50021FFF7DCFF08B13D2103E0FFF7DFFF00B13C21084600BD10B516F090FB04462046CE
:40CFC00010BD10B52DED028B0AF029F820B108F098FCB0EE408A16E016F088FA3948D0ED640A30EE600ADFED3E0A20EE200AD0ED650A90ED641A70EEC10A80EE201A9FED96
:40D00000390A31EE008AB0EE480ABDEC028B10BD01B59DF80000202801DD2020009000BF01226946304800684B300CF0A9F920B99DF80000234981F84B0000BF002023495D
:40D0400081F86D0108BD10B54FF4B8711F482EF0FAFA10BD25490870704724480078704710B52DED028BB0EE408A2148007830B9134800210160416001201D49087020F02A
:40D0800027F9F0EE408AF0EE680AB0EE480A16F0FFF8184880ED000A28210948154A92ED000A17F069F9BDEC028B10BDD8060020D706002040D8002000040140DC420020F0
:40D0C00038000020081F0020400000206C0D0020000000A046DF813F2FDDE43E0AD7A33B000048430000C8C2A4030020300000204100002034000020014890ED000A7047BE
:40D100003400002010B50446204622F0F4F810BD07B586B00020049000210898017006980078472881F06481DFE810F047004900C500E500130162098900160721072C0727
:40D140004101A7010D028202D7022C037903CE03330423045A008304F5046305A905F8057606C40890063707520943077F078E07C307D107DF0720082C083C0846085608E2
:40D180006209620962096608770890084F075B0773076707620962096209620962096209620962096209620962099A04620962096209C808F0080D09350901F01DB9FE4868
:40D1C00090F841000390069890ED010ABCEEC00A10EE100AC0B20290039916F0D8F9ECE70698007A032803D006210898017025E0069890ED010AF7EE000AB4EE600AF1EE84
:40D2000010FA02D114F05CFB18E0069890ED010AF0EE000AB4EE600AF1EE10FA02D114F037FB0BE0069890ED010AF0EE080AB4EE600AF1EE10FA01D114F088F9BDE7069823
:40D24000007A032809D1069890ED010A8DED030A9DED030A0DF08EFF2AE00698007A012811D1D548B0F8BE110A22079802FB001000EE100AB8EEC00A8DED030A9DED030A32
:40D280000DF078FF14E00698007A022810D1CA48B0F8BE110A22079802FB101000EE100AB8EEC00A8DED030A9DED030A0DF062FF0120049081E708F01FFDC0B90698007ABC
:40D2C000032811D1069890ED010A8DED030A9DED030A09F0B7FAB948D0F81801014603908020DFF8DCC200DF0120049002E001210898017061E713F0D3FC30BB0698007A9C
:40D3000003281ED1069890ED010ABCEEC00A10EE100A80B2039009F086FA09F006FA80B90821A848DFF8A0C200DF012809D0A748406840F00101A5484160A248DFF890C214
:40D3400000DF132020F018FD02E001210898017033E713F0A5FC30BB09F0E7F918B30698007A03281BD1069890ED010ABCEEC00A10EE100AC0B2039009F02FFA082191480A
:40D38000DFF844C200DF012809D09048406840F001008E4948608B48DFF834C200DF132020F0EAFC02E001210898017005E70698007A032817D1804890F8420003907E48C0
:40D3C00090F841000290069890ED010ABCEEC00A10EE100AC0B20190DDE9021210F03FFC0899087046E00698007A01281FD1724890F841105C3000EB41006F4991F84210BA
:40D40000415C0122079802FB0010C0B201906A4890F842000390684890F8410002900146039A019810F01BFC0899087022E00698007A02281ED1604890F841105C3000EB8B
:40D4400041015C3890F84200095C0122079802FB1010C0B20190584890F842000390564890F8410002900146039A019810F0F7FB08990870012004909FE60698007A0328CA
:40D4800017D14D4890F8420003904B4890F841000290069890ED010ABCEEC00A10EE100AC0B20190DDE9021210F033FC0899087046E00698007A01281FD13F4890F8411016
:40D4C000603000EB4101603890F84200095C0122079802FB0010C0B20190374890F842000390354890F8410002900146039A019810F00FFC0899087022E00698007A02283D
:40D500001ED12D4890F84110603000EB41002A4991F84210415C0122079802FB1010C0B20190254890F842000390234890F8410002900146039A019810F0EBFB0899087019
:40D540000120049039E60698007A032817D11A4890F842000390184890F841000290069890ED010ABCEEC00A10EE100AC0B20190DDE9021210F00AFC0899087055E00698B1
:40D58000007A01282ED10C4890F84110643000EB4100094991F84210415C0122079802FB0010C0B20190044890F842000390024890F8410002900DE0081F0020D03F00208F
:40D5C00089E70308B02F002051EC0308C02F00206DEB03080146039A019810F0D7FB0899087022E00698007A02281ED1FE4890F84110643000EB4100FB4991F84210415CC1
:40D600000122079802FB1010C0B20190F64890F842000390F44890F8410002900146039A019810F0B3FB0899087001200490C4E50698007A032810D1EB4890F84200039080
:40D64000069890ED010A8DED020A03989DED020A10F0FAFC089908703CE00698007A01281AD1E14890F842107C3000EB8100D0ED000A9DED070AB8EEC00A30EEC00A8DED27
:40D68000020AD94890F8420003909DED020A10F0DBFC089908701DE00698007A022819D1D14890F842107C3000EB8100D0ED000A9DED070AB8EEC00A30EE800A8DED020A26
:40D6C000C94890F8420003909DED020A10F0BCFC08990870012004906FE50698007A032810D1C14890F842000390069890ED010A8DED020A03989DED020A10F0EBFB08995E
:40D7000008703CE00698007A01281AD1B64890F842106C3000EB8100D0ED000A9DED070AB8EEC00A30EEC00A8DED020AAE4890F8420003909DED020A10F0CCFB0899087040
:40D740001DE00698007A022819D1A74890F842106C3000EB8100D0ED000A9DED070AB8EEC00A30EE800A8DED020A9F4890F8420003909DED020A10F0ADFB089908700120F3
:40D7800004901AE50698007A032812D1964890F842000390069890ED010ABCEEC00A10EE100AC0B20290039910F02EFB0899087032E00698007A012815D18B4890F84210FB
:40D7C0006830415C0122079802FB0010C0B20290854890F8420001460390029810F014FB0899087018E00698007A022814D17E4890F842106830415C0122079802FB10101B
:40D80000C0B20290784890F8420001460390029810F0FAFA0899087001200490CDE40698007A032810D1704890F842000390069890ED010A8DED020A03989DED020A10F05D
:40D840006CFC089908703CE00698007A01281AD1654890F84210843000EB8100D0ED000A9DED070AB8EEC00A30EE800A8DED020A5D4890F8420003909DED020A10F04DFC57
:40D88000089908701DE00698007A022819D1564890F84210843000EB8100D0ED000A9DED070AB8EEC00A30EEC00A8DED020A4E4890F8420003909DED020A10F02EFC0899FA
:40D8C00008700120049078E40698007A032810D1454890F842000390069890ED010A8DED020A03989DED020A10F052FB089908703CE00698007A01281AD13B4890F84210A9
:40D90000743000EB8100D0ED000A9DED070AB8EEC00A30EE800A8DED020A334890F8420003909DED020A10F033FB089908701DE00698007A022819D12B4890F84210743008
:40D9400000EB8100D0ED000A9DED070AB8EEC00A30EEC00A8DED020A234890F8420003909DED020A10F014FB089908700120049023E40698007A03280AD1069890ED010A75
:40D98000BCEEC00A10EE100AC0B20390FCF752FC13E40698007A032812D1134890F842000390069890ED010ABCEEC00A10EE100AC0B20290039910F05AFA0899087035E0EC
:40D9C0000698007A012818D1074890F842106A30415C0122079802FB0010C0B20290024890F84200014601E0081F00200390029810F03DFA0899087018E00698007A022890
:40DA000014D1FB4890F842106A30415C0122079802FB1010C0B20290F54890F8420001460390029810F023FA089908700120049004E40698007A032803D00621089801702E
:40DA40000DE0069890ED010A8DED030A9DED030A0A2007F026FC10B90121089801707AE20698007A032814D1069890ED010ABCEEC00A10EE100A80B200EE100AB8EE400AD6
:40DA80008DED030A9DED030A0DF074FB089908703EE00698007A01281BD10EF0B3F8F0EE400AD348B0F8BE0100EE100AB8EE401A9DED070AF8EE401AB0EE410A00EEA10AC0
:40DAC0008DED030A9DED030A0DF054FB089908701EE00698007A02281AD10EF093F8F0EE400AC348B0F8BE0100EE100AB8EE401A9DED070AF8EE401AB0EE410A00EEE10AB0
:40DB00008DED030A9DED030A0DF034FB08990870012004901FE20698007A032815D1B44890F842000390B24890F841000290069890ED010A8DED010ADDE902019DED010AEC
:40DB400010F03BF80899087050E00698007A012824D1A74890F842000290A54890F84100019002990EF0E2FDDDED070AF8EE600A9FEDA01A01EE200A8DED030A9C4890F86C
:40DB8000420002909A4890F84100019002999DED030A10F012F80899087027E00698007A022823D1924890F842000290904890F84100019002990EF0B9FDDDED070AF8EE4B
:40DBC000600A9FED8C1A01EE600A8DED030A884890F842000290864890F84100019002999DED030A0FF0E9FF0899087001200490B1E10698007A03280BD1069890ED010A97
:40DC00008DED030A9DED030A10F010FB0899087032E00698007A012815D17548D0ED7E0A9DED070AB8EE401ADFED731AB0EE600A01EE810A8DED030A9DED030A10F0F6FAE3
:40DC40000899087018E00698007A022814D16848D0ED7E0A9DED070AB8EE401ADFED661AB0EE600A01EEC10A8DED030A9DED030A10F0DCFA0899087001200490BCE30698CF
:40DC8000007A032814D1069890ED010ABCEEC00A10EE100A80B200EE100AB8EE400A8DED030A9DED030AFCF7E2FA0899087032E00698007A012815D14D48D0ED280A07989C
:40DCC00000EB8000400000EE100AB8EEC00A30EE800A8DED030A9DED030AFCF7C8FA0899087018E00698007A022814D14048D0ED280A079800EB8000400000EE100AB8EEDF
:40DD0000C00A30EEC00A8DED030A9DED030AFCF7AEFA08990870012004906DE30698007A03282DD1069890ED010ADFED340AB4EEE00AF1EE10FA06DD0221089801706420D9
:40DD4000FDF79AFC62E0069890ED010AF2EE040AB4EEE00AF1EE10FA06D20321089801700A20FDF789FC51E0069890ED010ABCEEC00A10EE100AC0B20390FDF77DFC45E024
:40DD80000698007A01281BD1194890F8401007984000C0F1650081420BDA154890F840100222079802FB0010C0B20390FDF764FC2CE00221089801706420FDF75DFC25E0EC
:40DDC0000698007A022821D1094890F84010079840000930814213DD054890F840100222079802FB1010C0B20390FDF745FC0DE0081F00200AD7233CCDCCCC3D0000C8429C
:40DE00000321089801700A20FDF736FC1920FFF779F901200490EFE20698007A032803D006210898017010E0069890ED010ABCEEC00A10EE100AC0B21FED100A039007F024
:40DE400030FA10B9012108980170D5E20698007A032803D00621089801707CE0069890ED010AF8EE000AB4EE600AF1EE10FA13D1FE4890F842107C3000EB810090ED000A6D
:40DE80008DED030A9DED030A082007F00AFA00BB0121089801705EE0069890ED010AFFEE000AB4EE600AF1EE10FA13D1EF4890F842106C3000EB810090ED000A8DED030AD8
:40DEC0009DED030A082007F0ECF910B901210898017040E0069890ED010AF7EE000AB4EE600AF1EE10FA13D1E04890F84210743000EB810090ED000A8DED030A9DED030AC6
:40DF0000082007F0CEF900BB01210898017022E0069890ED010AF0EE000AB4EE600AF1EE10FA13D1D14890F84210843000EB810090ED000A8DED030A9DED030A082007F04D
:40DF4000B0F910B901210898017004E09FEDC80A002007F0A6F94FE20020FEF701FA8DED030A00209DED030AFEF7E1F844E20020FEF7F6F98DED030A00209DED030AFEF75A
:40DF8000F8F839E20020FEF7EBF98DED030A00209DED030AFEF762F92EE2069890ED010ABCEEC00A10EE100AC0B203900DF08CFC22E2069890ED010ABCEEC00A10EE100ACD
:40DFC000C0B20390FEF78AFB16E2069890ED010ABCEEC00A10EE100AC0B2039010F083FA0AE2069890ED010ABCEEC00A10EE100AC0B203900EF01EFBFEE1069890ED010AB7
:40E00000BCEEC00A10EE100A80B203900EF0FAF8F2E1069890ED010ABCEEC00A10EE100A80B203900EF003F9E6E1069890ED010ABCEEC00A10EE100AC0B203900FF0CAF81C
:40E040002020FFF75FF8D7E10698007A032803D00621089801702BE0069890ED010AF7EE000AB4EE600AF1EE10FA05D1B7EE000A072007F016F91BE0069890ED010AF0EE47
:40E08000000AB4EE600AF1EE10FA05D19FED780A002007F006F90BE0069890ED010AF0EE080AB4EE600AF1EE10FA01D100F080FBA2E1069890ED010ABCEEC00A10EE100AFF
:40E0C00080B201460390022015F074F894E1069890ED010ABCEEC00A10EE100A80B201460390012015F066F886E10698007A03283BD1069890ED010AB5EEC00AF1EE10FA98
:40E100000BD15A4890F842000390584890F841000290039908F075FD27E0069890ED010AF7EE000AB4EE600AF1EE10FA07D14F4890F842000121039008F0CAFC15E00698B3
:40E1400090ED010AF0EE080AB4EE600AF1EE10FA0BD1464890F842000390444890F8410001220290039908F032FC45E1069890ED010ABCEEC00A10EE100AC0B2039008F0CA
:40E18000F2FB39E10698007A03280AD1069890ED010ABCEEC00A10EE100AC0B20390FCF765F929E112F07CFD28B90698007A032801D108F079FB1FE10698007A03280AD12D
:40E1C000069890ED010ABCEEC00A10EE100AC0B20390FDF715FF0FE10698007A03280AD1069890ED010ABCEEC00A10EE100AC0B20390FDF71DFFFFE00698007A03280BD18D
:40E20000069890ED010ABCEEC00A10EE100AC0B2012103900EF020F8EEE00698007A032813D1069890ED010ADFED120AB4EE600AF1EE10FA09D10CF02DF801200BF008FFD9
:40E2400000200D4908720D490870D5E00698007A032815D1069890ED010ABDEEC00A10EE100A00B20390FAF7FBFB22E0081F00200000000000007E43C02F0020C80400201E
:40E280000698007A012808D1F248B0F8AA00401C00B20390FAF7E4FB0BE00698007A022807D1EC48B0F8AA00401E00B20390FAF7D7FBA1E01B20FEF725FF9DE00698007AEC
:40E2C00003281AD1E34890F842106C3000EB810090ED000A8DED050A9DED050AB5EEC00AF1EE10FA03D19FEDDC0A8DED050A9DED050A082006F0D5FF07E00698007A20B9CA
:40E300001FED250A082006F0CCFF75E00698007A03280FD1CF4890F842107C3000EB810090ED000A8DED030A9DED030A082006F0B8FF07E00698007A20B91FED330A082075
:40E3400006F0AFFF58E00698007A03281AD1C14890F84210743000EB810090ED000A8DED050A9DED050AB5EEC00AF1EE10FA03D19FEDBA0A8DED050A9DED050A082006F03D
:40E3800090FF07E00698007A20B91FED470A082006F087FF30E00698007A03280FD1AD4890F84210843000EB810090ED000A8DED030A9DED030A082006F073FF07E0069819
:40E3C000007A20B91FED560A082006F06AFF13E00698007A03280AD1069890ED010ABCEEC00A10EE100AC0B2039008F09DFA03E007210898017000BF00BF049809B000BDD4
:40E4000086B04FF6FF7438219548DFF858C200DF0221954880F808110C228421934830F05DF8002874D103218F4880F8081100BF224605A98A48DFF838C200DF012857D094
:40E4400000208DF800008DF80D0001208DF80C0000208DF80E0005980078002839D004AA01210598FEF754FE05469DF8100068B100250599087821F077FA06460598837A52
:40E48000427A9DF81010304621F074FA07F034FC08B1002504E00598007A032800D100250DB39DF80D00F0B90598007AD8B1059A07CA8DE8070001208DF80D008DF80C00FA
:40E4C0004FF47A649DF80E00401CC0B28DF80E0009E006F01DFF30B16348D0F890110120DFF890C100DF61480599F9F709FF9FE79DF8000000289BDD9DF80E0000283DDD00
:40E500009DF80E00032804D102208DF80C000FE037E09DF80E00052803D106208DF80C0006E09DF80E00072802D110208DF80C009DF80E00FF2805DA9DF80E00401CC0B2BE
:40E540008DF80E009DF80C1004AA6846FEF7E0FD9DF8100078B100208DF80E000599087821F002FA06460598837A427A9DF81010304621F0FFF94FF4FA6459E74FF6FF740E
:40E5800056E70521384880F808110020DFF8E8C000DF00BFFEE72DE9F0472DED028B0546B0EE408A0E46174698464FF001092C48DFF8C8C000DFD0B900BF2B4890F8090147
:40E5C00040F00201284880F80911B0F814014FF6FF71884207DA2448B0F81401401C81B22148A0F8141100BF4FF000092CE01F48F9F776FE04466CB1257084ED018A26727D
:40E60000677284F80A800A2221461548DFF870C000DF19E000BF144890F8090140F00401114880F80911B0F814014FF6FF71884207DA0D48B0F81401401C81B20A48A0F8B7
:40E64000141100BF4FF000094846BDEC028BBDE8F0870000081F0020CDCCCCBDCDCCCC3D740F002011E90308D03F0020F00E0020A1EA030889E703080DF2030809E9030876
:40E68000FDE9030831B52DED020B0446FE4890EDD40ADDED000AB4EEE00AF1EE10FA00D3ACB100BF04226946F848006800F554700AF066FE20B99DED000AF34880EDD40AB2
:40E6C00000BFF348C16B0220DFF8C8C300DF3EBD31B52DED020B0446EB4890EDD30ADDED000AB4EEE00AF1EE10FA00DCACB100BF04226946E548006800F553700AF040FE17
:40E7000020B99DED000AE04880EDD30A00BFE048C16B0220DFF87CC300DF3EBD31B52DED020B0446D84890ED2F0ADDED000AB4EEE00AF1EE10FA00D3A4B100BF04226946A3
:40E74000D2480068BC300AF01BFE20B99DED000ACD4880ED2F0A00BFCD48C16B0220DFF834C300DF3EBD31B52DED020B0446C64890ED2E0ADDED000AB4EEE00AF1EE10FAC3
:40E7800000DCA4B100BF04226946C0480068B8300AF0F6FD20B99DED000ABB4880ED2E0A00BFBB48C16B0220DFF8E8C200DF3EBD10B54FF4C471B8482CF045FFB24890F8B0
:40E7C0002800B54981F8840127F0E3FBB2498860012081F88001002081F881019FEDAF0A084680ED390A002005F08FFB01209FEDAB0AFFF7B8FF01209FEDA80AFFF78EFF14
:40E8000001209FEDA60AFFF763FF01209FEDA30AFFF738FF10BD10B5002424F0FDFF40B39F4800680078012800D128E09C4800680078022801D1142421E099480068007860
:40E84000052801D128241AE0954800680078032801D13C2413E0924800680078062801D150240CE08E4800680078082807D1642405E024F0E9FF10B1874890F885412046C1
:40E8800010BD10B5844890F8810186490978884203D0FFF7C0FF8449087010BD70B52DED028B044612F0FCF900287DD1002596E07548C03000EB8400D0ED000AB0EE600A33
:40E8C00028460FF0EFFC7048C03000EB8400D0ED000AB0EE600A28460FF0FCFA6A48C83000EB8400D0ED000AB0EE600A28460FF0FDFC6548C83000EB8400D0ED000AB0EEB0
:40E90000600A28460FF044FB5F48D03000EB8400D0ED000AB0EE600A28460FF00BFD5A48D03000EB8400D0ED000AB0EE600A28460FF08AFB5448D83000EB8400D0ED000ABB
:40E94000B0EE600A28460FF019FD4F48D83000EB8400D0ED000AB0EE600A28460FF0DDFB4949E031085D29460FF02CFD4649E231085D29460FF044FD24F04EFF08B34249EE
:40E98000E0310A5D891C095D501800EBD071491000EE101AB8EEC00AB0EE408ABCEEC80A10EE101AC8B200E01DE021460FF02CFABCEEC80A10EE101AC8B221460FF057FA9B
:40E9C0000BE03149E031085D21460FF01DFA2E49E231085D21460FF04AFA681CC5B2022DFFF666AFA3E02848C03000EB8400D0ED000AB0EE600A20460FF054FC2248C030C2
:40EA000000EB8400D0ED000AB0EE600A20460FF061FA1D48C83000EB8400D0ED000AB0EE600A20460FF062FC1748C83000EB8400D0ED000AB0EE600A20460FF0A9FA124883
:40EA4000D03000EB8400D0ED000AB0EE600A20460FF070FC0C48D03000EB8400D0ED000AB0EE600A20460FF0EFFA0748D83000EB8400D0ED000AB0EE600A20460FF07EFC33
:40EA80000148D83012E00000081F0020A4030020D03F002089E70308B00F002000000000080300202F0300202E03002000EB8400D0ED000AB0EE600A20460FF02EFBFE499B
:40EAC000085D21460FF07EFCFB49891C085D21460FF096FC24F0A0FEF0B1F7490A5D891C095D501800EBD071491000EE101AB8EEC00AB0EE408ABCEEC80A10EE101AC8B28B
:40EB000021460FF081F9BCEEC80A10EE101AC8B221460FF0ACF90AE0E749085D21460FF073F9E549891C085D21460FF0A0F9BDEC028B70BD01B500BF01226946DF4800680B
:40EB400000F5E9700AF01CFC28B99DF80000DA49E03981F8D20100BF08BD10B5032005F0D4F91FED320A002006F09BFB0120FFF7E1FFD149E03991F84200FFF78FFE172066
:40EB80001FF0FAF810BD01B5B8B000203590349033903290319030902F902E901FED410A389880ED530A1FED430A389880ED560A1FED460A389880ED540A1FED480A389831
:40EBC00080ED580A1FED4B0A389880ED550A1FED4D0A389880ED590A01203790FEE3379830F072FF9FEDB60B53EC102BCDE926019DED260B51EC100B30F05EFDCDE92C0108
:40EC000037983690389890ED6A0B8DED200B9DED2C0B53EC102B9DED200B51EC100B30F0A3FFCDE92401389890ED680B8DED1A0B9DED2C0B53EC102B9DED1A0B51EC100B52
:40EC400030F092FFCDE91C019DED2C0B53EC102B9DED1C0B51EC100B30F086FFCDE92001389890ED660B8DED140B9DED2C0B53EC102B9DED140B51EC100B30F075FFCDE973
:40EC800016019DED2C0B53EC102B9DED160B51EC100B30F069FFCDE918019DED2C0B53EC102B9DED180B51EC100B30F05DFFCDE91C01389890ED640B8DED0E0B9DED2C0B09
:40ECC00053EC102B9DED0E0B51EC100B30F04CFFCDE910019DED2C0B53EC102B9DED100B51EC100B30F040FFCDE912019DED2C0B53EC102B9DED120B51EC100B30F034FF80
:40ED0000CDE914019DED2C0B53EC102B9DED140B51EC100B30F028FFCDE91801389890ED620B8DED080B9DED2C0B53EC102B9DED080B51EC100B30F017FFCDE90A019DEDBE
:40ED40002C0B53EC102B9DED0A0B51EC100B30F00BFFCDE90C019DED2C0B53EC102B9DED0C0B51EC100B30F0FFFECDE90E019DED2C0B53EC102B9DED0E0B51EC100B30F092
:40ED8000F3FECDE910019DED2C0B53EC102B9DED100B51EC100B30F0E7FECDE91401389890ED600B8DED020B9DED2C0B53EC102B9DED020B51EC100B30F0D6FECDE904017B
:40EDC0009DED2C0B53EC102B9DED040B51EC100B30F0CAFECDE906019DED2C0B53EC102B9DED060B51EC100B30F0BEFECDE908019DED2C0B53EC102B9DED080B51EC100B49
:40EE000030F0B2FECDE90A019DED2C0B53EC102B9DED0A0B51EC100B30F0A6FECDE90C019DED2C0B53EC102B9DED0C0B51EC100B30F09AFECDE91001389890ED5E0B8DEDA5
:40EE4000000B9DED2C0B53EC102B9DED000B51EC100B30F089FECDE902019DED2C0B53EC102B9DED020B51EC100B30F07DFECDE904019DED2C0B53EC102B9DED040B51EC6E
:40EE8000100B30F071FECDE906019DED2C0B53EC102B9DED060B51EC100B30F065FECDE908019DED2C0B53EC102B9DED080B51EC100B30F059FE07E0E81F0020A4030020FF
:40EEC0000000000000002440CDE90A019DED2C0B53EC102B9DED0A0B51EC100B30F044FECDE90C019DED2C0B53EC102B9DED0C0B51EC100B30F038FECDE90E019DED100BA2
:40EF000053EC102B9DED0E0B51EC100B30F018FBCDE912019DED140B53EC102B9DED120B51EC100B30F00CFBCDE916019DED180B53EC102B9DED160B51EC100B30F000FB05
:40EF4000CDE91A019DED1C0B53EC102B9DED1A0B51EC100B30F0F4FACDE91E019DED200B53EC102B9DED1E0B51EC100B30F0E8FACDE922019DED240B53EC102B9DED220BAC
:40EF800051EC100B30F0DCFACDE92601389890ED6C0B8DED240B9DED240B53EC102B9DED260B51EC100B30F0CBFACDE92A01389890ED7A0B8DED200B9DED2C0B53EC102BFB
:40EFC0009DED200B51EC100B30F0CEFDCDE92401389890ED780B8DED1A0B9DED2C0B53EC102B9DED1A0B51EC100B30F0BDFDCDE91C019DED2C0B53EC102B9DED1C0B51ECB7
:40F00000100B30F0B1FDCDE92001389890ED760B8DED140B9DED2C0B53EC102B9DED140B51EC100B30F0A0FDCDE916019DED2C0B53EC102B9DED160B51EC100B30F094FDF4
:40F04000CDE918019DED2C0B53EC102B9DED180B51EC100B30F088FDCDE91C01389890ED740B8DED0E0B9DED2C0B53EC102B9DED0E0B51EC100B30F077FDCDE910019DED8F
:40F080002C0B53EC102B9DED100B51EC100B30F06BFDCDE912019DED2C0B53EC102B9DED120B51EC100B30F05FFDCDE914019DED2C0B53EC102B9DED140B51EC100B30F074
:40F0C00053FDCDE91801389890ED720B8DED080B9DED2C0B53EC102B9DED080B51EC100B30F042FDCDE90A019DED2C0B53EC102B9DED0A0B51EC100B30F036FDCDE90C0102
:40F100009DED2C0B53EC102B9DED0C0B51EC100B30F02AFDCDE90E019DED2C0B53EC102B9DED0E0B51EC100B30F01EFDCDE910019DED2C0B53EC102B9DED100B51EC100B1F
:40F1400030F012FDCDE91401389890ED700B8DED020B9DED2C0B53EC102B9DED020B51EC100B30F001FDCDE904019DED2C0B53EC102B9DED040B51EC100B30F0F5FCCDE950
:40F1800006019DED2C0B53EC102B9DED060B51EC100B30F0E9FCCDE908019DED2C0B53EC102B9DED080B51EC100B30F0DDFCCDE90A019DED2C0B53EC102B9DED0A0B51EC55
:40F1C000100B30F0D1FCCDE90C019DED2C0B53EC102B9DED0C0B51EC100B30F0C5FCCDE91001389890ED6E0B8DED000B9DED2C0B53EC102B9DED000B51EC100B30F0B4FC25
:40F20000CDE902019DED2C0B53EC102B9DED020B51EC100B30F0A8FCCDE904019DED2C0B53EC102B9DED040B51EC100B30F09CFCCDE906019DED2C0B53EC102B9DED060BF5
:40F2400051EC100B30F090FCCDE908019DED2C0B53EC102B9DED080B51EC100B30F084FCCDE90A019DED2C0B53EC102B9DED0A0B51EC100B30F078FCCDE90C019DED2C0BF0
:40F2800053EC102B9DED0C0B51EC100B30F06CFCCDE90E019DED100B53EC102B9DED0E0B51EC100B30F04CF9CDE912019DED140B53EC102B9DED120B51EC100B30F040F9CB
:40F2C000CDE916019DED180B53EC102B9DED160B51EC100B30F034F9CDE91A019DED1C0B53EC102B9DED1A0B51EC100B30F028F9CDE91E019DED200B53EC102B9DED1E0BCF
:40F3000051EC100B30F01CF9CDE922019DED240B53EC102B9DED220B51EC100B30F010F9CDE92601389890ED7C0B8DED240B9DED240B53EC102B9DED260B51EC100B30F03C
:40F34000FFF8CDE928016421369890FBF1F201FB120008BB9DED2A0B51EC100B30F0BEF801466422369890FBF2F2521E389800F5027040F822109DED280B51EC100B30F0E8
:40F38000ADF801466422369890FBF2F2521E389800F50C7040F82210389890ED000AB1EE400A8DED250A259830F0D4FECDE926019DED2A0B53EC102B9DED260B51EC100BC2
:40F3C00030F0D0FC2AD23598401C80B235909DED350AB8EE400ADFEDFE0A00E028E2B4EEE00AF1EE10FA1BDD389890ED530AB5EEC00AF1EE10FA13D19DED2C0B51EC100B24
:40F4000030F06CF800EE100AB1EE400AF3EE040A30EE200A389880ED530A01E000203590389890ED000AB1EE400A8DED250A259830F090FECDE926019DED2A0B53EC102B56
:40F440009DED260B51EC100B30F08CFC26D23498401C80B234909DED340AB8EE400ADFEDDC0AB4EEE00AF1EE10FA19DD9DED2C0B51EC100B30F032F800EE100AF1EE400A52
:40F480009DED340AB8EE400AB2EE041AC0EE011A30EEA10A389880ED520A01E000203490389890ED010AB1EE400A8DED250A259830F050FECDE926019DED2A0B53EC102BBB
:40F4C0009DED260B51EC100B30F04CFC28D23198401C80B231909DED310AB8EE400AF1EE040AB4EEE00AF1EE10FA1BDD389890ED540AB5EEC00AF1EE10FA13D19DED2C0BCA
:40F5000051EC100B2FF0EAFF00EE100AB1EE400AF6EE000A30EE200A389880ED540A01E000203190389890ED030AB1EE400A8DED250A259830F00EFECDE926019DED2A0B76
:40F5400053EC102B9DED260B51EC100B30F00AFC28D22F98401C80B22F909DED2F0AB8EE400AF1EE040AB4EEE00AF1EE10FA1BDD389890ED550AB5EEC00AF1EE10FA13D1D7
:40F580009DED2C0B51EC100B2FF0A8FF00EE100AB1EE400AF6EE000A30EE200A389880ED550A01E000202F9038980068259030F0D1FDCDE926019DED280B53EC102B9DED70
:40F5C000260B51EC100B30F093FA26D23398401C80B233909DED330AB8EE400ADFED7C0AB4EEE00AF1EE10FA19DD389890ED560AB5EEC00AF1EE10FA11D19DED2C0B51EC6A
:40F60000100B2FF06BFF00EE100AF3EE040A30EE600A389880ED560A01E00020339038980068259030F096FDCDE926019DED280B53EC102B9DED260B51EC100B30F058FA0D
:40F6400024D23298401C80B232909DED320AB8EE400ADFED5F0AB4EEE00AF1EE10FA17DD9DED2C0B51EC100B2FF038FF00EE900A9DED320AB8EE400AB2EE041AC0EE011AF2
:40F6800030EEE10A389880ED570A01E00020329038984068259030F05DFDCDE926019DED280B53EC102B9DED260B51EC100B30F01FFA26D23098401C80B230909DED300A07
:40F6C000B8EE400AF1EE040AB4EEE00AF1EE10FA19DD389890ED580AB5EEC00AF1EE10FA11D19DED2C0B51EC100B2FF0F7FE00EE100AF6EE000A30EE600A389880ED580A91
:40F7000001E0002030903898C068259030F022FDCDE926019DED280B53EC102B9DED260B51EC100B30F0E4F926D22E98401C80B22E909DED2E0AB8EE400AF1EE040AB4EEAD
:40F74000E00AF1EE10FA19DD389890ED590AB5EEC00AF1EE10FA11D19DED2C0B51EC100B2FF0BCFE00EE100AF6EE000A30EE600A389880ED590A01E000202E90389890EDBC
:40F780005C0AB1EE400A8DED250A259830F0E2FCCDE926019DED2A0B53EC102B9DED260B51EC100B30F0DEFA19D29DED2A0B51EC100B2FF093FE3899C1F870019DED2C0B07
:40F7C00051EC100B2FF08AFE00EE100A02E0000000004843B1EE400A389880ED5A0A3898D0F87401259030F0B5FCCDE926019DED280B53EC102B9DED260B51EC100B30F031
:40F8000077F911D29DED280B51EC100B2FF066FE3899C1F874019DED2C0B51EC100B2FF05DFE3899C1F86C013798401C80B237903798B0F57A7F7FF7D2A9389890ED540A27
:40F84000B5EEC00AF1EE10FA0BD0389890ED540A80ED5A0A389890ED010AB1EE400A80ED5C0A389890ED580AB5EEC00AF1EE10FA09D0389890ED580A80ED5B0A389890ED1B
:40F88000010A80ED5D0A389890ED530AB5EEC00AF1EE10FA61D0389890ED560AB5EEC00AF1EE10FA59D0389890ED5A0AD0ED530AB7EE001A70EEC10AB4EEE00AF1EE10FAE4
:40F8C0004BDC389890ED5B0AD0ED560AB7EE001A70EE810AB4EEE00AF1EE10FA3DD3389890ED530AD0ED520A30EE600A8DED230A239830F02FFCCDE924019DED240B2DF03C
:40F9000003F88DED260B9FEDFD0B53EC102B9DED260B51EC100B30F025FA1ED3389890ED560AD0ED570A30EE600A8DED230A239830F010FCCDE924019DED240B2CF0E4FF5C
:40F940008DED260B9FEDED0B53EC102B9DED260B51EC100B30F006FA03D22320E94981F87E01389890ED550AB5EEC00AF1EE10FA04D19FEDE50A389880ED550A389890ED2E
:40F98000590AB5EEC00AF1EE10FA04D19FEDDF0A389880ED590A39B000BD70B52DED088B064600246FE09FEDDA0BB0EE408AF0EE608A9FEDD70BB0EE409AF0EE609A0025E9
:40F9C00051E006F1400000EB850090ED000A10EE101A084630F0BEFB41EC1B0B04EB440000EBC400CC4901EBC00000EBC50090ED001BB0EE410AF0EE610A53EC102B51EC32
:40FA00001B0B30F0B1F853EC182B2FF099FD41EC180B06F16C0000EB850090ED000A10EE101A084630F096FB41EC1B0B04EB440000EBC400B84901EBC00000EBC50090EDC0
:40FA4000001BB0EE410AF0EE610A53EC102B51EC1B0B30F089F853EC192B2FF071FD41EC190B681CC5B20B2DABDB06F5BC7000EBC40080ED008B06F5DC7000EBC40080ED70
:40FA8000009B601CC4B2082C8DDBBDEC088B70BDA24A92F82810022914D19FEDA10A80ED000A9FEDA00A80ED010A9FED9F0A80ED020A9FED9E0A80ED030A9FED9D0A80ED9E
:40FAC000040A6FE00D2914D19FED950A80ED000A9FED940A80ED010A9FED930A80ED020A9FED920A80ED030A9FED910A80ED040A58E00C2914D19FED8A0A80ED000A9FEDEF
:40FB0000890A80ED010A9FED880A80ED020A9FED870A80ED030A9FED860A80ED040A41E0032914D19FED7E0A80ED000A9FED7D0A80ED010A9FED7C0A80ED020A9FED7B0A11
:40FB400080ED030A9FED7A0A80ED040A2AE0012914D19FED730A80ED000A9FED720A80ED010A9FED710A80ED020A9FED720A80ED030A9FED710A80ED040A13E09FED680AF2
:40FB800080ED000A9FED670A80ED010A9FED660A80ED020A9FED670A80ED030A9FED660A80ED040A704770B52DED028B04466348FFF76EFF6148FFF7F0FE6048FEF7E3FF0F
:40FBC0005E48D0ED550AB0EE600A20460EF03CFA5A48D0ED550AB0EE600A20460EF0AAFB5648D0ED590AB0EE600A20460EF095FA5248D0ED590AB0EE600A20460EF0BEFB3A
:40FC00004E4890ED000AFFEE000A20EE200AB0EE408A90ED5A0AD0ED530A30EE600AD0ED5C0A70EEC80A80EE801A80ED7E1AD0ED7E0A90ED531AB0EE480A00EEC10A80EDE8
:40FC40007F0A90ED000AB0EE408A90ED5B0AD0ED560A30EE600AD0ED5D0A70EEC80A80EE801A80ED801AD0ED800A90ED561AB0EE480A00EEC10A80ED810A90ED040AD0ED05
:40FC80007E0A80EE201AB0EE418A9FED200A28EE000AB0EE408A9FED2A0AB4EEC08AF1EE10FA04DD9FED260AB0EE408A0AE0B7EE000AB4EEC08AF1EE10FA03D2B7EE000AE1
:40FCC000B0EE408AB6EE000A38EE000ABCEEC00A10EE100AC5B2214628460EF095F8214628460EF06FFB154890ED040AD0ED800A80EE201AB0EE418A24E0000000000000DA
:40FD00000000F03FB00F00200000C8C20000C842000000000000000048000020081F002035FA0E3DC2B8323E00000000C2B8B23E8FDAA53B920A063F88C3643B3811002027
:40FD400000007F431FED0F0A28EE000AB0EE408A1FED050AB4EEC08AF1EE10FA04DD1FED080AB0EE408A0AE0B7EE000AB4EEC08AF1EE10FA03D2B7EE000AB0EE408AB6EEBF
:40FD8000000A38EE000ABCEEC00A10EE100AC5B2214628460EF06BF8214628460EF030FBBDEC028B70BD70B502460C4600201FED222AF0EE420A1FED242AB0EE421A1FEDAE
:40FDC000262AB0EE420A1FED282AF0EE421A64B902F1400102F16C031FED2C2AB0EE420A9FEDF92AF0EE421A1CE0012C0CD102F1980102F1C403B0EE002AB0EE420AB7EEA6
:40FE0000002AF0EE421A0DE0022C0BD102F1F00102F58E73B3EE042AB0EE420AB2EE042AF0EE421AB5EEC00AF1EE10FA7EDD1FED422A81ED002A1FED442A83ED002A1FEDE9
:40FE4000462A82ED052A012082E002EE100AB8EE422AF2EE042A22EE222A02F1140505EB800585ED002A451ED84E06EB850595ED002AB5EEC02AF1EE10FA06DD1FED562AB9
:40FE800001EB800585ED002A09E0451ECF4E06EB850595ED002A01EB800585ED002A451ECA4E2C3606EB850595ED002AB5EEC02AF1EE10FA06D21FED642A03EB800585EDC7
:40FEC000002A0AE0451EC14E2C3606EB850595ED002A03EB800585ED002A01EB800595ED002A451E01EB8505D5ED002A32EE622AF0EE420A03EB800595ED002A451E03EBBC
:40FF00008505D5ED002A32EE622AB0EE421AB1EE402AF4EEC20AF1EE10FA12D3F4EEE10AF1EE10FA0DDCB4EEC01A00E013E0F1EE10FA06DCB1EE612AB4EEC21AF1EE10FAD6
:40FF400004D22325A14E243E86F87E51451CE8B20B28FFF67AAF70BD10B500219C48FFF722FF01219A48FFF71EFF02219848FFF71AFF10BD10B5974890F82840042C17D0CA
:40FF800006DC012C0DD0022C08D0032C17D104E00C2C05D00D2C12D101E000BF00BF00BF00BF9FED8D0A8948243880ED390A0DE09FED8A0A8548243880ED390A06E01FED76
:40FFC000A60A8248243880ED390A00BF00BF13F037FAB5EEC00AF1EE10FA09DD7B48243890ED390AFFEE000A20EE200A80ED390A10BD73B52DED020B04460D460A2C21D2ED
:020000040801F1
:4000000000BF05EB85027649096801F5177101EBC20101EB84000422694609F0B1F950B99DED000A05EB85016E4800EBC10000EB840080ED000A00BF6B48C16B0220DFF853
:40004000ACC100DF7FBD10B5FAF771FE10BD73B52DED020B04460D460A2C21D200BF05EB85025F49096801F59A7101EBC20101EB84000422694609F083F950B99DED000A9B
:4000800005EB85015A4800EBC10000EB840080ED000A00BF5448C16B0220DFF850C100DF7FBD73B52DED020B04460D460A2C22D200BF05EB85024A49096801F5037101EB44
:4000C000C20101EB84000422694609F059F958B99DED000A05EB85014248503800EBC10000EB840080ED000A00BF3F48C16B0220DFF8F8C000DF7FBD10B5FAF718FE10BD17
:4001000073B52DED020B04460D460A2C21D200BF05EB850232490968E43101EBC20101EB84000422694609F02BF958B99DED000A05EB85012E48503800EBC10000EB84002E
:4001400080ED000A00BF2848C16B0220DFF89CC000DF7FBD1F4A92F82810042917D006DC01290DD0022908D0032917D104E00C2905D00D2912D101E000BF00BF00BF00BF1A
:400180009FED150A114A243A82ED390A0DE09FED130A0E4A243A82ED390A06E09FED150A0A4A243A82ED390A00BF00BF032809D1064A243A92ED390AFFEE000A20EE200A14
:4001C00082ED390A70470000920A863ED40F002038110020081F002000008C4200004842A403002064210020D03F002089E703083C20002000000000FE4A92F82810062960
:4002000005D19FEDFD0AFD4A82ED390A0CE0042905D11FED0E0AF94A82ED390A04E01FED120AF64A82ED390A062808D1F34A92ED390AFFEE000A20EE200A82ED390A7047B8
:40024000B5EEC00AF1EE10FA01D2012070470020FCE7B5EEC00AF1EE10FA01DD012070470020FCE72DE9F04106460C4615460427E04890F828802868A0B925F08AFE28609A
:400280000020DF4908709FEDDF0A13F0F7F920B1BFEE000ADC4880ED000A13F0D1F8DB4880ED000AB8F1040F1FD009DCB8F1010F11D0B8F1020F0BD0B8F1030F1FD106E03D
:4002C000B8F10C0F06D0B8F10D0F18D101E000BF00BF00BF00BFCC4890ED000A5FED420A20EE200A84ED000A13E0C74890ED000A5FED460A20EE200A84ED000A09E0C24828
:4003000090ED000A5FED450A20EE200A84ED000A00BF00BF41F28831286825F040FE20B1212030700127002595E040F6C411286825F035FEE0B1B2480078C8B99FEDB40A76
:4003400013F09CF920B99FEDB20A13F03CF978B10120AB490870AC4890ED000AFFEE000A20EE200A80ED000A25F013FE286072E0D4ED000AB0EE600AFFF76BFF68B113F066
:400380005FF8A248D0ED000A30EE600ADFEDA00AB4EEE00AF1EE10FA14DCD4ED000AB0EE600AFFF74DFFA8B113F04AF89748D0ED000A30EE600ADFED970AB4EEE00AF1EE19
:4003C00010FA07D203271FED750A84ED000A0020286040E0D4ED000AB0EE600AFFF739FF68B113F02DF88948D0ED000A30EE600ADFED880AB4EEE00AF1EE10FA14D3D4ED45
:40040000000AB0EE600AFFF71BFF20B313F018F87E48D0ED000A30EE600ADFED7D0AB4EEE00AF1EE10FA16DD724890F89C0018B90120F9F7FFFE07E06E4890F89C0001283D
:4004400002D10020F9F7F6FE03271FED960A84ED000A002028603846BDE8F08110B52DED048B0424654890F880010A287DD2DFE800F00506FD477CFC487CFBFA00BF5F48AE
:4004800090F8810120B1102821D0112835D110E011205A4981F8810112F0D2FF574880ED080AB6EE000A80ED390A00205349086024E0524A02F1E40101F19A00FFF7D2FEFD
:4004C000032803D110204D4981F8810116E006204A4981F88001022081F881010A2081F887010020086012F0ABFF444880ED080AB6EE000A80ED390A00E000BF00BF1CE351
:4005000000BF3E4890F88101801E0B2870D2DFE800F0066FB6FC5EDE6F6F6F6F8F003748006870B925F035FD34490860084690F885010A2805DD084690F88501C01F81F894
:4005400085012E4991F88001FFF756FE2B4908684FF47A6125F023FDB0B112F071FF2748D0ED080A30EEC00A00E0F7E3B0EEC00ADFED290AB4EEE00AF1EE10FA04D221204D
:400580001E4981F87E0121E09FED210A13F076F820B11A4890F88001032809D09FED1C0A13F011F890B1154890F8800106280DD1B6EE000A114880ED390A06200F4981F854
:4005C00081010C2081F8830100200860B4E2B6EE000A0A4880ED390A006818B925F0D9FC0649086005490868C82125F0D8FC15E0A1E20000081F002000002042B00F002018
:4006000031030020C2B8323E3403002038030020C2B8B23DC2B8B2BD35FA0E3D38B1FE4890F88301FC4981F881010020086083E2F94991F88001FFF78DFDF748006818B952
:4006400025F0A7FCF4490860F34908684FF4FA7125F0A5FC90B1B6EE000AEF4880ED390A0620ED4903E0CEE3E4E367E267E281F8810100200860042081F883015CE212F00A
:40068000DFFEF0EE409A4FF6FF71E44813F074FEE148006818B925F07CFCDF490860DE4908684FF4FA7125F07AFC78B1DA4890ED510A80ED080A0720D74981F881010020FC
:4006C000086001F5807000214164816434E2D248006818B925F05DFCCF490860CE4890F8870100EB8000400000EE100AB8EEC00AC94880ED390A90F8800103280AD1C64883
:4007000090ED390AFFEE000A00E044E020EE200A80ED390A1FED420A12F0B0FF20B1BE4890F88001062809D01FED470A12F04BFFB0B1B94890F88001032811D10220B649E4
:4007400081F8810101F5807000214164816412F077FEB14880ED080A0020AF49086019E0AD4908684FF4FA7125F019FC90B1B6EE000AA94880ED390A0620A74981F88101A6
:40078000086825F02EFCA449C86100200860052081F88301D0E112F053FEF0EE409A4FF6FF719E4813F0E8FD9B48006818B925F0F0FB99490860984908684FF4FA7125F011
:4007C000EEFB00287DD0944890ED510AD0ED080A30EE608AB0EEC80AF0EE409A12F0F3FE20B18D4890F8800103281FD01FED780A12F0E9FE20B1884890F88001032815D0FB
:40080000B0EEC80AF0EE409A12F038FF20B1824890F88001062809D01FED830A12F02EFF98B17D4890F8800106280ED102207A4981F88101084690ED510A80ED080A00F546
:4008400080700021416481640DE00720724981F88101084690ED510A80ED080A00F580700021416481646C4890F88701401E6A4981F88701084690F8800103285AD108460D
:4008800090ED070AF8EE400A9FED651A80EE810AC8EE000A90F88711243000EB8100C0ED000A604A92F842105B4A92F8870192F88731243202EB8302D2ED000AB0EE600A07
:4008C00000E037E1FFF71CFC534890F88711243000EB8100D0ED000AB0EE600A0020FDF742FFFFF709FC4C4890F887117C3000EB810080ED000A4B4A92F84210464A92F88A
:40090000870192F887317C3202EB8302D2ED000AB0EE600AFFF7C5FB3F4890F887117C3000EB8100D0ED000AB0EE600A0020FDF7CFFE57E0384890ED070AF8EE400A9FEDD6
:40094000381A80EE810AC8EE000A90F88711503000EB8100C0ED000A324A92F842102E4A92F8870192F88731503202EB8302D2ED000AB0EE600AFFF76AFB274890F88711D6
:40098000503000EB8100D0ED000AB0EE600A0020FDF7C4FEFFF757FB1F4890F88711A83000EB810080ED000A1E4A92F842101A4A92F8870192F88731A83202EB8302D2ED15
:4009C000000AB0EE600AFFF714FB134890F88711A83000EB8100D0ED000AB0EE600A0020FDF776FE0C4890F88701002813D10A4890F88001062817D10320074981F880017C
:400A0000022081F88101B6EE000A084680ED390A0A2081F887018AE0B00F0020F410002000007A44081F0020B7EE000AF94880ED370A0920F849087026E0F6485030F649CD
:400A400091F9001000EB810090ED000ADFEDF30AB4EEE00AF1EE10FA10D2EF4890F9000000EE100AB8EEC00AF2EE040A20EE200AE84880ED370AFF20E7490870E648007820
:400A8000401E40B2E4490870E34890F900000028D3DAB7EE000ADF4880ED360A0920DE49087026E0DB482430DB4991F9001000EB810090ED000ADFEDDA0AB4EEE00AF1EE24
:400AC00010FA10DDD44890F9000000EE100AB8EEC00AFAEE040A20EE200ACE4880ED360AFF20CD490870CC480078401E40B2CA490870C94890F900000028D3DAC54890EDE4
:400B0000370A80ED380A0520C24981F880010D2081F88101B6EE000A084680ED390A002081F887019FEDBF0A084680ED350A0020B849086000E000BF00BF99E100BFB5483A
:400B400090F8810106281CD00D2802D00E287DD131E0FFF70FFA9FEDB10A12F064FD78B1B6EE000AAB4880ED390A0620A94981F881010E2081F8830125F00BFAA5490860E4
:400B80003FE1B6EE000AA34880ED390A014608684FF4FA7125F003FA60B19E4890F883019C4981F881010020086012F049FC994880ED080A25E1974890F88001052807D150
:400BC00012F03EFC9348D0ED080A70EE608A06E012F036FC8F48D0ED080A70EEC08A8D48006818B925F0D5F98A4908609FED8E0AF4EEC08AF1EE10FA7EDD864890ED350A15
:400C0000D0ED390A30EE200A80ED350A90F88701401C804981F88701B6EE000A084680ED390A0D2081F88101086825F0DAF900EE100AB8EE400A5FED860A80EE209A7548A5
:400C400090F88001052818D1724800E0D8E090ED380A30EE090AF1EE040A30EE600A80ED380A90ED380AB5EEC00AF1EE10FA1AD29FED6C0A80ED380A15E0664890ED380ADB
:400C800030EE490AF1EE040A30EE200A80ED380A90ED380AB5EEC00AF1EE10FA03DD9FED610A80ED380A5B4890F88701032839DB5848D0ED350A90F8870100EE100AB8EEF8
:400CC000400A80EE801A534880ED351A90F88001052828D1554991F842004E49D1ED350AB0EE600A0DF002FB9FED4E0A494880ED350AB6EE000A00E031E080ED390A00208D
:400D0000444981F88701022081F880010D2081F8810125F03EF93F490860084690ED360A80ED380A6BE0414991F842003949D1ED350AB0EE600A0DF0B5FA9FED3A0A3548CB
:400D400080ED350AB6EE000A80ED390A0820314981F880010F2081F8810150E087E02D4890ED390AB0EEC00ADFED310AB4EEE00AF1EE10FA07DA0146086825F032F94EF6D7
:400D80006021884207D92120224981F87E01092081F8800133E01F4890F88001022817D11C49086825F01DF900EE100AB8EE400AFFEE000A60EE200A1FEDE71A80EE810A3F
:400DC0001448D0ED380A30EE200A80ED390A16E01049086825F005F900EE100AB8EE400AF7EE000A60EE200A1FEDF31A80EE810A0848D0ED380A30EE200A80ED390A00E036
:400E000000BF00BF34E002249FED060A014880ED390A2DE0B00F00203003002035FA0E3D35FA0EBD0000000035FA8E3C081F002000008C42FFF790F8FE4890F87E0120B108
:400E40000920FC4981F8800110E0FB4991F84200FEF7A9FE1020F74981F8810103241FED0F0A084680ED390AFDF777FE00E000BF00BFF04890F88201EE4991F88111884294
:400E800014D0EC4890F88501401CEA4981F88501084690F88501642802DD642081F88501E44890F88101E34981F88201E14890ED390AB5EEC00AF1EE10FA08D0D0ED390ABF
:400EC000B0EE600A01210846F9F754FA08E0D948D0ED390AB0EE600A00210120F9F74AFA2046BDEC048B10BD002070471FED330AD04880ED5B0A1FED350A80ED5D0A1FED15
:400F0000370A80ED550A1FED390A80ED530A1FED3B0A80ED590A1FED3D0A80ED570A704770B52DED048B0446F0EE408AB0EE609AF0EE419A0D46C04890F8300070280CD1F9
:400F4000F7EE000A80EEA80ADFEDBC0A89EE201A20EE010A20EE298A60E0B74890F830000A280CD1F0EE000A80EEA80ADFEDB30A89EE201A20EE010A20EE298A4EE0A81E2F
:400F80000C283DD2DFE800F02D3C063C13203C3C3C3C2F2EF0EE080A80EEA80ADFEDA70A89EE201A20EE010A20EE298A35E0DFEDA40A80EEA80ADFEDA10A89EE201A20EE0F
:400FC000010A20EE298A28E0DFED9E0A80EEA80ADFED9A0A89EE201A20EE010A20EE298A1BE000BF00BFDFED980A80EEA80ADFED930A89EE201A20EE010A20EE298A0CE0A7
:40100000DFED920A80EEA80ADFED8C0A89EE201A20EE010A20EE298A00BF00BFB2EE040AB4EEC08AF1EE10FA04D2B2EE040AB0EE408A0AE09FED860AB4EEC08AF1EE10FA73
:4010400003DD9FED830AB0EE408A012C0AD17A4A92F84210BCEEC80A10EE102AD0B20DF0B1F909E0744A92F84210BCEEC80A10EE102AD0B20DF0C4F9BDEC048B70BD00B5FD
:401080002DED028B95B06B4890ED390A8DED140A24F07FFF0E9004200C9012F050F9654880ED3B0AC068634948610846006988616848007826F002FF5E49C86024F069FFF8
:4010C0005C490861084680690B9024F08AFF4FF47A71B1FBF0F00F905648C06855494969401A00EE100AB8EEC00AF7EE000A20EE200A9FED591AC0EE010A9DED0F0AB8EE0A
:40110000C00A20EE800A8DED130A052153489DED130A13F031F90521504808309DED140A13F02AF91CF0D4F88DED0B0A1E214B4818389DED0B0A13F01FF9494890ED000A02
:401140008DED0B0A1E21454820389DED0B0A13F013F9434890ED000A364880ED3A0A414800780EF019FA8DED0B0A05213B4808389DED0B0A13F000F93B4800780EF0C9FBEB
:401180008DED050A05982EF0E5FFCDE906019DED060B2BF0B9FB8DED080B9DED080B51EC100B2EF09BF905210B902C4810389DED0B0A13F0E1F82048B0F8BE014FF496719B
:4011C00090FBF1F000EE100AB8EEC00A8DED0D0A194890F82800062850D0174890F8280007284BD0134890F88001042804D0114890F88001072841D10E4890ED5D0ADFEDB5
:401200001B0AB4EEE00AF1EE10FA38DD90ED5B1A9DED0D0AF2EE040AF1EE041A41EEC00AB4EEE01AF1EE10FA28D20920014981F880011DE0B00F0020081F002000007A44BB
:40124000CDCC4C406666A6408FC2753E9A99193F00007F43D806002052EC2F451C110020DC42002093060020E406002000004842242081F87E01002081F881016EE0FE48D3
:4012800090ED5D0ADFEDFD0AB4EEE00AF1EE10FA19D290ED5B1A9DED0D0AFAEE040AF1EE041A41EE800AB4EEE01AF1EE10FA55DD0920F14981F88001242081F87E01002068
:4012C00081F881014AE0EC48D0F8740107902EF041FFCDE908019DED080B2BF015FB8DED0A0B9FEDE70B53EC102B9DED0A0B51EC100B2EF039FB31D1DDED0D0AB1EE040A7C
:40130000B1EE041A01EE200A8DED070A07982EF021FFCDE90A01D848D0F86C0105902EF019FFCDE906019DED060B2BF0EDFA8DED080B9DED0A0B53EC102B9DED080B51ECB4
:40134000100B2EF00FFD09D20920CB4981F88001242081F87E01002081F88101C64890F88101062813D1C448806801460B900E9824F046FEC0494968884241F2A783BE48DA
:4013800090F88301BC4981F8810101F09FBBBA4890F880010A2881F09783DFE810F030000A0040002804950B34020807950B8B0B760BB14890F87F0180B1AF4890F87F01D4
:4013C000AD4981F88001062081F88101002081F88301192048600E9888600EE00020A64981F88001062081F88101002081F883014FF47A7048600E98886001F066BB022084
:401400009D4981F88001062081F88101002081F883014FF47A7048600E988860EDE7964890F88001944981F87F01084690F8810108287CD003DC38B1052879D15AE109281B
:4014400077D00B28F9D10BE006208B4981F881010B2081F88301192048600E988860D0E18548806801460B900E9824F0C9FD41F28831884207D909207F4981F88001262022
:4014800081F87E0170E0804890F8280006280ED07D4890F82800072809D0774890ED3B0ADFED7A0AB4EEE00AF1EE10FA13DC764890F82800062804D0734890F828000728A4
:4014C0000FD16D4890ED3B0ADFED710AB4EEE00AF1EE10FA05DDBBEE0E0A674880ED390A42E0694890F8280006280ED0664890F82800072809D0604890ED3B0ADFED650A3D
:40150000B4EEE00AF1EE10FA17D35F4890F82800062804D05C4890F82800072813D1564890ED3B0ADFED5C0AB4EEE00A02E034E060E11AE0F1EE10FA05D2B3EE0E0A4E482E
:4015400080ED390A10E006204B4981F88101092081F883014FF47A7048600E9888609FED4F0A084680ED390A4BE10620424981F88101082081F88301192048600E9888603E
:40158000BAEE000A084680ED390A4548007826F095FC3949C1F82C0133E13B4890F82800062804D0384890F82800072810D13248C0683149D1F82C11401A00EE100AB8EEB4
:4015C000C00ADFED380AB4EEE00AF1EE10FA31D32D4890F830000A2800D010E02648C0682549D1F82C11401A00EE100AB8EEC00ADFED2D0AB4EEE00AF1EE10FA1AD32248D0
:4016000090F82800062851D01F4890F8280007284CD01948C0681849D1F82C11401A00EE100AB8EEC00ADFED1F0AB4EEE00AF1EE10FA3BD2144890F842000B909DED140AA7
:401640000CF030FE06200C4981F88101052081F883014FF47A7048600E9888609DED140A084680ED390A0E48007826F027FC0249C1F82C013DE00000B00F0020000048C261
:401680000000000000002040081F0020CDCCCC3CCDCC4C3DCDCCCCBCCDCC4CBD00000000D80600206CE7DBC57390EAC4F74890ED390A5FED0E0AB4EEE00AF1EE10FA0BD8A0
:4016C0001FED0A0A80ED390A0920F04981F88001272081F87E010CE09DED140ADFEDEC0A30EE600A8DED140A9DED140AE74880ED390A86E0E548D0ED390A9FEDE61A80EEF5
:40170000810A8DED010A01982EF024FDCDE902019DED020B2BF0F8F88DED060BDB48D0F8640103902EF016FDCDE904019DED060B53EC102B9DED040B51EC100B2EF014FADA
:401740009FEDD50B53EC102BCDE908019DED080B51EC100B2DF0B0FFCDE90A019DED0A0B51EC100B2DF0BAFEC849C1F8FC00084690ED570ADFEDCA0A80EE201A80ED431A72
:40178000C84890F830000A2804D1B3EE090A8DED100A03E0B1EE040A8DED100A9DED100ADFEDC10A80EE201A9FEDC00A21EE000ABDEEC00AB8EEC00AB44880ED470AB0F855
:4017C0007C0140F00400B149A1F87C01052081F88001062081F88101002081F883014FF47A7048600E9888601FED540A084680ED390A06E00020A549A1F87C0181F88001FC
:4018000000BF00BFF9E5A14890F880019F4981F87F01084690F8810108287CD003DC38B1052879D15AE1092877D00B28F9D10BE00620964981F881010B2081F8830119206A
:4018400048600E988860D0E19048806801460B900E9824F0D5FB41F28831884207D909208A4981F88001282081F87E0170E08D4890F8280006280ED08A4890F828000728F7
:4018800009D0824890ED3B0A5FED800AB4EEE00AF1EE10FA13DC834890F82800062804D0804890F8280007280FD1784890ED3B0A5FED890AB4EEE00AF1EE10FA05DDBBEE24
:4018C0000E0A724880ED390A42E0764890F8280006280ED0734890F82800072809D06B4890ED3B0A5FED950AB4EEE00AF1EE10FA17D36C4890F82800062804D0694890F8F9
:401900002800072813D1614890ED3B0A5FED9E0AB4EEE00A02E034E060E11AE0F1EE10FA05D2B3EE0E0A594880ED390A10E00620564981F88101092081F883014FF47A7083
:4019400048600E9888601FEDAB0A084680ED390A4BE106204D4981F88101082081F88301192048600E988860B2EE000A084680ED390A4F48007826F0A1FA4449C1F82C0120
:4019800033E1484890F82800062804D0454890F82800072810D13D48C0683C49D1F82C11401A00EE100AB8EEC00ADFED420AB4EEE00AF1EE10FA31DC3A4890F830000A2874
:4019C00000D010E03148C0683049D1F82C11401A00EE100AB8EEC00ADFED370AB4EEE00AF1EE10FA1ADC2F4890F82800062836D02C4890F82800072831D02448C06823490E
:401A0000D1F82C11401A00EE100AB8EEC00ADFED290AB4EEE00AF1EE10FA20DD214890F842000B909DED140A0CF060FC0620174981F88101052081F883014FF47A70486017
:401A40000E9888609DED140A084680ED390A1848007826F033FA0D49C1F82C013DE00B4890ED390ADFED150AB4EEE00AF1EE10FA26DB1FEDF60A80ED390A0920034981F8A0
:401A80008001292081F87E0127E00000B00F0020CDCCCC3D0000C8420000000000408F4000007A44081F0020000070428DED2448D80600206CE7DB457390EA4400004842FA
:401AC0009DED140A5FED0E0A30EE200A8DED140A9DED140AFE4880ED390A86E0FC48D0ED390A1FED141A80EE810A8DED010A01982EF030FBCDE902019DED020B2AF004FFAB
:401B00008DED060BF248D0F8640103902EF022FBCDE904019DED060B53EC102B9DED040B51EC100B2EF020F81FED250B53EC102BCDE908019DED080B51EC100B2DF0BCFDAE
:401B4000CDE90A019DED0A0B51EC100B2DF0C6FCDF49C1F80401084690ED570A5FED300A80EE201A80ED451ADA4890F830000A2804D1B3EE090A8DED100A03E0B1EE040A09
:401B80008DED100A9DED100A5FED390A80EE201A1FED3A0A21EE000ABDEEC00AB8EEC00ACB4880ED490AB0F87C0140F02000C849A1F87C01032081F88001062081F88101BB
:401BC000002081F883014FF47A7048600E9888609FEDC10A084680ED390A06E00020BC49A1F87C0181F8800100BF00BF05E4B84890F88001B64981F87F01084690F8810135
:401C000030B105287ED007287DD00A287CD10BE00620AF4981F881010A2081F88301192048600E988860C0E2A948806801460B900E9824F0E5F942F21071884207D9092036
:401C4000A34981F88001262081F87E01BCE0A14890F8280006280ED09E4890F82800072809D09B4890ED3B0A5FED770AB4EEE00AF1EE10FA13DC974890F82800062804D0FA
:401C8000944890F8280007282AD1914890ED3B0ADFED920AB4EEE00AF1EE10FA20DD8D4890F82800062804D08A4890F8280007280BD100BF874890ED300AF0EE040A30EE96
:401CC000600A834880ED390A7EE0824890ED300AF2EE0E0A30EE600A7D4880ED390A73E07C4890F82800062812D07A4890F8280007280DD07648D0ED3B0A9FED790AF4EE25
:401D0000C00A02E061E0F3E148E2F1EE10FA13D3704890F82800062804D06E4890F8280007282AD16A4890ED3B0A5FEDA70AB4EEE00AF1EE10FA20D2664890F8280006288B
:401D400004D0644890F8280007280BD100BF614890ED320AF0EE040A30EE200A5C4880ED390A31E05B4890ED320AF2EE0E0A30EE200A574880ED390A26E00620544981F841
:401D80008101052081F8830140F6B83048600E988860504890F8280007280AD14D48D0ED320A9FED500A20EE800A084680ED390A04E09FED490A464880ED390A0020444921
:401DC000C1F82C01C1F83801EFE14148D0F82C01D0BB4548007826F071F83D49C1F82C01084690ED530A80ED4C0A90ED550A80ED4D0A062081F88101072081F883013548F5
:401E000090F82800072803D14FF47A70486003E04FF47A702E4948602D490E9888602D4890F82800062804D02A4890F8280007280BD1284890ED300AF2EE0E0A30EE600AEC
:401E4000234880ED390A52E10AE0224890ED300A5FEDE60A30EE600A1D4880ED390A46E11B48D0F8380100287DD11F48007826F025F81749C1F83801084690ED530A80ED36
:401E80004F0A90ED550A80ED500AD0F83801D1F82C11401A0B9012F0DBFC00EE100AF8EE400A9FED120A20EE800ADFED100A80EE201A074880ED481AD0F838010449D1F816
:401EC0002C11401A00EE100AB8EEC00A10E00000B00F0020081F002000000000CDCC4C3ECDCC4C3D9A99193FD806002000007A44DFEDFE0AB4EEE00AF1EE10FA7DD2FC4855
:401F000090F82800062804D0F94890F82800072804D19FEDF80A8DED130A04E0F64890ED550A8DED130AF24890F82800072839D1F14890F884010B90ED4890ED0F0A8DEDF7
:401F40000A0AED4890ED4F0A8DED090A0B989DED0A1ADDED130A9DED090A10F0D6FAE64880ED3E0A00E0C2E090F884010B90E04890ED0F0A8DED0A0ADF4890ED4C0A8DED43
:401F8000090A0B989DED0A1ADDED130A9DED090A10F0BBFAD848D0ED3E0A30EEC00A80ED3E0A38E0D44890F884010B90D04890ED0F0A8DED0A0AD04890ED4F0A8DED090A2F
:401FC0000B989DED0A1ADDED130A9DED090A10F09CFAC94880ED3E0A90F884010B90C44890ED0F0A8DED0A0AC34890ED4C0A8DED090A0B989DED0A1A00E06CE0DDED130A09
:402000009DED090A10F081FABB48D0ED3E0A30EEC00A80ED3E0AB84890F884010B90B64890ED400AB1EE400A8DED0A0A90ED3E0A8DED090A0B999DED0A1A5FED540A9DED27
:40204000090A0120FEF76CFFAB4890ED3E0AF7EE000A80EE201A1FED600A31EE408AA74800780DF099FA5FED5F0A80EE201AA24890ED400AB1EE400AC0EE010A9C4890ED16
:40208000300A9FED9F1A10EE810AC8EE000A9A48C0ED3C0AB0F87C0140F008009649A1F87C010846B0F87C0140F01000A1F87C01062081F8800181F88101002081F8830130
:4020C0004FF47A7048600E9888601FED7D0A084680ED390A0BE01FED800A874880ED390A0920854981F880012B2081F87E015CE00620814981F88101052081F883010A2045
:4021000048600E9888600846D0ED390A9FED7C1A80EE810A8DED010A01982EF01BF8CDE902019DED020B2AF0EFFB8DED060B7248D0F8640103902EF00DF8CDE904019DEDF0
:40214000060B53EC102B9DED040B51EC100B2DF00BFD9FED6C0B53EC102BCDE908019DED080B51EC100B2DF0A7FACDE90A019DED0A0B51EC100B2DF0B1F95F49C1F80001EE
:40218000084690ED570A5FEDA70A80EE201A80ED441ABAEE000A80ED390A06E000205649A1F87C0181F8800100BF00BFFEE3524890F88001504981F87F01084690F8810180
:4021C00030B105287ED007287DD00A287CD10BE00620494981F881010A2081F88301192048600E988860F1E34348806801460B900E9823F005FF42F21071884207D90920E6
:402200003D4981F88001282081F87E01D3E0384890F8280006280ED0354890F82800072809D0354890ED3B0ADFED380AB4EEE00AF1EE10FA13D32E4890F82800062804D0EA
:402240002B4890F8280007282AD12B4890ED3B0ADFED2F0AB4EEE00AF1EE10FA20D2244890F82800062804D0214890F8280007280BD100BF1E4890ED320AF0EE040A30EE46
:40228000200A1D4880ED390A95E0194890ED320AF2EE0E0A30EE200A174880ED390A8AE0134890F82800062812D0114890F8280007280DD0104890ED3B0ADFED160AB4EEBF
:4022C000E00A02E078E082E3D1E3F1EE10FA2ADC074890F82800062804D0054890F82800072841D1044890ED3B0A15E0FF4680C6081F002039B40040B00F002093060020D9
:402300000000C8420000000000408F40CDCCCCBDCDCC4CBECDCC4CBD5FED040AB4EEE00AF1EE10FA20DDFE4890F82800062804D0FB4890F8280007280BD100BFF84890EDDF
:40234000300AF0EE040A30EE600AF64880ED390A31E0F34890ED300AF2EE0E0A30EE600AF04880ED390A26E00620EE4981F88101052081F8830140F6B83048600E98886082
:40238000E74890F8280007280AD1E54890ED300ADFEDE50A20EE200A084680ED390A04E09FEDE20ADF4880ED390A0020DD49C1F82C01C1F8380166E3DA48D0F82C01D0BB23
:4023C000DB48007825F07AFDD649C1F82C01084690ED530A80ED4C0A90ED550A80ED4D0A062081F88101072081F88301CC4890F82800072803D14FF47A70486003E04FF41F
:402400007A70C8494860C7490E988860C44890F82800062804D0C24890F8280007280BD1BF4890ED320AF2EE0E0A30EE200ABD4880ED390ACAE20AE0B94890ED320ADFED07
:40244000BD0A30EE200AB74880ED390ABEE2B548D0F838010028EDD1B548007825F02EFDB049C1F83801084690ED530A80ED4F0A90ED550A80ED500AD0F83801D1F82C11E2
:40248000401A0B9012F0E4F94FF47A71B0FBF1F000EE100AB8EE400ADFEDA70A20EE200AA04880ED4A0AD0F838019E49D1F82C11401A00EE100AB8EEC00ADFEDA00AB4EE60
:4024C000E00AF1EE10FA7DDD954890F82800062804D0934890F82800072804D11FED7B0A8DED130A04E08F4890ED550A8DED130A8B4890F82800072837D18A4890F88401A2
:402500000B90874890ED0F0A8DED0A0A854890ED4F0A8DED090A0B989DED0A1ADDED130A9DED090A0FF0F1FF7E4880ED3E0A90F884010B907A4890ED0F0A8DED0A0A79484F
:4025400090ED4C0A8DED090A0B989DED0A1ADDED130A9DED090A0FF0D8FF7248D0ED3E0A30EEC00A80ED3E0A38E06E4890F884010B906B4890ED0F0A8DED0A0A694890ED79
:402580004F0A8DED090A0B989DED0A1ADDED130A9DED090A0FF0B9FF624880ED3E0A90F884010B905E4890ED0F0A8DED0A0A5D4890ED4C0A8DED090A0B989DED0A1ADDEDB8
:4025C000130A00E0F6E19DED090A0FF09EFF5548D0ED3E0A30EEC00A80ED3E0A514890F884010B904F4890ED420A8DED0A0A90ED3E0A8DED090A0B999DED0A1ADFED4E0A98
:402600009DED090A0220FEF78BFC464890ED3E0AF7EE000A80EE201A9FED440A31EE408A474800780CF0B8FFDFED430A80EE201A3C4890ED420AC0EE010A394890ED320AF7
:402640001FEDD11A10EE810AC8EE000A3548C0ED3D0AB0F87C0140F040003249A1F87C010846B0F87C0140F08000A1F87C010846D0ED3F0A90ED410A30EE800A80ED3F0AD0
:4026800090ED3F0AF0EE000A80EE201A80ED3F1AD0ED400A90ED420A30EE800A80ED400A90ED400AF0EE000A80EE201A80ED401AD0ED430A90ED450A30EE800A80ED430A79
:4026C00090ED430AF0EE000A80EE201A80ED431A90ED440AD0ED460A30EE200A80ED440A90ED440AF0EE000A80EE201A80ED441A90ED470AD0ED490A30EE200A80ED470AD1
:4027000090ED470AF0EE000A80EE201A80ED471A90ED470ADFED0B0A20EE200A14E00000081F0020B00F00209A99193F00000000D80600200000484200007A44FF46804690
:40274000930600205F43BA3980ED470A90ED480AD0ED4A0A30EE200A80ED480A90ED480AF0EE000A80EE201A80ED481A90ED480A5FED0C0A20EE200A80ED480A90ED440A45
:40278000D0ED430A70EE600A90ED400A90ED3F1A30EE411A80EE810A8DED0B0A9DED0B0A08F0A0FDFE4890ED440AFE48D0ED700AFB4890ED401A00EEC10A8DED0B0A9DEDFB
:4027C0000B0A08F064FDF64890ED480AD0ED470A70EE600A90ED400A90ED3F1A30EE411A80EE810A8DED0B0A9DED0B0A08F035FDEB4890ED480AEB48D0ED720AE84890ED06
:40280000401A00EEC10A8DED0B0A9DED0B0A08F00AFDE54800780CF0BFFE5FED390A80EE201AE04890ED700A21EE000AD0ED710AB2EE001A71EE600A80EE801A9FEDDB0A57
:4028400021EE000A8DED130A90F82800062804D19FEDD70A8DED110A0DE0D24890F830000A2804D19FEDD20A8DED110A03E09FEDD10A8DED110ACA48D0ED3C0A9DED110A97
:4028800080EE201AC74890ED300A31EE400A8DED120A9DED130ADFEDC50AB4EEE00AF1EE10FA10DD9DED120ADFEDC00AB4EEE00AF1EE10FA07DD90F842009FEDBF0A0B90B8
:4028C0000BF038FD1DE09DED130ADDED120AB4EEE00AF1EE10FA0ADDB24890F842000B909DED120AB1EE400A0BF024FD09E0AD4890F842000B909DED130AB1EE400A0BF0EA
:4029000019FDA748D0ED3D0A9DED110A80EE201AA44890ED320A31EE000A8DED120A9DED130ADFEDA20AB4EEE00AF1EE10FA10DD9DED120ADFED9D0AB4EEE00AF1EE10FACE
:4029400007DD90F842009FED990A0B900BF016FD19E09DED130ADDED120AB4EEE00AF1EE10FA08DD8F4890F842000B909DED120A0BF004FD07E08B4890F842000B909DED6A
:40298000130A0BF0FBFC0820854981F88001062081F88101002081F883014FF47A7048600E9888601FED9F0A084600E08DE080ED390A0BE01FEDA30A794880ED390A092039
:4029C000774981F880012B2081F87E015BE00620734981F88101052081F883010A2048600E9888600846D0ED390A9FED701A80EE810A8DED030A03982DF0ACFBCDE9040142
:402A00009DED040B29F080FF8DED080B6448D0ED590A1FEDB71A80EE810A8DED050A05982DF098FBCDE906019DED080B53EC102B9DED060B51EC100B2DF096F8CDE90A012D
:402A40009DED0A0B51EC100B2CF048FD5449C1F80801084690ED570A5FEDC90A80EE201A80ED461AB2EE000A80ED390A0BE000204B49A1F87C0181F880011FEDD40A08469E
:402A800080ED390A00BF00BF1FE002200C900620434981F88101002081F88301192048600E9888601FEDDF0A084680ED390AFEF71DFA0AE003200C901FEDE40A384880ED63
:402AC000390AFCF74AF800E000BF00BF344890ED390AB5EEC00AF1EE10FA0AD090ED390A8DED0B0A012108469DED0B0AF7F742FC0AE02B4890ED390A8DED0B0A002101201C
:402B00009DED0B0AF7F736FC0C9815B0BDEC028B00BD10B50124224890F87E01B8B920F07BFE18B1FEF7ABFA04460EE020F08CFE58B11C4890F82800072803D1FEF7D4F90E
:402B4000044602E0FDF78AFC0446FBF79AFE204601F0DBF9124890F87E0120B1104991F87E0101F0A9FE204610BD10B50C4890F880010A2849D2DFE800F0494A30054831EB
:402B80000648484B00BF0220054981F881010020086010F055FC024880ED080A0EE00000B00F0020081F0020930600200000C8423333B33F3333B33E0000C8C290F8870148
:402BC000401C8E4981F88701084690F887010A2802DD0A2081F887011DE000BF0D20874981F8810123F0D5F9844908609FED840A084680ED350A002081F88701084690F832
:402C00008501C01E81F8850105E000BF00BF00BFFBF7CEFD00BF00BF7A480021416481640020764981F87E01B6EE000A084680ED390A10BD10B520F0EFFD10B301F038FE6C
:402C40002B2802D1FBF7B4FD1DE06C4890F87F016A4981F88001062081F88101002081F883014FF47A70486023F093F9634988609FED630A084680ED390A002081F87E01D0
:402C800001E0FFF772FF10BDB7EE000A70475B4890F87E01704710B55B48FCF7F9FE5A48FCF77BFE5848FBF76EFF10BD10B55648FCF7EEFE5448FCF770FE5348FBF763FFDE
:402CC00010BD4E4890F8800170474C4890F88101704710B50424494890F88001012804D10620464981F8800186E04FF4FA714748008823F054F900287ED023F04AF9434945
:402D000008803E4890F88001801E072872D2DFE800F0450571440471700000BF374890F88101801E0B2835D2DFE800F00634151F0B1A3434343410000620304981F88101EC
:402D400029E00C202D4981F8810124E004202B4981F881011FE00720284981F881011AE00520264981F8810115E0244890F88001062807D10320214981F88001022081F869
:402D8000810106E005201D4981F880010D2081F8810100E000BF00BF2DE000BF174890F88101062804D00D2807D00E281ED109E00D20124981F8810119E00E200F4981F8D4
:402DC000810114E00D4890F88001052809D102200A4981F88001062081F8810105E00BE008E00820054981F8800100E000BF00BF01E000E000BF00BF204610BDB00F002091
:402E000000000000B0100020381100203C03002070B541201CE0C41700EBD4646511CD4C54F82540C51700EBD5656D11A0EB45160125B5402C40C51700EBD5656D11A0EB34
:402E400045160125B540AC4200D103E0411EC8B20028E0DC00BF70BD30B5C31700EBD3635C11BC4B183353F824300246C41700EBD4646411A0EB44150124AC4023430146F6
:402E8000C41700EBD4646511B24C183444F8253030BD13B50C4600BFAF49096801F5B07108190122694606F06BFA18B99DF80010AA48015500BF1CBD13B50C4600BFA64911
:402EC000096801F25F2108190122694606F058FA20B99DF80010A148FF30015500BF1CBD70B504469E480470E21704EBD2625311984A52F823202146E31704EBD3635B1185
:402F0000A4EB43150123AB409A432046E31704EBD3635D118F4B43F82520E21704EBD26253118C4A0C3252F82320E31704EBD3635B11A4EB43150123AB409A43E31704EB09
:402F4000D3635D11834B0C3343F82520E21704EBD26253117F4A183252F82320E31704EBD3635B11A4EB43150123AB409A43E31704EBD3635D11774B183343F82520002068
:402F8000FFF79AFF70BD30B50146CB1701EBD3635C11704B53F82430CC1701EBD4646411A1EB44150124AC4023400BB1012030BD0020FCE76B49087070476A4800787047F8
:402FC00070B52DED048B04460025422C70D2DFE804F02122272C2D2E2F37424D586069737F88A3A8BBFEFDFCFBFAF9F8F7F6F5F4F3F2F1F0EFEEEDECEBEAE9E8E7E6E5E437
:40300000E3E2E1E0DFDEDDDCDBDAD9D8D7D6D5D4D3D2D194F2E20DF043FE80F00105EDE220F0F2FB80F00105E8E2E7E2E6E2E5E2F9F79CFF08B1012000E000200546DDE273
:403040000EF09AFC30B1F9F789FF08B1012000E000200546D2E20EF08FFC30B1F9F796FF08B1012000E000200546C7E20EF084FC30B1F9F783FF08B1012000E000200546D7
:40308000BCE210F02BFB012800D100E000200546B4E210F023FB032801D1012000E000200546ABE2304890F83800012801D101E0A3E200200546A1E20EF05EFC38B12A4823
:4030C00090F8380008B9012000E00020054695E2254890F89000012800D100E0002005468CE20EF049FC38B11F4890F8900008B9012000E00020054680E21B4890F83800D7
:40310000022804D0184890F89000022801D1012000E00020054671E209F06DFA80F001056CE21248007D60B90A48001F006900F48030B0F5803F04D002F0DEFD08B10120ED
:4031400000E00020054659E20948007D08B901203FE03DE0E8160020AC0300200825002048030020490300202C27002028280020402800203DE212E200E2F3E1EAE1DDE10F
:40318000D1E1C5E1BCE1B3E1A7E19EE192E189E180E177E16EE165E15CE153E14AE141E138E12FE126E121E115E103E1DAE0CDE0C0E0B3E0A6E099E08CE082E077E06CE080
:4031C00054E047E03AE029E01CE00FE006E002E00020054612E2F74805780FE2F7F78DF908B1012000E00020054607E20DF0ECFAB0EE408A9FEDF01ADFEDF00A0DF063FA0F
:403200000546FBE10DF0E0FAB0EE408A9FEDEC1ADFEDEC0A0DF057FA0546EFE103F02BF8B0F57B4F07DB03F026F84FF6FF71884201DA012000E000200546DFE102F0DCFFA0
:4032400028B1E1488078FE2801D0012000E000200546D3E1DC488078FE2806D0F9F7E2FD18B101250020D9490872C7E1D6488078FE2805D0D648007810B103F0A0FD20B13A
:4032800001251A20FFF796FE06E0FFF796FE1A2802D10020FFF78EFEB0E1CE48007800F0B40008B1012000E000200546A6E1C948007800F0480008B1012000E000200546A8
:4032C0009CE1C5480088102801D0012000E00020054693E10DF0C7FAB0EE408A9FEDB61ADFEDB80A0DF0EFF9054687E10DF0C3FAB0EE408A9FEDB01ADFEDB20A0DF0E3F952
:4033000005467BE10DF0BFFAB0EE408A9FEDAA1ADFEDAC0A0DF0D7F905466FE10DF07CFAB0EE408A9FEDA41ADFEDA60A0DF0CBF9054663E10CF0E5FAB0EE408A9FED9E1A16
:40334000DFEDA00A0DF0BFF9054657E10DF06CFAB0EE408A9FED981ADFED9A0A0DF0B3F905464BE120F058FA18B3F7F7E0FCB0EE408AF7F7B1FC38EE400A10EE106A3046AE
:403380002CF0E8FE41EC190BB0EE490AF0EE690A29F0BAFAB0EE408AF0EE608A9FED8F0B53EC102B51EC180B2CF0DCFC00D2012500BF23E1F7F7BBFCDFED8A0AB4EEE00A3B
:4033C000F1EE10FA04DDF6F7FDFA08B1012000E00020054612E102F08FFC20B903F091F908B9012000E00020054607E108F004FA054603E10EF0C0FA18B103F0C5FD80F054
:403400000105FBE0F7F784F808B1012000E000200546F3E0F7F789F808B1012000E000200546EBE0F7F729F908B1012000E000200546E3E0F7F75FF908B1012000E00020D2
:403440000546DBE0F7F791F908B1012000E000200546D3E0F7F7C3F908B1012000E000200546CBE0F7F7F9F908B1012000E000200546C3E0F7F72BFA08B1012000E00020E7
:403480000546BBE0F7F75DFA08B1012000E000200546B3E0F7F793FA08B1012000E000200546ABE0F7F7C5FA08B1012000E000200546A3E00EF060FA30B1F7F725FB08B1A9
:4034C000012000E00020054698E0F7F739FB08B1012000E00020054690E00EF04DFA30B1F7F749FB08B1012000E00020054685E0F7F760FB08B1012000E0002005467DE084
:40350000F7F774FB08B1012000E00020054675E00EF032FA30B1F7F785FB08B1012000E0002005466AE00EF027FA30B1F7F796FB08B1012000E0002005465FE00DF02FFAC3
:4035400006460DF0AFFA06430EB1012000E00020054653E00DF0DEFA08B1012000E0002005464BE00EF008FA38B108F0C4FB012803D103F07AFC00B901253FE0F6F75EFF3F
:4035800028B9F7F70EFC10B9F7F725FC20B103F06CFC08B9012000E0002005462EE00DF05FFB20B91048007820F07AFDF0B101201DE000008D03002000FF7F4700A025462D
:4035C00000007A460000000078C70020C02F0020C8040020A103002042070020000000000070A7400000FA45130700200020054604E003F0B5F8054600E000BF00BF05B166
:4036000000BF3DB9FE480078002807DDFC480078844203D10120BDEC048B70BD0020FAE74FF00008C1464FF0010A4FF0500B0321F44880F8B81000248FE0F348005D04EB42
:40364000840101EBC401F14A02EB810189680870ED48FF30005D00287DD0E21704EBD2625311EB4A52F82320E31704EBD3635B11A4EB431C012303FA0CF31A43E31704EBAA
:40368000D3634FEA631CE24B43F82C20E21704EBD2625311DE4A0C3252F82320E31704EBD3635B11A4EB431C012303FA0CF31A43E31704EBD3634FEA631CD54B0C3343F88E
:4036C0002C2004EB840000EBC400D04901EB8000007BE0B1E21704EBD2625311CC4A183252F823202146E31704EBD3635B11A4EB431C012303FA0CF31A432046E31704EBB2
:40370000D3634FEA631CC24B183343F82C2022F040FCC04941F8240000BFE21704EBD2625311BB4A243252F823202146E31704EBD3635B11A4EB431C012303FA0CF39A4304
:403740002046E31704EBD3634FEA631CB04B243343F82C2000BF601CC4B2422CFFF66DAF4FF47A60DFF8B0C200DFA648D0F8DC100120DFF8A8C200DF4FF47A60DFF898C28D
:4037800000DF00BF002259460320DFF894C200DF0646022E21D1DFF88CC200DF074607F00200D0B1002416E0002004EB840101EBC401964A02EB81018968087004EB8401B7
:4037C00001EBC40102EB8101896808782146FFF760FB601CC4B2422CE6DB0024AAE22046FFF7EEFB05462046FFF7CDFBA8427DD0002D7CD1A946E31704EBD3634FEA631C84
:40380000834B0C3353F82C304FEAE47C04EBDC6C4FEA6C1CA4EB4C1E4FF0010C0CFA0EFC03EA0C034FEAE47C04EBDC6C4FEA6C1CA4EB4C1E4FF0010C0CFA0EFC634501D093
:403840004FF0010904EB840000EBC4006F4901EB800090F8330000F0010008B14FF0010904EB840000EBC400684901EB800090F8330000F0020020B108F075FD08B14FF0EC
:40388000010904EB840000EBC400604901EB800090F8330000F0040038B107F0B5FF10B91FF0E5FF08B14FF0010904EB840000EBC400564901EB800090F8330000F00800E6
:4038C00020B1BAF1000F01D04FF0010904EB840000EBC4004D4901EB800090F8330000F0100038B15048005D012801E010E010E000D18146B9F1010F0AD100204A4908553F
:403900004FF001082046FFF7EBFA3520F9F7FAFB03E1E31704EBD3634FEA631C3C4B53F82C304FEAE47C04EBDC6C4FEA6C1CA4EB4C1E4FF0010C0CFA0EFC03EA0C034FEAC0
:40394000E47C04EBDC6C4FEA6C1CA4EB4C1E4FF0010C0CFA0EFC6345DAD000203249085500BF02F0C9F9E8B1E21704EBD2625311274A243252F823202146E31704EBD363EA
:403980005B11A4EB431C012303FA0CF31A432046E31704EBD3634FEA631C1D4B243343F82C201CE0E21704EBD2625311184A243252F823202146E31704EBD3635B11A4EB6B
:4039C000431C012303FA0CF39A432046E31704EBD3634FEA631C0E4B243343F82C20E21704EBD26253110A4A52F82320E31704EBD3635B11A4EB431C012303FA0CF315E008
:403A00004A030020D03F0020082500203C030408E8160020DC15002029E7030889E70308E9E7030831E703089A1500201A43E31704EBD3634FEA631CFE4B43F82C2022F0AA
:403A4000A8FAFD4941F8240004EB840000EBC400FA4901EB800080680078401C04EB840101EBC401F54A02EB81018968087004EB840000EBC400114601EB800080680078F3
:403A80007E2808DD7E2004EB840101EBC40102EB81018968087000BF00BF02F02DF901281DD1E21704EBD2625311E24A243252F823202146E31704EBD3635B11A4EB431CC4
:403AC000012303FA0CF31A432046E31704EBD3634FEA631CD74B243343F82C201CE0E21704EBD2625311D34A243252F823202146E31704EBD3635B11A4EB431C012303FA8F
:403B00000CF39A432046E31704EBD3634FEA631CC84B243343F82C2000BF002D7DD0E21704EBD2625311C34A0C3252F82320E31704EBD3635B11A4EB431C012303FA0CF351
:403B40001A40002A53D104EB840000EBC400BB4901EB8000406AE8BBE21704EBD2625311B44A0C3252F82320E31704EBD3635B11A4EB431C012303FA0CF31A43E31704EB96
:403B8000D3634FEA631CAB4B0C3343F82C204FF0010804EB840000EBC40001EB8000806800787E2811DA04EB840000EBC40001EB800080680078401C04EB840101EBC40125
:403BC0009E4A02EB81018968087021460120FFF773F900E00CE004EB840101EBC401974A02EB8101896808782146FFF752F95BE004EB840202EBC402904B03EB8202516A56
:403C00008D4A52F8240022F0CAF9E8B3E21704EBD2625311874A0C3200E083E052F82320E31704EBD3635B11A4EB431C012303FA0CF31A43E31704EBD3634FEA631C7D4BDB
:403C40000C3343F82C204FF0010804EB840000EBC4007A4901EB8000806800787E2811DA04EB840000EBC40001EB800080680078401C04EB840101EBC401704A02EB81015C
:403C800089680870214600E00EE00120FFF714F904EB840101EBC401684A02EB8101896808782146FFF7F5F804EB840202EBC402624B03EB8202127BA2B3E21704EBD262FC
:403CC00053115C4A183252F82320E31704EBD3635B11A4EB431C012303FA0CF31A400ABB02F00AF810B901F013FBE0B104EB840000EBC400514901EB8000806A68B104EBC4
:403D0000840202EBC4020B4603EB8202916A4A4A52F8240022F043F920B12046FFF79CF84FF0010804E02046FFF796F84FF00108601CC4B2422CFFF652ADB8F1010F0BD134
:403D40003F48D0F8DC100120DFF8F8C000DF4FF000083520F9F7D6F94FF0000AFFF758F804460FE5002107E0324850F8210008B101207047481CC1B20329F5DB0020F8E703
:403D8000002108E02B48183050F8210008B101207047481CC1B20329F4DB0020F8E770B541201DE0C41700EBD4646511214C183454F82540C51700EBD5656D11A0EB4516AE
:403DC0000125B5402C40C51700EBD5656D11A0EB45160125B540AC4200D103E0411EC8B20028DFDC00BF70BD70B5002401F084FFF8B1412437E0E31704EBD3635D110D4BAB
:403E00000C3353F82530E51704EBD5656D11A4EB45160125B5402B40E51704EBD5656D11A4EB45160125B540AB421AD104EB84030AE01BE0E8160020DC1500203C0304083B
:403E4000D03F002089E7030803EBC403294D05EB830393F83330102B03D1274B1B5D03B903E0601EC4B2002CC5DC00BF204670BD0121214A1154704701460020FF2906DA46
:403E80001D4A525C0AB1012200E000221046704700B5002304E01846FFF7EAFF581CC3B2422BF8DB00BD0EB5144A07CA8DE807001BF058F91CF0BCFE0C226946FF201BF08A
:403EC0001DF90EBD014601EB810000EBC100094A52F820007047014601EB810000EBC100044A02EB800000797047704704490870704700003C0304089A150020A4100408B5
:403F00004A030020FE48007B7047FD490873704710B52DED088BF0EE409AF0EE608A04469FEDF80AF0EE40AA9FEDF70AC0EE290AB0EE608AB1EE000A28EE800AC0EE080A93
:403F4000B0EE60AA9FEDEF0AB0EE40BA204622F048F8BCEEC80A10EE101AB0FBF1F201FB120000EE100AB8EE400AB0EE409AB5EE000A28EE000AB4EEC90AF1EE10FA15D8FC
:403F8000B6EE080A28EE000AB4EEC90AF1EE10FA0CDDBFEE000A2AEE000AB0EE40AAB0EE000A28EE800AB0EE40BA0EE0B6EE080A28EE000AB4EEC90AF1EE10FA05D8B9EEFD
:403FC000000A28EE800AB0EE40BAB0EE4B0A0AEE090AF0EE40AAB0EE6A0ABDEC088B10BD70B52DED068B04460D46284621F0F9FF00EE100AB8EE400AB0EE408A9FEDC20A02
:40400000C8EE000AB0EE608A94ED000AD4ED020A00EE880ADFEDBD0A68EE200A20EE200A10EE101A08462CF095F841EC1A0BB0EE4A0AF0EE6A0A29F027FBB0EE409AF0EECF
:40404000609A51EC190B2BF049FA08EE100A94ED040A20EE080AB0EE408AB0EE480ABDEC068B70BD2DE9F0412DED028B05460F4690460024002600BF32E0322108FB01F043
:4040800000EE100AB8EEC00ADFED9F0A80EE201A05F1300000EB840090ED000A30EE410A05F1300000EB840080ED000A08FB01F000EE100AB8EEC00ADFED930A80EE201A5D
:4040C00005F1700000EB840090ED000A30EE410A05F1700000EB840080ED000A601CC4B2082CCADB0024D8E007F1300000EB840090ED000A07F1700000EB8400D0ED000A4C
:4041000030EE600AF0EE000A20EE200AB0EE408A05F1300000EB840090ED000A07F1300000EB8400D0ED000A30EE600A05F1900000EB860080ED000A05F1900000EB860008
:4041400090ED000AC0EE080A9FED710A20EE800A05F1CC0000EB860080ED000A05F1500000EB840090ED000A05F1100000EB8400D0ED000A30EE600A07F1500000EB8400F8
:40418000D0ED000A07F1100000EB840090ED001A70EEC10A80EE201A05F5847000EB860080ED001AB7EE000AC0EE080A05F5A27000EB8600C0ED000A701CC6B20F2E6ADA4B
:4041C00007F17000611C00EB810090ED000A07F1300000EB8400D0ED000A30EE600AF0EE000A20EE200AB0EE408A05F1700000EB810090ED000A07F1700000EB8100D0ED8F
:40420000000A30EE600A05F1900000EB860080ED000A05F1900000EB860090ED000AC0EE080A9FED3B0A20EE800A05F1CC0000EB860080ED000A05F1500000EB810090EDFE
:40424000000A05F1100000EB8400D0ED000A30EE600A07F1500000EB8100D0ED000A07F1100000EB840090ED001A70EEC10A80EE201A05F5847000EB860080ED001AB7EE8B
:40428000000AC0EE080A05F5A27000EB8600C0ED000A701CC6B2601CC4B2082CFFF624AF1C4B0F221C4901F13C0012F0C6F91B4B0F2219493C3901F1780012F0BEF9154834
:4042C00090ED010A0E4880ED1D0A124890ED000A0B4880ED230A114890ED010ADFED100A30EEC00AD0ED000A80EE201A044880ED261A0F210848783812F085F9004811E07E
:404300002C1700200000000000007A44DB0FC9400000B44350030020DC180020580300200000344380ED200ABDEC028BBDE8F08170B52DED028B0446B0EE408A0D462078AD
:4043400000F0100000280AD094ED020A84ED030A84ED028AA078082802D10420208086E0207800F00100D8B394ED020AD4ED030AB4EEE00AF1EE10FA20DD94ED020AFD483B
:40438000817804F1500000EB810080ED000AFA49486821F026FE00EE100AB8EE400A5FED260A80EE201AF348817804F1700000EB810080ED001A0020E07002E0E078401C06
:4043C000E070E0782179884251DD208840F002002080208820F0010020800020E07046E0FFE7207800F00200F0B394ED020AD4ED030AB4EEE00AF1EE10FA1ED294ED020ABA
:40440000A17804F1100000EB810080ED000ADA49486821F0E6FD00EE100AB8EE400A5FED460A80EE201AA17804F1300000EB810080ED001A0020E07002E0E078401CE070F1
:40444000E0782179884212DD208840F001002080208820F002002080A078401CA0700020E0700DB1207900E001E0401E2071BDEC028B70BD10B52DED028BF0EE408AB0EEAE
:40448000608ABD49486821F0ACFDB0F57A7F0BD90121B0EE480AB948FFF74AFF0021B0EE680AB448FFF744FFB448008804280DD1B0480088042809D10222AE49AF48FFF74C
:4044C000D1FD2020AD490880AA490880BDEC028B10BD10B52DED0C8B044602F0A0FD60B1F8F76FFDB0EE408AD4ED098AB1EE00AAF1EE00AAB0EE009A2BE00EF020FFB0EE6B
:40450000408A9F4991F8280091ED0F0AF0EE400AB0EE480A0EF02AFEDFED9A0A20EE200AB0EE408A964991F8280091ED0F1AF0EE410A94ED091AB0EE410A0EF017FEDFED67
:40454000910A60EE208AB0EE00AAF0EE00AAB7EE009A4020005D40B994ED0B0A38EEC00A84ED0E0A0121402001551AEE100A2BF0F1FD41EC1B0B94ED0B0A30EE480A10EE7A
:40458000101A08462BF0E6FD41EC1D0BB0EE4D0AF0EE6D0A28F0B8F9B0EE40CAF0EE60CA53EC1B2B51EC1C0B2BF0DCFB0ED24C20005D58B9606821F014FD00EE100AB8EE40
:4045C000400A84ED110A01214C2001551AEE900A2BF0C0FD41EC1B0B38EEC80A10EE101A08462BF0B7FD41EC1D0BB0EE4D0AF0EE6D0A28F089F9B0EE40CAF0EE60CA53ECCF
:404600001B2B51EC1C0B2BF073FA0ED25820005D58B9606821F0E5FC00EE100AB8EE400A84ED140A01215820015519EE100A2BF091FD41EC1D0B38EEC80A10EE101A0846C4
:404640002BF088FD41EC1C0BB0EE4C0AF0EE6C0A28F05AF9B0EE40BAF0EE60BA53EC1D2B51EC1B0B2BF07EFB0DD8002164200155607B454951F8200000EE100AB8EE400ADB
:4046800084ED170A31E019EE100A2BF063FD41EC1B0B38EEC80A10EE101A08462BF05AFD41EC1D0BB0EE4D0AF0EE6D0A28F02CF9B0EE40CAF0EE60CA53EC1B2B51EC1C0B13
:4046C0002BF016FA11D26420005D70B9012164200155606821F085FC00EE100AB8EE400A84ED170A21F055FCA06078EEC89A94ED0E0AB5EEC00AF1EE10FA0BD2B4EEE88AB8
:40470000F1EE10FA06D294ED1B0AB4EEE90AF1EE10FA12D394ED0E0AB5EEC00AF1EE10FA25DDB4EEE88AF1EE10FA20DD94ED1B0AB4EEE90AF1EE10FA19DDC4ED1B9A94EDC3
:404740001B0A10EE101A08462BF004FD41EC1C0BB0EE4C0AF0EE6C0A28F0D6F8B0EE40BAF0EE60BA51EC1B0B2AF0B8FEA066BDEC0C8B10BD541900202C170020D41700202F
:40478000081F0020E02E6542B010040800200022002100BF33E0FA4B03EB820393ED000AB5EEC00AF1EE10FA01D14B1C99B2F44B403303EB820393ED000AB5EEC00AF1EEE5
:4047C00010FA01D14B1C99B2EE4B03EB820393ED000AB5EEC00AF1EE10FA01D14B1C99B2E84B403303EB820393ED000AB5EEC00AF1EE10FA01D14B1C99B2531CDAB2082A71
:40480000C9DB00224FE0E04B93ED1D0ADFEDDF0AB4EEE00AF1EE10FA06DC93ED1D0AB5EEC00AF1EE10FA01D24B1C99B2D64B93ED230ADFEDD60AB4EEE00AF1EE10FA08DC50
:4048400093ED230ADFEDD20AB4EEE00AF1EE10FA01D24B1C99B2CC4B93ED260ADFEDCB0AB4EEE00AF1EE10FA06DC93ED260AB5EEC00AF1EE10FA01D24B1C99B2C24B93ED12
:40488000200ADFEDC20AB4EEE00AF1EE10FA06DC93ED200AB5EEC00AF1EE10FA01D24B1C99B2531CDAB20F2AADDB01B901207047B54890F8A4007047B34981F8A40070475C
:4048C000B148407B0C281FD0AF48407B0B281BD0AD48407B072817D0AB48407B082813D0A948407B0A280FD0A748407B04280BD0A548407B052807D0A348407B0F2803D0C0
:40490000A148407B102801D1012070470020FCE770B5002426F03EFB00287DD101F06CFC18B10720FFF7C8FFC5E007F064FE58B99548407B082807D09348407B0A2803D091
:404940000220FFF7B9FFB6E018F0E2FCB5EEC00AF1EE10FA17D28C48407B082813D08A48407B0A280FD08848407B0B280BD08648407B102807D08448407B0F2803D0092081
:40498000FFF79AFF97E018F0C3FCDFED820AB4EEE00AF1EE10FA17D27B48407B082813D07948407B04280FD07748407B05280BD07548407B0A2807D07348407B0B2803D0DD
:4049C0007148407B10280CD16F48407B0F280CD118F0A2FCDFED6F0AB4EEE00AF1EE10FA03D20420FFF768FF65E018F091FCDFED6A0AB4EEE00AF1EE10FA21DD6248407B00
:404A000008281DD06048407B042819D05E48407B052815D05C4800E054E0407B0A280FD05948407B0B280BD05748407B0F2807D05548407B102803D00520FFF73DFF3AE044
:404A40005648007D18B90120FFF736FF33E0F5F7F5FC50B102F009FA38B94B48407B0F2803D10D20FFF728FF25E006F0A0FF28B106F09DFF0546FFF71FFF1CE0F8F78EFAAD
:404A800028B1F8F78BFA0546FFF716FF13E006F0B3FE38B13C48407B0B2803D02420FFF70BFF08E0FFF76CF928B1FFF709FF10B90A20FFF701FFFFF7FBFE18B10120FFF775
:404AC00024FA0124204670BDC9B1DFED350AC0ED000ADFED340AC0ED010A334AD2ED060AB8EE601ADFED311AC1EE210A9FED301AC1EE201AC0ED021A80ED040A1CE0DFEDBA
:404B00002D0AC0ED000ADFED2C0AC0ED010A264AD2ED0D0AB8EE601ADFED241AC1EE210ADFED261A81EEA01AF6EE000A61EE200AC0ED020A80ED040A704710B501219FED89
:404B4000200A11481030FFF7BFFF4FF4C0710C48303826F078FD4FF4C0710A48303826F072FD0A20064930390871064930390871112003493039088002493039088010BD4D
:404B800004180020841900202C17002000409C4500409CC52FDDE43E2FDDE43F40280020CDCCCC3D14AE473FB010040800007A447A142E3FCDCC4C3E0000204233331F4237
:404BC00035FA0E3D2DED028B84B04FF47A66A821FE4826F038FD1421FD4826F034FD00BF002231460320DFF8ECC300DF0546022D70D1DFF8E4C300DF0446022C6BD1F4483A
:404C00000078002867D0F2480078112863DC0120F2490870EE480078EC49487321F0B9F9EA494860EA4890ED010A084680ED090A407BEB4908700020E449886008460021D0
:404C40008166C1660167C165016641668163C163016441648164C1640165416581650020DA4981F8A4000846407BDE4951F82000D64908600846407B11287DD2DFE800F0B4
:404C80008F4B4E4F505109434849478A412C3A4C4D00CE48002141678167C1678030C160016141618161C1610162016041608160FFF743FF04208DF8040003208DF805004E
:404CC00005208DF80600022201A9FF201AF016FA042665E097E067E000219FEDC30ABB481030FFF7F1FE9FEDC10AB84880ED090A042655E09FEDBD0AB44880ED090A0426FF
:404D00004EE0C8264CE0FDF795FFC82648E000BF00BF042644E000BF00BF00BF00BF00BF00BF02F07CF950B1F8F74BF9B0EE408AA64880ED0B8A012180F8341018E00EF080
:404D4000FEFAB0EE408AAA4991F8280091ED0F0AF0EE400AB0EE480A0EF008FADFEDA50A20EE200A994880ED0B0A012180F8341004208DF8040000E011E003208DF8050061
:404D800005208DF80600032201A9FF201AF0B6F9042605E04FF4C87606F01EFF00E000BF00BF042089490873012C2CD1002087494873002101209FED8D0AF5F7DBFA00200F
:404DC000864908709FED890A814880ED010A9FED870A7E4880ED090A4FF47A665620F8F791F95720F8F78EF9FFF78CF8042802D10020FFF78AF80C2018F0BEFF002201A9DC
:404E0000FF201AF07BF97148407B00287DD06F4A1168506821F0C3F8F8B9FFF773F804280BD06A48407B072817D06848407B0B2813D06648407B0C280FD0FFF769FD60B928
:404E4000624890F8640001286DD16049886840F6C41121F0A4F8002865D05C48407B022807D05A48407B012803D05848407B032819D1564890F8640030B9544890ED000AC8
:404E8000B8EE400A80ED170A504890F8580030B94E4890ED000AB8EE400A80ED140A5720F8F730F91FE04948407B06281BD1FFF76DFC80B99FED500A444880ED1D0A9FED5D
:404EC0004E0A80ED230A9FED4C0A80ED260A9FED4A0A80ED200A002048490880484908805620F8F70FF90C2018F046FF002037494873FFF707F8042802D10020FFF705F830
:404F0000002101209FED390A00E00CE0F5F732FA0020324908709FED350A2D4880ED010A4FF47A665CE62948407B112871D2DFE800F0090A1D8CD7F0FFEDECEBEAE9E8E705
:404F4000E60B0C0098E100BF00BF9FED280A1F4880ED090AD0ED090AB0EE600A0121032008F0EAFC1948FFF7B4FA85E102F057F868B19FED240A154880ED090AD0ED090A71
:404F8000B0EE600A0121032008F0AAFD59E01EF06EFCE8B3164890ED640ADFED1B0A20EE200ADFED1A0A20EE200AB0EE408A014691F8280091ED0F0AF0EE400AB0EE480A10
:404FC0000DF072FB014880ED090A31E02C17002018170020E9E7030831E703084C03002068030020B01004080000A04200000000081F0020E02E6542003C1C46D417002070
:405000005419002000008CC200008C420AD7233C00E017E1FE4991F8280091ED0F0AF0EE400A9FEDFC0A0DF03FFBFB4880ED090AF948D0ED090AB0EE600A0121032008F016
:405040007BFCF548FFF745FA16E101F0E8FF68B11FED130AF04880ED090AD0ED090AB0EE600A0121032008F03BFD35E01EF0FFFBD8B1E74890ED650A5FED1D0A20EE200AC5
:405080005FED1E0A20EE200AB0EE408A014691F8280091ED0F0AF0EE400AB0EE480A0DF003FBDD4880ED090A0DE0D94991F8280091ED0F0AF0EE400A9FEDD80A0DF0F4FABD
:4050C000D54880ED090AD448D0ED090AB0EE600A0121032008F030FCCF48FFF7FAF9CBE0CB4890F84210D03000EB8100D0ED000AB0EE600A01210846F5F73CF9BCE061E075
:405100004FE08AE083E076E080E075E070E00FE0FFE7BF4890F84210D83000EB8100D0ED000AB0EE600A01210846F5F723F9A3E0B94841681030FEF753FFB74880ED090A74
:40514000B34991F8280091ED0F1AF0EE410AB24991ED091AB0EE410A0DF0A6FAF0EE408A0121032008F0E8FBAB4890F82900B8B10020A94981F829000EF05EF9F0EE408A0A
:405180000321A7480FF0F8F8A54890ED001AF0EE410AA14890ED091AB0EE410AFFF76AF96AE09D4841681030FEF71AFF9A4880ED090AD0ED090AB0EE600A01210846F5F7B9
:4051C000D9F859E0944948689649D1ED000A964991ED000AFEF79CFE8F4880ED090AD0ED090AB0EE600A01210846F5F7C3F843E0FDF78FFC40E000BF8748D0ED090AB0EE77
:40520000600A01210846F5F7B5F835E034E006F0E9FB8046FEF779FE2EE07F4A083202F11C0101F18000FBF71DF88046FEF76DFE7948D0ED090AB0EE600A01210846F5F711
:4052400099F819E00020744948730873002101201FED9A0AF5F78EF80020744908701FED9D0A734880ED010A002201A9FF2019F045FF4FF47A6600BF00BFFEF743FE0428B7
:405280007FF450AE4FF4FA71384620F088FE00283FF448AE20F07DFE07460C2018F06CFD9EE470B52DED028B0446B0EE408A0025B5EEC08AF1EE10FA0AD04CB1112C07DC03
:4052C0005B4890ED010AB4EE480AF1EE10FA0DD15848D0F890110120DFF85CC100DF1FEDBD0A534880ED010A00250DE00CB1504804704F4880ED018A4E48D0F8901102205A
:40530000DFF834C100DF01252846BDEC028B70BD46480078704701203F4981F8290070477A2303703C4BD3ED0E0A9FED440AB2EE041A00EE810ABDEEC00A10EE103A1AB203
:405340004270130A8370344B93ED110ABCEEC00A10EE103A99B2C1700B0A03712E4B93ED140ABCEEC00A10EE103A99B241710B0A8371294B93ED170ABCEEC00A10EE103AE6
:4053800099B2C1710B0A0372234BD3ED1A0A9FED2B0AB2EE041A00EE810ABDEEC00A10EE103A1AB24272130A837270477B230370194BD3ED1D0A9FED221A9FED200A00EECE
:4053C000810ABDEEC00A10EE103A19B241700B0A8370114BD3ED230A9FED191A9FED170A00EE810ABDEEC00A10EE103A19B2C1700B0A0371084BD3ED260A9FED111A9FEDEB
:405400000F0A00EE810ABDEEC00A10EE103A19E0081F0020C2B8B2BE2C170020C2B8B23E60030020700300206C0300204C03002018170020D03F002089E7030800000047D2
:405440000000C84219B241710B0A83714E4B93ED200ADFED4E0A20EE200ABCEEC00A10EE103A9AB2C271130A0372704710B500244548407B112812D2DFE800F01213161722
:4054800018191A091D1E1C0D111B11141500FDF718FC044611E006F099FB04460DE000BF00BF00BF00BF00BF00BF00BF00BF00BF00BF00BF00BF00BF00BF00BF204610BD66
:4054C00010B500243048407B112812D2DFE800F01213161718191A091D1E1C0D111B11141500FDF7F2FB044611E006F06FFB04460DE000BF00BF00BF00BF00BF00BF00BF60
:4055000000BF00BF00BF00BF00BF00BF00BF00BF204610BD1C48407B70471B4890F86400704710B500241848407B112815D2DFE800F0161718191A1B1C091F201E15141D2E
:40554000140D0E00F9F767F9044613E000BFFFF7E4FF642110FB01F40CE000BF00BF00BF00BF00BF00BF00BF00BF00BF00BF00BF00BF00BF00BF204610BD002002490873DB
:4055800070470348007870472C17002000007A446803002010B5F7F7B6FA2820F7F7B2FD2920F7F7AFFD01F03AFD70B1DFF874C300DF0446042120F025FEDFF868C300DF2A
:4055C0000446022120F01EFE0DE0DFF858C300DF0446042120F033FEDFF848C300DF0446022120F02CFE10BD10B5CF48C16B012020F042FECC48C16B0120DFF830C300DFEC
:4056000010BD10B52DED0C8BB0EE408AC84890ED630AB0EE409AB4EEC98AF1EE10FA02DDF7F761FA38B9B4EEC98AF1EE10FA2CD2F7F759FA48BBBE4890ED6A0A10EE101A17
:4056400008462AF087FD41EC1B0B38EE490A10EE101A08462AF07EFD41EC1D0BB0EE4D0AF0EE6D0A27F050F9B0EE40CAF0EE60CA53EC1B2B51EC1C0B2AF076FA41EC1A0BF3
:4056800029F02CFF08EE900A3BE0B4EEC98AF1EE10FA02DDF7F727FA38B1B4EEC98AF1EE10FA2CD2F7F71FFA48B3A14890ED6B0A10EE101A08462AF04DFD41EC1B0B38EE3A
:4056C000490A10EE101A08462AF044FD41EC1D0BB0EE4D0AF0EE6D0A27F016F9B0EE40CAF0EE60CA53EC1B2B51EC1C0B2AF03CFA41EC1A0B29F0F2FE08EE900A01E0DFED40
:405700008D8A9FED8D0AF4EEC08AF1EE10FA03DD9FED890AF0EE408A9FED880AF4EEC08AF1EE10FA03D29FED850AF0EE408AB0EE680ABDEC0C8B10BD10B52DED028B20F00F
:4057400028FC7F4908600020F6F70AFEB0EE408AFFF757FF7A4880ED030AF6F7D9FFBDEC028B10BD2821764825F06DFF01216E4880F82012DFF8ACC100DF06460122042147
:4057800020F011FDDFF89CC100DF06461922022120F009FDDFF88CC100DF064631460120DFF888C100DF03215F4880F8201200BF00224FF6FF710720DFF888C100DF85B2AA
:4057C000012DF5D0022DF3D1DFF87CC100DF044604F0040008B1F7F705F804F0020018B1FFF7AAFFFFF700FF04F001000028DFD0FFF7D0FEDCE710B504464B48D0F81C12AC
:405800002046DFF828C100DF10BD10B52DED088B474890ED630AD0ED610A30EE600ADFED470A80EE801A11EE104A20462AF092FC41EC1B0BB0EE4B0AF0EE6B0A27F064F863
:40584000B0EE40AAF0EE60AA51EC1A0B29F03AFE41EC190B29F042FE08EE900A344890ED620AD0ED630A30EE600ADFED330A80EE801A11EE104A20462AF06CFC41EC1A0B10
:40588000B0EE4A0AF0EE6A0A27F03EF8B0EE409AF0EE609A51EC190B29F020FE08EE100A0020F6F71BFF224890F830000A280CD11F4890F8B201032807D19FED240AB0EE0A
:4058C000408AB1EE480AF0EE408AB0EE680AF6F759FFB0EE480AF6F769FFBDEC088B10BD70B505460C46F6F7B4FE2846F6F788FB2046F6F79DFBFFF788FF0120FFF77BFF6A
:4059000070BD0F48D0ED030AB0EE600A70470C4890F82400032801D0012070470020FCE702207047C9F30308D03F002089E70308081F0020000000000000C8420000C8C25E
:40594000D41A0020E9E7030831E70308D051863970B50023012113E0CC1701EBD4646511FE4C54F82540CD1701EBD5656D11A1EB45160125B5402C4004B10B46481CC1B293
:405980004029E9DB184670BD70B504460D46E21704EBD2625311F14A52F823202146E31704EBD3635B11A4EB43160123B3401A432046E31704EBD3635E11E84B43F826202F
:4059C0002846FDF7F7FA002C37D00821E448DFF894C300DF012813D0E1482038817F807F401CDF4A203A907710464454807F1E2802DB002011468877D948DFF86CC300DFC1
:405A00000821DA48DFF85CC300DF012815D020F0C0FAD74901EBC4014860D54810F83400FF2806DAD24810F83400401CD04901F83400CE48DFF830C300DF70BDCD49087023
:405A4000704710B5CC480079052876D2DFE800F003152563B700FEF793F910B90220C6490871C648007838B10120C5490870FFF7E5FF0020C1490870E6E0FEF781F910B916
:405A80000220BD490871BD48007828B10120BC4908700020B9490870D6E0FEF771F918B10020B549087135E0B448007838B30120B3490870FEF764F950B1FEF770F904463E
:405AC00021460920FFF760FF0120FFF7B7FF21E005F092FE38B127210320FFF755FF0120FFF7ACFF16E0A748007800F0080038B918213120FFF748FF0120FFF79FFF09E063
:405B000003209D49087120F044FA9F4908600020FDF750FA98E099480078002844D005F06BFE58B127210320FFF72EFF0120FFF785FF01209249087040E084E0FEF720F944
:405B400068B10120FFF77AFF01208D490870FEF726F9044621460920FFF716FF2EE04FF47A718948006820F01AFA90B18548007800F0020010BB0120FFF760FF1821312038
:405B8000FFF702FF01207E49087000207A49087114E07C48007800F00B0078B104207649087106F004FC09E018210220FFF7ECFE01207349087002206F49087144E06F48E5
:405BC000007850B918210220FFF7DEFE01206C49087002206849087123E005F00DFE68B127210320FFF7D0FE0220634908710120FFF724FF01206249087012E0FEF7C0F8AE
:405C000078B100205C4908710120FFF717FFFEF7C6F8044621460920FFF7B6FE0120584908705548007904280CD006F0BFFB08F07DFC38B1FFF76CFB20B99FED540A0F20E8
:405C4000FFF72FFB00E000BF00BF4B4800794A49487110BD4148001F0021016041608160C16070474A490870704710B5494991F8300001F0CAF830B1002213466421464809
:405C800012F06BFB11E0434991F8300001F0DFF828B9404991F8300001F0E1F828B10022134631213C4812F058FB10BD10B50024384991F8300001F0A8F858B9354991F879
:405CC000300001F0C4F828B9324991F8300001F0C6F800B10124204610BD2D480078704710B504462D480078844204D02B480470112018F041F810BD1F490979042901D1B1
:405D0000012100E000210846704700EE900AB8EE601ADFED230AF5EE001A51EE210AB0EE600ADFED200A80EE201AB0EE410A70471D480078704710B52DED028BFFF7F8FF00
:405D4000022807D0FFF7F4FF032803D0FFF7F0FF05283CD10BF0D2FD40B328E0701D00205C1D002051EC03086DEB0308FC1A00203C1B0020820300207803002083030020D3
:405D8000840300208C030020880300200000C84280030020081F0020B8CC0020760300200000FB4500007A447403002006E00BF09FFD022802D19FEDF88A0AE00BF09EFD14
:405DC00010B19FEDF68A04E09FEDF58A01E09FEDF48AB0EE480ABDEC028B10BD10B52DED028B17F079FAB0EE408AFFF7A4FFB4EEC08AF1EE10FA03DB0120BDEC028B10BD4B
:405E00000020FAE710B52DED048BF0EE408AB0EE609A0446F0EE689AFFF7E0FF00EE100AB8EE400AB4EEC90AF1EE10FA07DDFFF7D5FF00EE100AB8EE400AB0EE409A29EE29
:405E4000090ADFEDD80A80EE808AECB1F4EEC88AF1EE10FA05DDF0EE489A0120D249087015E0B1EE480AF4EEC08AF1EE10FA07D2B1EE480AF0EE409A0120CB49087006E0C9
:405E80000020C949087002E00020C7490870B0EE690ABDEC048B10BD10B504460020206060606071207120F074F8206010BD2DED048B92B04FF05008002406E04FF6FF70BE
:405EC00001A921F81400601CC4B2022CF6DB0020FFF7C8FE00208DF80800B4490870FFF7ADFD0020B2490870B248DFF8CCC200DFB248DFF8C4C200DFB148DFF8BCC200DF08
:405F00000020AC4914390874AE48FFF7C5FF0321AD4880F8441100BF002241460720DFF8ACC200DF0746022F7ED1DFF8A4C200DF054605F00200002877D010219D48DFF8B3
:405F400094C200DF012809D024229A49143909A825F01DFB9748DFF880C200DFBDF82460FFF7CAFE08B1012000E00020814617F0B3F9F0EE408A3046FFF7C7FEB0EE409A23
:405F80004846F0EE680AFFF73DFFB0EE408AFFF7B3FE00B387481438007C01280BD1DDED0B0AB0EE600A0121042007F03CFD8146FFF796FE1EE07F481438007C02280BD132
:405FC000DDED0A0AB0EE600A0121052007F088FD8146FFF785FE0DE076481438007C032808D101210220B0EE480A07F0A5FC8146FFF776FE9DF83500012800D100E0002080
:40600000764908709DF8350040B97548007840F00800734908700020FFF710FD4FF6FF70864223D06E4801E035E01FE0007800F00200D8B96A48007800F00800B0B10024E6
:4060400011E001A931F81410711A08B20EF0F9FB022806DC6248007840F002006049087003E0601CC4B2022CEBDB00BF05F0040088B15C4801889DF80820501CC0B28DF879
:40608000080001A820F812109DF80800022802DB00208DF808001AF0E3FD68B10AF000FE50B1FFF71AFE38B9FFF700FE08B1FFF7DCFD0120FFF7D6FD9DF8360090B10C9893
:4060C0001FF08FFFB0F5C87F0CD30120374908703D48D0F8B4100120DFF80CC100DF0BF057FC02E00020314908704048007D01281CD19DF8200028B90020394908701FF04E
:4061000048FF824640F2E24150461FF048FF60B31DF0ADFB48BB0120254908702A48D0F8B4100120DFF8C0C000DF1EE09DF8200001281AD12D48007DB8B900201C490870C1
:40614000FFF788FD2048D0F8B4100120DFF898C000DF2348007840F00100214908700120234908701FF015FF824618221F4903A825F00DFAFFF765FC1D48007801287FF462
:40618000CBAEFFF7E5FB1B490870002018490870122017F0F1FDBFE60AD7A33C9A99193E2FDDE43ED222FB3F85030020810300208D030020201B00205DEB03085C1D002006
:4061C000FC1A002078030020D03F0020E9E7030831E7030851EC03086DEB0308830300208C030020301B002089E70308102800208403002075030020FE4800787047FE4869
:4062000000787047FD480078704770B50025FC48007D012801D1002405E0F948007D08B9012400E002242543F648C472FDF7A8FD08B9012400E0002445EA8400C5B2F14840
:406240004472F148007D08B9012406E0EE48007D012801D1002400E0022445EA0410C5B2E8488472FFF7CEFF044645EA8415E5480472284670BDE548008870472DE9F04168
:4062800005460C4617469846069EB5F52D4F28D12821DE481430DFF878C300DF012820D0A078DA49C874A07800F0030048742078617840EA0120D54908801FF06AFED34953
:4062C000C8600120887403200874D248D0F840110220DFF844C300DFCC481430DFF83CC300DFBDE8F081F0EE400A9FEDCD0A30EEC01ADFEDCC1A81EE210A70472DE9F041B8
:406300002DED028B04460D4616461F462078AD2833D12821BD481430DFF8F4C200DF012863D0E078B949C874E07800F0030048746078A17840EA012000EE100AB8EEC00A3C
:40634000B0EE408AB0EE480AFFF7CDFFAF4880ED020A1FF01EFEAD49C860012088740874AC48D0F840110220DFF8ACC200DFA7481430DFF8A8C200DF37E02078AE2834D181
:406380002821A2481430DFF888C200DF01282CD0E0789E49C874E07800F0030048746078A17840EA012000EE100AB8EEC00AB0EE408AB0EE480AFFF796FF944880ED010AD4
:4063C0001FF0E7FD9149C86001208874022008749048D0F840110220DFF83CC200DF8B481430DFF838C200DF00BFBDEC028BBDE8F0819FED8D1ADFED8D0A40EE010AF1EEA6
:40640000001AB6EE001A00EEA11AFCEEC10A10EE901A88B2704710B52DED028B0CF08FFFB0EE408A9FED820AB4EE408AF1EE10FA06D0B0EE480AFFF7DCFF7249088003E005
:406440004FF6FF706F4908807248D0F840110420DFF8C4C100DF6B480088BDEC028B10BD70B58CB006460025002E50D01DF0FFF900284DD040F2B240012102220023CDE90B
:406480000532CDE90710042017210193CDE902310490972013460022114600900AA811F05DFD0AA9304611F04FFA044640F292400440844204D11DB904205E490870012566
:4064C00040F2B240012102220023CDE90532CDE90710042017210193CDE902310490972001230022114600900AA811F037FD0AA9304611F029FA044640F292400440844278
:4065000005D1002DFCD105204A4908700125DAE040F2B240012102220023CDE90532CDE9071017210193CDE902319720049300900123002211460AA811F010FD0AA930461B
:4065400011F002FA044640F292400440844204D11DB9032037490870012540F2B240012102220023CDE90532CDE9071017210193CDE902319720049300901346002211462E
:406580000AA811F0EBFC0AA9304611F0DDF9044640F292400440844204D11DB9022025490870012540F2B240012102220023CDE90532CDE9071017210193CDE9023197205D
:4065C000049300900323002211460AA811F0C6FC0AA9304611F0B8F9044640F292400440844204D11DB9032012490870012540F2B24021E08103002076030020820300205F
:4066000040280020301B0020E82700200C1B002051EC0308D03F002089E703086DEB030800401C460000C84200007A440000FB4500FF7F4774030020012102220023CDE977
:406640000532CDE9071017210193CDE902319720049300900423002211460AA811F07EFC0AA9304611F070F9044640F292400440844204D11DB9022043490870012540F2A2
:40668000B240012102220023CDE90532CDE9071017210193CDE9023197201A461946049300900AA811F05AFC0AA9304611F04CF9044640F292400440844204D11DB90120D7
:4066C00031490870012515B15420F6F71BFD28460CB070BD10B52D4890F8280007280DD116F0FAFDDFED2A0AB4EEE00AF1EE10FA01DB012000E00020044600E001242046D1
:4067000010BD10B516F0E8FDDFED220AB4EEE00AF1EE10FA01D8012010BD0020FCE79FED1E0A70479FED1D0A70471748007803280FD01548007802280BD013480078012819
:4067400007D011480078042803D00F480078052801D1012070470020FCE711480079704710B500F034FC10B10E48047800E00024204610BDF0EE400A1FED561A1FED580A7F
:4067800000EE810A7047000074030020081F00202FDDE43E83C00041B81E4141A2454841780300208503002010B5044600BF28222146FD48006802F0E3FD20B92822214686
:4067C000FA4824F09FFE00BF10BD10B504462822F649204624F096FE10BD01B500BF04226946F1480068283002F0CAFD18B99DF80000EE49886200BFED48C16B0220DFF80B
:40680000B4C300DF08BD01B500BF04226946E64800682C3002F0B4FD18B99DF80000E349C86200BF08BD01B500BF04226946DE480068303002F0A4FD10B9DC490098086362
:4068400000BF08BD10B52DED020B00BF04226946D54800683C3002F093FD20B99DED000AD24880ED0F0A00BF03F090FED048C16B0220DFF840C300DF0220F6F743FC4E2079
:40688000F6F740FC1CBD01B500BF01226946C6480068483002F074FD20B99DF80000C34981F8480000BF08BD08B5002000901CF0CBFFA0B10021C04800781CF0EFFFBF4849
:4068C00000781DF0EDFB28B10220FFF7DCFF0120009004E00120FFF7D6FF0220009000BF01226946B0480068493002F049FD20B99DF80000AD4981F8490000BFAC48016D43
:406900000120DFF8B0C200DF08BD01B500BF04226946A5480068443002F032FD10B9A3490098486400BF08BD01B5A04890F841009DF80010884215D000BF012269469A486A
:406940000068413002F01CFD20B99DF80000974981F8410000BF18F005FC07F0F6FD1E20F6F7D0FB08BD01B500BF012269468E480068423002F004FD20B99DF800008B4992
:4069800081F8420000BF18F0EDFB2520F6F7BAFB8748C16B0220DFF81CC200DF07F0D5FD08BD01B500BF0422694685480068AC3002F0E6FC18B97D480099C0F89C1400BFC2
:4069C00008BD8048006870477E490860704770B52DED028B04460D4616461CF01DFFF8B17249E0314A5D891C495D501800EBD071491000EE101AB8EEC00AB0EE408ABCEE2A
:406A0000C80A10EE101AC8B2294607F0FDF9BCEEC80A10EE101AC8B2294607F028FA0EE01CF012FF58B16149E031485D294607F0EBF95E49E231485D294607F018FA6248A1
:406A400000EB8400D0ED000AB0EE600A2946204607F0B3F85C490831085D2A46214607F0FEF859490A31085D2A46214607F051F955490C31085D2A46214607F087F946B17B
:406A8000182017F079F94A48016D0120DFF824C100DFBDEC028B70BD70B500240CE0002506E0002229462046FFF791FF681CC5B2022DF6DB601CC4B2022CF0DB182017F024
:406AC0005BF93B48016D0120DFF8E8C000DF70BD70B52DED028B04460D461CF09DFE00B33248D03000EB840090ED000AB1EE400A2E48D83000EB8400D0ED000A30EE200A8D
:406B0000F0EE000A80EE201AB0EE418A2046B1EE480A07F099FA2046B0EE480A07F0FDFA18E01CF091FEA8B12048D03000EB8400D0ED000AB0EE600A204607F085FA1B4866
:406B4000D83000EB8400D0ED000AB0EE600A204607F0E3FA1548C03000EB8400D0ED000AB0EE600A204607F0B5F91048C83000EB8400D0ED000AB0EE600A204607F008FA12
:406B800075B1142017F0F8F8182017F0F5F8142017F0F2F80648016D0120DFF818C000DFBDEC028B70BD0000A4030020081F0020D03F002089E70308F70600201807002051
:406BC000A803002090030020EC20002010B5002405E000212046FFF77BFF601CC4B2022CF7DB142017F0C8F8182017F0C5F8142017F0C2F8FB48016D0120DFF8ECC300DF11
:406C000010BD70B505460C4600212046FFF760FF002221462846FFF7DAFE70BD70B52DED028B05460024B5E0F04890F84900C0EB001105F1380000EB81000E3030F914004D
:406C400000EE900AF8EEE00AB0EE600A204607F029FBE64890F84900C0EB001105F1380000EB8100123030F9140000EE900AF8EEE00AB0EE600A204607F038FBDB4890F8C4
:406C80004900C0EB001105F1380000EB8100163030F9140000EE900AF8EEE00AB0EE600A204607F047FBD14890F84900C0EB001105F1380000EB81001A3030F9140000EEFE
:406CC000900AF8EEE00AB0EE600A204607F056FBC64991F84910C1EB011205F1380101EB82010931085D214607F06CFBBF4991F84910C1EB011205F1380101EB82010B313F
:406D0000085D214607F07CFBB84890F84900C0EB001105F1380000EB8100401C005D00EE100AB8EE400ADFEDB20A80EE201AB0EE418A2046B0EE480A07F080FBAB4991F863
:406D40004910C1EB011205F1380101EB8201C91C085D214607F08BFBA44991F84910C1EB011205F1380101EB8201491D085D214607F091FB9D4991F84910C1EB011205F1D1
:406D8000380101EB8201C91D085D214607F097FB601CC4B2022CFFF647AF944890F84900C0EB001105F1380000EB8100D0ED080AB0EE600A07F03AFABDEC028B70BD8B48AA
:406DC00090F8280008B9012070470020FCE710B5012019F0F9F90146864880F83910002019F0F2F983494874012019F0EDF904462146012010F099FD002019F0E5F904462B
:406E00002146002010F091FD10BD01460020282901D1012200E00022402901D1012300E000231A43492901D1012300E000231A434A2901D1012300E000231A434B2901D12B
:406E4000012300E000231A4302B10120704701460020562901D0612900D10120704701460020592900D10120704710B500245F4890F830000A2803D11CF0E6FC00B1012475
:406E8000204610BD594890F82810082905D0092903D00A2901D00E2901D1012070470020FCE7524890F828100A2901D1012070470020FCE74D4890F82810082901D1012098
:406EC00070470020FCE7494890F82810092901D1012070470020FCE7444890F828100E2901D1012070470020FCE710B504461CF0ABFC70B11CF0BBFC00B92CB901213E488C
:406F000000781CF0CBFC04E000213B4800781CF0C5FC10BD354890F83000C0EB001101EB4010364901EBC000408E70470246012109E001EB0110324B13F81000904201D103
:406F4000C8B27047491C1A29F3DB0020F9E7274890ED0F0A7047254890F84900022801D1012070470020FCE7204890F84900012800D170470020FCE71C4890F8490008B9B6
:406F8000012070470020FCE710B50024FFF7F4FF08B1012419E01CF057FCB0B1FFF7E4FF20B1184800781DF07BF868B9FFF7D3FF58B1F3F74FFA38B9F3F74CFA28B911480B
:406FC00000781DF06DF800B90124204610BD074890F8970020B1054890F89700012813D101207047D03F002089E70308081F00200000C84278CD0020F20600206814040806
:40700000F4100408180700200020EAE74C4890F82800072801D1012070470020FCE7484890F89700022804D0454890F89700032801D1012070470020FCE7414890F8970017
:40704000032801D1012070470020FCE73C4890F89700022801D1012070470020FCE7384890F8970008B9012070470020FCE7344890F89700012800D170470020FCE73048BC
:4070800090F89700042801D1012070470020FCE72B4890F89700042801D1012070470020FCE701B500BF0122694626480068973002F066F920B99DF80000214981F8970050
:4070C00000BF08BD01B500BF012269461D48006800F2853002F054F920B99DF80000184981F8850300BF08BD10B50024144890F8300028281DD0124890F83000402818D022
:407100000F4890F83000492813D00D4890F830004A280ED00A4890F830004B2809D0084890F83000592804D0054890F830005C2800D101242046FFF7C5FF204610BD00000A
:40714000081F0020A40300201FB51CF0A4FB062808D01CF0A0FB072804D01CF09CFB082841F077821CF083FB00287DD0002000900190029003460122FE4903901CF065FC50
:40718000002000900190029003460322FA49039001201CF05AFC002000900190029003460322F649039002201CF04FFC002000900190029003460322F149039010461CF039
:4071C00044FC002000900190029003460322ED49039004201CF039FC002000900190029003460422E849039005201CF02EFC002002220123CDE901200093039003460322AC
:40720000E24906201CF021FC002000900190029003460322DE49039007201CF016FC002000900190029003460322DA49039008201CF00BFC00200090019002900346012223
:40724000D549039009201CF000FC002000900190029003460122D14903900A201CF0F5FB00200090019000E0E0E3029003460122CB4903900B201CF0E8FB002001210090A5
:40728000CDE9010103460A46C64903900C201CF0DCFB002000900190029003460246C249039011201CF0D1FB002000900190029003460322BD49039012201CF0C6FB0020C8
:4072C0000222CDE9000202900346B949039016201CF0BBFB002001210090CDE9010103460A46B449039017201CF0AFFB002000900190029003460222AF49039019201CF09A
:40730000A4FB00200222CDE9000202900346AB4903901A201CF099FB002000900190029001230222A64903901B201CF08EFB002000900190029001230222A24903901C2034
:407340001CF083FB00200222CDE90002029003469D4903901E201CF078FB00200222CDE90002029003460246984903901F201CF06CFB002000900190029003460322944913
:40738000039021201CF061FB0020009001900290034603228F49039022201CF056FB0020009001900290034603228B49039023201CF04BFB002000900190029003460322C8
:4073C0008649039024201CF040FB0020009001900290034603228249039025201CF035FB0020009001900290034603227D49039026201CF02AFB0020009001900290034653
:4074000001227949039027201CF01FFB0020009001900290034601227449039028201CF014FB0020009001900290034601227049039029201CF009FB0020009001900290BE
:40744000034602226B4903902B201CF0FEFA002000900190029003460222674903902C201CF0F3FA002000900190029003460122624903902D201CF0E8FA00200090019048
:407480000290034601225E4903902E201CF0DDFA002000900190029003460122594903902F201CF0D2FA0020009001900290034601225549039031201CF0C7FA002000908A
:4074C00001900290034601225049039032201CF0BCFA00200121CDE9000103460A46CDE902104B4936201CF0B0FA002000900190029003460122474903903B201CF0A5FA5B
:40750000002000900190029003460122424903903C201CF09AFA00200122CDE90002029003463E4903903D201CF08FFA00200122CDE9000202900346394903903E201CF0BB
:4075400084FA002001210090CDE9010103460A463449039041201CF078FA0020009001900290034601223049039042201CF06DFA00205BE0BB060020D8060020D706002024
:407580001C0700201D070020DB060020DC060020D6060020D9060020EF060020EE060020ED06002010070020A4060020E106002097060020AE060020980600209D060020F0
:4075C0001E0700201F0700209C060020A10600209106002093060020E4060020E5060020E6060020E7060020E9060020E8060020EA060020EB060020EC060020DD06002086
:40760000DF060020DE060020F0060020F1060020F2060020F4060020F5060020F6060020F7060020F8060020C206002000900190029003460122FE49039043201CF005FA21
:40764000002000900190029003460122F949039044201CF0FAF9002001210090CDE9010103460A46F449039048201CF0EEF9002001210090CDE9010103460A46EF49039057
:407680004B201CF0E2F9002001210090CDE9010103460A46EA4903904D201CF0D6F9002000900190029003460322E64903904F201CF0CBF9012000220092CDE90120134600
:4076C0000246E149039050201CF0BFF9002001210090CDE9010103460A46DC49039051201CF0B3F9002000900190029003460122D749039052201CF0A8F9002000900190FB
:40770000029003460322D349039054201CF09DF9002000900190029003460322CE49039055201CF092F9002000900190029003460322CA49039056201CF087F900200090F4
:407740000190029003460322C549039057201CF07CF900200222CDE90002029003460246C049039057201CF070F9002000900190029003460322BC49039058201CF065F97D
:40778000002000900190029003460322B749039059201CF05AF9002000900190029003460322B34903905A201CF04FF9002000900190029003460322AE4903905B201CF02D
:4077C00044F9002001210090CDE9010103460A46A94903905C201CF038F9002000900190029003460122A54903905D201CF02DF9002000900190029003460122A0490390C1
:407800005E201CF022F90020009001900290034601229C4903905F201CF017F900200222CDE900020290034601229749039061201CF00BF900200222CDE90002029003467C
:4078400001229249039062201CF0FFF80020009001900290034601228D49039064201CF0F4F80020009001900290034601228949039065201CF0E9F8002001210090CDE930
:40788000010103460A468449039067201CF0DDF8002001210090CDE9010103460A467F49039069201CF0D1F800200222CDE900020290034602467A4903906A201CF0C5F8C1
:4078C00001200021009101910B460246CDE9021074496B201CF0B9F800200222CDE9000202900346704903906D201CF0AEF800200222CDE90002029003466C4903906E20AE
:407900001CF0A3F800200222CDE9000202900346674903906F201CF098F8002001210090CDE9010103460A466249039073201CF08CF800200222CDE90002029003460246B8
:407940005D49039079201CF080F8002000900190029003460222594903907A201CF075F8002000900190029003460122544903907B201CF06AF80020009001900290034695
:407980000122504903907C201CF05FF80020009001900290034601224B4903907D201CF054F8002001210090CDE9010103460A46464903907E201CF048F8002000900190AE
:4079C000029003460122424903907F201CF03DF8002001210090CDE90101034602223D49039082201CF031F8002001210090CDE90101034602223849039083201CF025F8CD
:407A0000002001210090CDE90101034602223349039084201CF019F801200021009101910B460222CDE902102D495BE0DAE00000F9060020FA0600202007002021070020A4
:407A40000F070020DA060020FB060020FC060020FD06002025070020260700202707002028070020A90600200207002003070020040700209F0600200507002007070020C8
:407A80000807002006070020E3060020E2060020090700200A0700200C0700200E070020CF060020BC0600202207002023070020240700201107002013070020140700202E
:407AC000B5060020B6060020150700201607002012070020BF060020C0060020C10600201807002086201BF0B0FF01200021009101910B460222CDE90210FE4987201BF031
:407B0000A4FF01200021009101910B460246CDE90210F94988201BF098FF002000900190029003460322F54903908E201BF08DFF002000900190029003460322F0490390EC
:407B40008F201BF082FF002000900190029003460322EC4903908F201BF077FF012008F0C0FD0021E84800781BF098FE0021E74800781BF093FE0021E54800781BF08EFE90
:407B80000021E44800781BF089FE01200021009101910B460222CDE90210DF4986201BF054FF01200021009101910B460222CDE90210DA4987201BF048FF0121D848007828
:407BC0001CF0F1FA0121D74800781CF0ECFA0121D54800781CF0E7FA0121D44800781CF0E2FAE1E3002000900190029003460122CF4903901BF029FF0020009001900290ED
:407C000003460322C649039001201BF01EFF002000900190029003460322C249039002201BF013FF002000900190029003460322C049039010461BF008FF00200090019047
:407C4000029003460322BC49039004201BF0FDFE002000900190029003460422B749039005201BF0F2FE002002220123CDE901200093039003460322B14906201BF0E5FE6C
:407C8000002000900190029003460322A749039007201BF0DAFE002000900190029003460322A149039008201BF0CFFE002000900190029003460122A249039009201BF047
:407CC000C4FE0020009001900290034601229E4903900A201BF0B9FE002000900190029003460122994903900B201BF0AEFE002001210090CDE9010103460A4694490390F4
:407D00000C201BF0A2FE0020009001900290034603229049039011201BF097FE0020009001900290034603228B49039012201BF08CFE00200222CDE90002029003468749D8
:407D4000039016201BF081FE002001210090CDE9010103460A466E49039017201BF075FE0020009001900290034602227C49039019201BF06AFE00200222CDE900020290BC
:407D80000346784903901A201BF05FFE002000900190029001230222734903901B201BF054FE0020009001900290012302226F4903901C201BF049FE00200222CDE9000292
:407DC000029003466A4903901E201BF03EFE00200222CDE90002029003460246654903901F201BF032FE00200222CDE900020290034602466049039020201BF026FE002019
:407E0000009001900290034603225C49039021201BF01BFE0020009001900290034603225749039022201BF010FE0020009001900290034603225349039023201BF005FEF4
:407E40000020009001900290034603224E49039024201BF0FAFD0020009001900290034603224A49039025201BF0EFFD0020009001900290034603224549039026201BF0FB
:407E8000E4FD0020009001900290034601224149039027201BF0D9FD0020009001900290034601223C49039028201BF0CEFD0020009001900290034601223849039029204C
:407EC0001BF0C3FD002000900190029003460222334903902B201BF0B8FD0020009001900290034602222F4903902C201BF0ADFD002059E0190700201A070020C806002049
:407F0000C9060020C706002005070020FC060020AE060020F1060020AB060020AA060020D8060020D7060020D9060020D6060020BB0600201C0700201D070020DB0600202C
:407F4000DC060020EF060020EE060020ED06002010070020A5060020E106002097060020980600209D0600201E0700201F0700209C060020A1060020A806002091060020E3
:407F800093060020E4060020E5060020E6060020E7060020E9060020E8060020EA060020EB060020EC06002000900190029003460122FE4903902D201BF047FD0020009045
:407FC0000190029003460122F94903902E201BF03CFD002000900190029003460122F54903902F201BF031FD002000900190029003460122F049039031201BF026FD002049
:4080000000900190029003460122EC49039032201BF01BFD00200121CDE9000103460A46CDE90210E64936201BF00FFD002000900190029003460122E24903903B201BF08B
:4080400004FD002000900190029003460122DE4903903C201BF0F9FC00200122CDE9000202900346D94903903D201BF0EEFC00200122CDE9000202900346D54903903E20E8
:408080001BF0E3FC002001210090CDE9010103460A46D049039041201BF0D7FC002000900190029003460122CB49039042201BF0CCFC002000900190029003460122C7495E
:4080C000039043201BF0C1FC002000900190029003460122C249039044201BF0B6FC002001210090CDE9010103460A46BD49039048201BF0AAFC002001210090CDE9010165
:4081000003460A46B84903904B201BF09EFC002001210090CDE9010103460A46B34903904D201BF092FC002000900190029003460322AF4903904F201BF087FC012000223E
:408140000092CDE9012013460246AA49039050201BF07BFC002001210090CDE9010103460A46A549039051201BF06FFC002000900190029003460122A049039052201BF0BA
:4081800064FC0020009001900290034603229C49039054201BF059FC0020009001900290034603229749039055201BF04EFC0020009001900290034603229349039056202E
:4081C0001BF043FC0020009001900290034603228E49039057201BF038FC0020009001900290034603228A49039058201BF02DFC00200090019002900346032285490390DF
:4082000059201BF022FC002000900190029003460322814903905A201BF017FC0020009001900290034603227C4903905B201BF00CFC002001210090CDE9010103460A461C
:40824000774903905C201BF000FC002000900190029003460122734903905D201BF0F5FB0020009001900290034601226E4903905E201BF0EAFB002000900190029003460F
:4082800001226A4903905F201BF0DFFB00200222CDE900020290034601226549039061201BF0D3FB00200222CDE900020290034601226049039062201BF0C7FB0020009027
:4082C00001900290034601225B49039064201BF0BCFB0020009001900290034601225749039065201BF0B1FB002001210090CDE9010103460A465249039067201BF0A5FB41
:40830000002001210090CDE9010103460A464D49039069201BF099FB00200222CDE90002029003460246484903906A201BF08DFB01200021009101910B460246CDE90210A3
:4083400042496B201BF081FB00200222CDE90002029003463E4903906D201BF076FB00200222CDE90002029003463A4903906E201BF06BFB00200222CDE9000202900346A3
:40838000354903906F201BF060FB002001210090CDE9010103460A463049039073201BF054FB002002225BE053E10000DD060020DF060020DE060020F0060020F1060020AF
:4083C000F2060020F4060020F5060020F6060020F7060020F8060020C2060020F9060020FA06002020070020210700200F070020DA060020FB060020FC060020FD06002087
:40840000250700202607002027070020280700200207002003070020040700209F06002005070020070700200807002006070020E3060020E2060020090700200A0700209B
:408440000C0700200E070020CF060020BC06002022070020230700202407002011070020CDE90002029003460246FE49039079201BF0EBFA00200090019002900346022229
:40848000F94903907A201BF0E0FA002000900190029003460122F54903907B201BF0D5FA002000900190029003460122F04903907C201BF0CAFA0020009001900290034651
:4084C0000122EC4903907D201BF0BFFA002001210090CDE9010103460A46E74903907E201BF0B3FA002000900190029003460122E24903907F201BF0A8FA002001210090D9
:40850000CDE9010103460222DD49039082201BF09CFA002001210090CDE9010103460222D849039083201BF090FA002001210090CDE9010103460222D349039084201BF0E2
:4085400084FA01200021009101910B460222CDE90210CE4986201BF078FA01200021009101910B460222CDE90210C94987201BF06CFA01200021009101910B460246CDE921
:408580000210C44988201BF060FA002000900190029003460322C04903908E201BF055FA002000900190029003460322BB4903908F201BF04AFA00200090019002900346B8
:4085C0000322B74903908F201BF03FFA012008F088F80021B34800781BF060F90021B24800781BF05BF90021B04800781BF056F90021AF4800781BF051F9012000210091AA
:4086000001910B460222CDE90210AA4986201BF01CFA01200021009101910B460222CDE90210A54987201BF010FA0121A34800781BF0B9FD0121A24800781BF0B4FD0121BD
:40864000A04800781BF0AFFD01219F4800781BF0AAFD1FBD1FB50020009001900290034603229A49039001201BF0EFF90020009001900290034603229549039002201BF056
:40868000E4F90020009001900290034603229149039010461BF0D9F90020009001900290034603228C49039004201BF0CEF900200090019002900346042288490390052092
:4086C0001BF0C3F90020009001900290034603228349039006201BF0B8F90020009001900290034603227F49039007201BF0ADF90020009001900290034603227A49039026
:4087000008201BF0A2F90020009001900290034602225549039009201BF097F90020009001900290034602227049039017201BF08CF90020009001900290034602466C49CA
:40874000039019201BF081F90020009001900290034603226749039021201BF076F90020009001900290034603226349039022201BF06BF9002000900190029003460222F8
:408780004D49039027201BF060F90020009001900290034602224749039028201BF055F90020009001900290034602465349039029201BF04AF901200021009101910B4601
:4087C0000A46CDE902104E492A201BF03EF90020009001900290034602464A4903902B201BF033F9002000900190029003460122454903902D201BF028F900200090019018
:40880000029003460246414903902E201BF01DF90020009001900290034602463C4903902F201BF012F90020009001900290034602463849039030201BF007F90020009025
:4088400001900290034602463349039046201BF0FCF80020009001900290034602462F4903905DE01307002014070020B5060020B606002015070020160700201207002046
:40888000BF060020C0060020C106002018070020190700201A070020C8060020C9060020C706002005070020FC060020AE060020F1060020AB060020AA060020D8060020A4
:4088C000D7060020D9060020D6060020E406002091060020920600209306002094060020E70600209506002096060020C30600209B0600209E0600209F060020AC0600200B
:40890000A5060020A2060020CC060020CD060020CE060020CF060020A0060020D106002047201BF092F8002000900190029003460246F649039048201BF087F80020009045
:408940000190029003460122F149039057201BF07CF8002000900190029003460222ED49039059201BF071F8002000900190029003460222E84903905A201BF066F80020A8
:4089800000900190029003460122E44903905B201BF05BF8002000900190029003460122DF4903905C201BF050F8002000900190029003460122DB4903905D201BF045F87B
:4089C000002000900190029003460122D64903905E201BF03AF8002000900190029003460122D24903905F201BF02FF8002000900190029003460122CD49039060201BF0BA
:408A000024F8002000900190029003460122C949039061201BF019F8002000900190029003460122C449039064201BF00EF8002000900190029003460122C04903906520C5
:408A40001BF003F8002000900190029003460122BB49039066201AF0F8FF002000900190029003460122B749039067201AF0EDFF002000900190029003460122B249039077
:408A800068201AF0E2FF002000900190029003460122AE49039069201AF0D7FF002000900190029001231A46A94903906A201AF0CCFF002000900190029003460122A549A9
:408AC00003906C201AF0C1FF002000900190029003460122A04903906D201AF0B6FF0020009001900290034601229C4903906E201AF0ABFF01200021009101910B460A4687
:408B0000CDE9021096497C201AF09FFF01200021009101910B460A46CDE9021091497D201AF093FF002001210090CDE9010103460A468D49039081201AF087FF00200090FC
:408B400001900290034602228849039082201AF07CFF0020009001900290034602228449039083201AF071FF0020009001900290034602227F49039084201AF066FF00204F
:408B8000009001900290034602227B49039086201AF05BFF0020009001900290034602227649039087201AF050FF0020009001900290034602467249039088201AF045FFFA
:408BC0000020009001900290034603226D4903908D201AF03AFF002000900190029003460322694903908E201AF02FFF002000900190029003460322644903908F201AF055
:408C000024FF0121584800781AF048FE0121604800781AF043FE01215E4800781AF03EFE1FBD1FB500240CE000205B4901EB041189680870584901EB0411C9680870601CBF
:408C4000C4B2902CF0DB1AF07BFD1BF019FC1EF05BFF0121022021F01AFA0020009001900290034601224D49039016201AF0EDFE002001210090CDE9010103460A4648493D
:408C800003901E201AF0E1FE002000900190029003460122434903906B201AF0D6FE1AF0FAFDFF2831D00121084621F0F0F90121042021F0ECF90121082021F0E8F9012106
:408CC000102021F0E4F90121202021F0E0F90121402021F0DCF90121802021F0D8F90121080221F0D4F91AF0D6FD0A2862D2DFE800F06105060708095B5C5D5E00BF00BF86
:408D000000BF00BFFFF7A6FC55E055E0A1060020D5060020AD060020AE060020AF060020B0060020B1060020D2060020D3060020D4060020B2060020F5060020F6060020CE
:408D4000B5060020B6060020B7060020B8060020B9060020BC060020BD060020BE060020A8060020A7060020C2060020BF060020C0060020C1060020D8060020D7060020C9
:408D8000C4060020C7060020C8060020C9060020C5060020C606002048300408970600209C060020BB06002000BF00BF00BFFEF7CBF900E000BF00BF1FBD10B50120FE49E7
:408DC00008701DF0E6F8FC494860012021F010F81CE0612020F0AEFF78B145F25550F74908600120486040F6B83088604CF6CC4008600220F049087008E0EF4948681DF0CD
:408E0000F0F8642802D90320EB490870EA4800780128DED010BD10B50020E74908704FF4FA701DF08FF8FA201DF0CDF8FFF7C5FFFFF7F7FE1AF0F0FCC8B1E14800781BF04C
:408E40002FF940B90121DF4800781AF027FD0020DD4908700BE0DD4800781BF021F918B10220D949087002E00120D749087019F045FFEFF727FA00221146D548DFF854C37F
:408E800000DF002010BD10B572B66FF0040000F054FA6FF0010000F050FA4FF0FF3000F04CFA042000F049FA052000F046FA062000F043FA072000F040FA082000F03DFA7B
:408EC000092000F03AFA0A2000F037FA0B2000F034FA0C2000F031FA0D2000F02EFA0E2000F02BFA0F2000F028FA102000F025FA112000F022FA122000F01FFA132000F0A7
:408F00001CFA142000F019FA152000F016FA162000F013FA172000F010FA182000F00DFA192000F00AFA1A2000F007FA1B2000F004FA1C2000F001FA1D2000F0FEF91E2012
:408F400000F0FBF91F2000F0F8F9202000F0F5F9212000F0F2F9222000F0EFF9232000F0ECF9242000F0E9F9252000F0E6F9262000F0E3F9272000F0E0F9282000F0DDF927
:408F8000292000F0DAF92A2000F0D7F92B2000F0D4F92C2000F0D1F92D2000F0CEF92E2000F0CBF92F2000F0C8F9302000F0C5F9312000F0C2F9322000F0BFF9332000F050
:408FC000BCF9342000F0B9F9352000F0B6F9362000F0B3F9372000F0B0F9382000F0ADF9392000F0AAF93A2000F0A7F93B2000F0A4F93C2000F0A1F93D2000F09EF93E201C
:4090000000F09BF93F2000F098F9402000F095F9412000F092F9422000F08FF9432000F08CF9442000F089F9452000F086F9462000F083F9472000F080F9482000F07DF946
:40904000492000F07AF94A2000F077F94B2000F074F94C2000F071F94D2000F06EF94E2000F06BF94F2000F068F9502000F065F9512000F062F96FF0040000F067F96FF0FA
:40908000010000F063F94FF0FF3000F05FF9042000F05CF9052000F059F9062000F056F9072000F053F9082000F050F9092000F04DF90A2000F04AF90B2000F047F90C2071
:4090C00000F044F90D2000F041F90E2000F03EF90F2000F03BF9102000F038F9112000F035F9122000F032F9132000F02FF9142000F02CF9152000F029F9162000F026F937
:40910000172000F023F9182000F020F9192000F01DF91A2000F01AF91B2000F017F91C2000F014F91D2000F011F91E2000F00EF91F2000F00BF9202000F008F9212000F0BA
:4091400005F9222000F002F9232000F0FFF8242000F0FCF8252000F0F9F8262000F0F6F8272000F0F3F8282000F0F0F8292000F0EDF82A2000F0EAF82B2000F0E7F82C2046
:4091800000F0E4F82D2000F0E1F82E2000F0DEF82F2000F0DBF8302000F0D8F8312000F0D5F8322000F0D2F8332000F0CFF8342000F0CCF835200FE09803002000300040FC
:4091C000A2060020BE06002094030020CF060020BF1A02089DEF030800F0B8F8362000F0B5F8372000F0B2F8382000F0AFF8392000F0ACF83A2000F0A9F83B2000F0A6F869
:409200003C2000F0A3F83D2000F0A0F83E2000F09DF83F2000F09AF8402000F097F8412000F094F8422000F091F8432000F08EF8442000F08BF8452000F088F8462000F02C
:4092400085F8472000F082F8482000F07FF8492000F07CF84A2000F079F84B2000F076F84C2000F073F84D2000F070F84E2000F06DF84F2000F06AF8502000F067F8512030
:4092800000F064F862B610BD38B5044660680090009D206880F3088800BFA84738BD00BFBFF34F8F2E48006800F4E0602D490843001D2B490860BFF34F8F00BF00BFFEE715
:4092C00010B50021284800781AF0E8FA0021274800781AF0E3FA01DF10BD01B500BF04226946234800688C3000F04AF818B921480099C0F87C1400BF08BD01B500BF0422D3
:4093000069461B480068903000F03AF818B919480099C0F8801400BF08BD01B500BF0422694613480068943000F02AF818B911480099C0F8841400BF08BD00F01F02012189
:4093400091400D4A430942F82310704700F01F0201219140094A430942F82310704700000CED00E00000FA05F60600200B070020A8030020081F002080E100E080E200E0D3
:4093800070B504460D461646324629462046EFF73EFD70BD2DE9F34F82B0844600BF00210A460B460E460F46002001908046009063E09CF80000A0F13004E5179CF8000043
:4093C0002E2838D1B8F1000F0CD1F9494FF00009A2FB010A03FB01A102FB0919861949EB07071FE0B8F1010F0CD1F2494FF00009A2FB010A03FB01A102FB0919861949EB55
:4094000007070FE0B8F1020F0CD14FF47A714FF00009A2FB010A03FB01A102FB0919861949EB070708F1010000F0FF0800200090002213461BE09CF80000C0B1009810B95D
:4094400022462B460FE0009801280CDB0A214FF0000B9146A9FB010E03FB01E102FB0B19021949EB05030098401CC0B200900CF1010C0198401CC0B201900399019888422E
:4094800097DBB6185F413046394604B0BDE8F08F2DE9F04F83468946924600BF00BF51465846FFF777FF05460E4651464846FFF771FF07468846781B78EB060001DA0124DA
:4094C00007E0E81B76EB080002DA4FF0FF3400E000242046BDE8F08FF0B585B00546B6A2B8A101A821F01EFF1022294601A8FFF7CFFF00283CDDB44890F82464012434E0FC
:40950000062C0CD2DFE804F00B0C09070503AF4F08E0AF4F06E0AF4F04E0AF4F02E000BFAE4F00BF00BF40F6C41000900222694607F56070FFF724FFB44204D1BDF8000099
:40954000A149A1F880034FF47A5000900222694607F28230FFF714FFB44204D1BDF800009949A1F88203601CC4B2052CC8DD00BF05B0F0BD2DE9F04105460E4617463A4695
:4095800031462846EFF7B9FC044604B103DF2046BDE8F081F0B585B0054691A289A101A821F0C0FE1022294601A8FFF771FF00282FDD854890F82474012427E0062C0CD2C7
:4095C000DFE804F00B0C09070503804E08E0804E06E0804E04E0804E02E000BF7F4E00BF00BF042206F5C6716846FFF7C3FF0422694606F56270FFF7C3FEBC4204D19DED37
:40960000000A714880EDE20A601CC4B2052CD5DD00BF05B0F0BDF0B585B0054673A269A101A821F07FFE1022294601A8FFF730FF00282BDD644890F82464012423E0062CE8
:409640000CD2DFE804F00B0C090705035F4F08E05F4F06E05F4F04E05F4F02E000BF5F4F00BF00BF002000900122694607F19700FFF786FEB44204D19DF80000524981F8EC
:409680009700601CC4B2052CD9DD00BF05B0F0BD2DE9F04186B0054657A24AA102A821F041FE1022294602A8FFF7F2FE002836DD002001900026444890F8247400242BE055
:4096C000062C13D2DFE804F0130F0C090603DFF8FC800FE0DFF8F8800CE0DFF8F88009E0DFF8F48006E0DFF8F48003E000BFDFF8148100BF00BF042201A908F1B400FFF728
:409700003FFEBC4206D130490198C1F8B4000846C0F89860601CC4B2052CD1DD00BF06B0BDE8F081F0B587B0064637A225A103A821F0F8FD1022314603A8FFF7A9FE0028AD
:4097400069DD214890F82474002483E0062C0ED2DFE804F00E0B090705031C4D0AE01C4D08E01C4D06E01C4D04E01C4D02E000BF244D00BF00BF042205F1300101A8FFF770
:40978000F9FE13208DF809000198FDF73EFB18B90198FDF764FB18B190208DF808003EE00198FDF754FBA8B313208DF8080036E000CA9A3B40420F00322E342E302E353385
:4097C0000000000025730000081F0020581B00687017006888130068A00F0068B80B0068322E342E302E343400000000322E332E302E333000000000322E322E302E3436E9
:4098000000000000D0070068322E322E302E31380000000000E021E0FF208DF8080001220DF1090105F1B300FFF7AAFD012202A905F1B200FFF7A4FDBC4209D19DF80910D1
:40984000FE4880F8B3109DF80800FC4981F8B200601CC4B2052C7FF779AF00BF07B0F0BDF0B585B00546F6A2AFF2A80101A821F059FD1022294601A8FFF70AFE00282DDDE5
:40988000EE4890F8246401200090002423E0062C0ED2DFE804F00E0B09070503EA4F0AE0EA4F08E0EA4F06E0EA4F04E0EA4F02E000BFEA4F00BF00BF0122694607F14B0066
:4098C000FFF75EFDB44204D19DF80000DB4981F84B00601CC4B2052CD9DD00BF05B0F0BDF0B587B00546DEA2AFF2281103A821F019FD1022294603A8FFF7CAFD002839DD3B
:40990000CE4890F82474002431E0062C0ED2DFE804F00E0B09070503CB4E0AE0CB4E08E0CB4E06E0CB4E04E0CB4E02E000BFCB4E00BF00BF012206F1280102A8FFF71AFE72
:409940009DF80800042810D0B2EE040A8DED010A042201A906F5FC70FFF712FDBC4204D19DED010AB54880ED7E0A601CC4B2052CCBDD00BF07B0F0BDF0B585B00646BAA205
:40998000AFF2C01101A821F0CDFC1022314601A8FFF77EFD002843DD0727B6A2AFF2DC1101A821F0BFFC1022314601A8FFF770FD002800DD09270020009000242DE0062C21
:4099C0000ED2DFE804F00E0B090705039E4D0AE09E4D08E09E4D06E09E4D04E09E4D02E000BF9E4D00BF00BF042205F130016846FFF7C0FD009838440090009814280BD35A
:409A00000422694605F13000FFF7BAFC9348854202D18A4900980863641C062CCFD300BF05B0F0BD2DE9F3410D468449ADEB01040846071988482618AAB239463046FFF7F5
:409A40009FFC7E48071983482618AAB239463046FFF796FC794807197D482618AAB239463046FFF78DFC7548071978482618AAB239463046FFF784FC70480719724826185D
:409A8000AAB239463046FFF77BFCBDE8FC812DE9FE4F81468A46174698460020009000262D2200233846414621F0B2FB05462D2200233846414621F0ABFB934615B9BBF1BA
:409AC000000F35D0D5B1002416E0C4EB041000EB400048440290C4EB041000EB4000504401902D22DDE90110FFF74AFC0646009931430091601CC4B2AC42E6D3BBF1000FF3
:409B000018D0C5EB051000EB400048440290C5EB051000EB4000504401901FFA8BF2DDE90110FFF72DFC064600993143009101E0402000900098BDE8FE8F01B500BF012271
:409B400069464F4800682D30FFF71AFC20B99DF800103A4880F81D1400BF08BD2DE9FE4F81468A46174698460020009000262D2200233846414621F04BFB05462D2200230B
:409B80003846414621F044FB934615B9BBF1000F35D0D5B1002416E0C4EB041000EB400048440290C4EB041000EB4000504401902D22DDE90110FFF7DDFC064600993143DC
:409BC0000091601CC4B2AC42E6D3BBF1000F18D0C5EB051000EB400048440290C5EB051000EB4000504401901FFA8BF2DDE90110FFF7C0FC064600993143009101E040202B
:409C000000900098BDE8FE8F3EB5002002900A200190002000904FF47B71084821F013FDB021184821F00FFD4FF458711548B03021F009FD012201A9114825E0081F0020FA
:409C4000322E322E302E3200581B00687017006888130068A00F0068B80B0068D0070068322E322E302E3100322E312E302E373300000000322E312E302E353400000000EA
:409C8000A8030020F822002000689830FFF778FB0122FB480168983102A8FFF76BFC9DF80800401CC0B20190012201A9F44800689830FFF765FB0122F1480168983102A8A4
:409CC000FFF758FC9DF808009DF80410884207D0EC48007840F08000EA49087001248CE00122E74801682E316846FFF743FC9DF8000044284CD0FF224FF47B71E24821F0F6
:409D000078FC4FF47B720023DF49E048FFF7BFFE4FF47B720023DC49DD48FFF7B8FE4FF47B720023D849DB48FFF7B1FE4FF47B720023D549D848FFF7AAFE4FF47B72002352
:409D4000D149D648FFF7A3FE4FF47B720023CE49D348FFF79CFE4FF47B71CB4821F073FCB0220023CF494FF0D040FFF790FE4FF458720023CB49B031CB48FFF788FE442045
:409D8000009001226946BE4800682E30FFF7F8FAB02200234FF0D041C248FFF7DFFE4FF458720023C049BF48B030FFF7D7FE0122B34801682D31BB482D30FFF7DBFBB24875
:409DC00090F81D04672810D001246720FFF7B5FE4FF47B71AC4821F036FC4FF47B720023A949AA48FFF753FE07E002244FF47B720023A649A448FFF7B1FE20463EBD10B50C
:409E0000AA48EEF7B3FF0446204610BD70B58CB000240020089009900A900B9004900590069007900090019002900390954908709F49087001200870FFF7E1FFFFF7E4FE78
:409E40009C4908709C4AAFF2846108A821F06AFA04A81AF00DFB99A104A821F01BFC08B1012000E00020054645B196A01AF0ECFA92A01AF0E9FA97A01AF0CCFA04A81AF00B
:409E8000DBFA102204A908A8FFF702FB044689480078012806D100208549087008A81AF0B9FAC3E0002CFCD0002005F063FA002005F0B3FA08A81AF0ADFA002C39DA002056
:409EC000FFF73BFEFF224FF47B716F4821F091FB4FF47B7200236C496C48FFF7D8FD4FF47B72002368496A48FFF7D1FD4FF47B72002365496748FFF7CAFD4FF47B720023CE
:409F000061496548FFF7C3FD4FF47B7200235E496248FFF7BCFD4FF47B7200235A496048FFF7B5FD4FF47B71574821F08CFB03DF7CE06AA2AFF27471684621F0F3F9102268
:409F400004A96846FFF7A4FA002838DD0020FFF7F4FDFF224FF47B714B4821F04AFB4FF47B72002348494948FFF791FD4FF47B72002345494648FFF78AFD4FF47B7200233D
:409F800041494448FFF783FD4FF47B7200233E494148FFF77CFD4FF47B7200233A493F48FFF775FD4FF47B72002337493C48FFF76EFD4FF47B71344821F045FB03DF4AA2FC
:409FC000AFF60001684621F0ADF9102204A96846FFF75EFA002811DD012007F0F9FA01212948B130FFF71EFD19F016FC30B10320F2F71EF801213F48FFF714FD04A8FFF765
:40A00000BBFC04A8FFF76CFC04A8FFF729FC04A8FFF788FB04A8FFF73BFB04A8FFF7FBFA04A8FFF7B7FA04A8FFF756FA0020FCF7B8FC0020FCF7C8FCFDF756F80646FCF7A0
:40A0400054FF1B4800780CB070BD19480078704701B500BF01226946094800683430FFF78FF920B99DF80010074880F8241400BF2148C16B0220DFF884C000DF08BD0000A5
:40A08000A8030020A1030020081F0020D0070068B80B0068A00F00688813006870170068581B0068F8220020F401006800380040A2030020A00300209CBE0008322E302EC5
:40A0C0003100000030303030303030303030303000000000322E302E302E3100322E302E302E363500000000322E312E302E333900000000BB200020D03F002089E70308ED
:40A100007CB505460E46FE4C042204F1340101A8FFF730FA012204F1B1016846FFF72AFA0198854205D19DF80000B04201D101207CBDF44C042204F1340101A8FFF71AFA2E
:40A14000012204F1B1016846FFF714FA0198854205D19DF80000B04201D10220E8E7EA4C042204F1340101A8FFF704FA012204F1B1016846FFF7FEF90198854205D19DF890
:40A180000000B04201D10320D2E7E04C042204F1340101A8FFF7EEF9012204F1B1016846FFF7E8F90198854205D19DF80000B04201D10420BCE7D64C042204F1340101A83D
:40A1C000FFF7D8F9012204F1B1016846FFF7D2F90198854205D19DF80000B04201D10520A6E70020A4E738B5C54C042204F5EC716846FFF7BFF940F2FD110098884201D02A
:40A20000012038BDBF4C042204F5EC716846FFF7B1F940F2FD110098884201D00220F0E7B94C042204F5EC716846FFF7A3F940F2FD110098884201D00320E2E7B34C042282
:40A2400004F5EC716846FFF795F940F2FD110098884201D00420D4E7AD4C042204F5EC716846FFF787F940F2FD110098884201D00520C6E70020C4E710B54FF47B71A5487A
:40A2800021F0E1F94FF47B720023A249A248FFF7FEFB10BD10B54FF47B719E4821F0D3F94FF47B7200239B499B48FFF7F0FB4FF47B72002397499248FFF7E9FB4FF47B7206
:40A2C000002394498F48FFF7E2FB4FF47B72002390498D48FFF7DBFB4FF47B7200238D498A48FFF7D4FB4FF47B72002389498848FFF7CDFB4FF47B71864821F0A4F910BDFC
:40A300002DE9F0410446884615461F463CB982482E183A4641463046FFF732F830E0012C07D177482E183A4641463046FFF728F826E0022C07D173482E183A464146304625
:40A34000FFF71EF81CE0032C07D16F482E183A4641463046FFF714F812E0042C07D16B482E183A4641463046FFF70AF808E0052C06D167482E183A4641463046FFF700F89A
:40A38000BDE8F0812DE9F04104460F46154698463CB961482E18424631463846FFF7EAF830E0012C07D156482E18424631463846FFF7E0F826E0022C07D152482E18424677
:40A3C00031463846FFF7D6F81CE0032C07D14E482E18424631463846FFF7CCF812E0042C07D14A482E18424631463846FFF7C2F808E0052C06D146482E184246314638464E
:40A40000FFF7B8F8BDE8F08110B5424890F82444062C2CD2DFE804F02C030B131B234FF47B7200233B493648FFF731FB21E04FF47B72002337493348FFF729FB19E04FF48F
:40A440007B72002333493048FFF721FB11E04FF47B7200232F492D48FFF719FB09E04FF47B7200232B492A48FFF711FB01E000BF00BF00BF10BD70B505460E4631462846D3
:40A48000FFF73EFE0446062C6CD2DFE804F06C03152747594FF47B72002319491D48FFF75DFB4FF47B7200231A491B48FFF7EFFA0120FFF7CDFD62E04FF47B72002311497A
:40A4C0001448FFF74BFB4FF47B72002311491248FFF7DDFA0220FFF7BBFD50E04FF47B72002309490B48FFF739FB4FF47B72002308490948FFF7CBFA0320FFF7A9FD3EE041
:40A50000B80B0068A00F00688813006870170068581B0068081F0020D00700684FF47B72002339493948FFF719FB4FF47B72002336493748FFF7ABFA0420FFF789FD1EE09C
:40A540004FF47B72002333493048FFF707FB4FF47B7200232D492E48FFF799FA0520FFF777FD0CE000BFFFF787FE0020FFF770FD002029494860222013F0FEFB00BF00BFA6
:40A5800004B103DF70BD4FF40050704710B51F4890F82404062831D2DFE800F031030C151E271E4C042219493C3104F13C00FEF7E7FE25E01A4C042214493C3104F13C0039
:40A5C000FEF7DEFE1CE0174C042210493C3104F13C00FEF7D5FE13E00B4C04220B493C3104F13C00FEF7CCFE0AE00A4C042207493C3104F13C00FEF7C3FE01E000BF00BFBC
:40A6000000BF10BD0848704770170068081F0020D0070068581B0068C02F0020B80B0068A00F006888130068AFD3D73B10B51BF0B0FCF949086008F003FFF74880ED010A78
:40A6400010BD10B5F54890F83800032804D1F34890F8900003280AD0FBF74EFBC4B22346FA22ED490C3102200CF01EF948E0EC4890F84A0002281FD1E84890ED020ADFED48
:40A68000E90AB4EEE00AF1EE10FA0ADBFBF734FBC4B223467D22E0490C3101200CF004F92EE0FBF729FBC4B223467D22DA490C3100200CF0F9F823E0D848D0ED010AD84814
:40A6C000B0F8BE0100EE100AB8EE400AF4EEC00AF1EE10FA0ADBFBF70FFBC4B22346FA22CD490C3101200CF0DFF809E0FBF704FBC4B22346FA22C8490C3100200CF0D4F838
:40A7000010BD10B52DED048B19F09EF8002867D0FFF797FFEFF79EFE18B10020BE49087261E0BD48007A60B9BB4890F82000002859D10120B84908721BF02BFCB64908605D
:40A7400051E0B548007A01280CD1B349C86947F230511BF024FCA0B30220AF490872FFF765FF40E0AC48007A02283CD108F068FEA948D0ED010A30EEC00A10EE104A204656
:40A7800025F0E8FC41EC190BB0EE490AF0EE690A22F0BAF8B0EE408AF0EE608A9FEDA20B53EC102B51EC180B25F0DCFA0ED29A4890F82000012805D10020974948720120D7
:40A7C000087210E00120944948720CE0924908684FF4FA611BF0E3FB28B1FFF727FF02E000208D494872BDEC048B10BD8B4981F890007047894981F838007047F0EE400AF7
:40A800009FED8B0A20EE800A704770B52DED0A8B0446834890F8BD010E287DD2DFE800F07C355DFB36FAF9F87C7C077C7CF7EFF70DFE10EE105A284625F08CFC41EC1A0B6F
:40A84000B0EE4A0AF0EE6A0A22F05EF8B0EE409AF0EE609A51EC190B24F040FEA0619FED750A84ED1C0A94ED060A84ED010AEFF735FE18B10020FFF7BDFF02E00320FFF7CA
:40A88000B9FF0320FFF7B2FF32E300BF6A48007819F006FC20B19FED690A84ED060A03E09FED640A84ED060A6548007819F0F8FB20B19FED620A84ED1C0A03E09FED5D0A07
:40A8C00084ED1C0A0320FFF795FF0320FFF78EFF94ED060A84ED010A0AE35748007819F0A3F900EE100AF8EE400A9FED561A9FED560A10EE810A84ED0C0AE16821611BF0B2
:40A9000048FBE060D4E90310091A6161D4ED0C0AB0EE600A0A2100E0DBE204F1180009F02BFD94ED060ADFED490AB4EEE00AF1EE10FA03D20020FFF75DFF0FE094ED060A1E
:40A94000F0EE040AB4EEE00AF1EE10FA03DD0120FFF750FF02E00320FFF74CFF0320FFF745FF94ED0C0AB5EEC00AF1EE10FA02D29FED308A01E094ED068A94ED0F0A84ED89
:40A98000100A84ED0F8A94ED050AB8EE400ADFED2B0A80EE201A11EE105A284625F0DAFB41EC1A0B94ED0F0AD4ED100A30EE600A10EE101A084625F0CDFB41EC1C0BB0EEF5
:40A9C0004C0AF0EE6C0A21F09FFFB0EE40BAF0EE60BA53EC1A2B51EC1B0B24F06DFE41EC190B24F07BFD60639FED120A84ED1C0AB0EE480AFFF702FF84ED010AD4ED0D0AEE
:40AA0000B0EE600AFFF7FAFE84ED020A70E251E2A1E10CE11CE063E0082700202C270020081F002000C0DA44000000401857B63FC0A9064600000000D606002000007A4476
:40AA4000DA0600203333533A9A99193FCDCCCCBEF948007819F0E8F800EE100AB8EE400A5FED080A20EE200ADFEDF40A80EE201A84ED0C1AD4ED0C0AB0EE600A0A2104F1FD
:40AA8000180009F079FC94ED060ADFEDED0AB4EEE00AF1EE10FA03D20020FFF7ABFE0FE094ED060ADFEDE70AB4EEE00AF1EE10FA03DD0120FFF79EFE02E00320FFF79AFEDB
:40AAC0000320FFF793FE1FED250A84ED1C0AD4ED060AB0EE600AFFF791FE84ED010A07E2D548007819F0A0F800EE100AF8EE400A1FED2C1A1FED2C0A10EE810A84ED0C0A05
:40AB0000D4ED0C0AB0EE600A0A2104F1180009F033FC94ED060A5FED330AB4EEE00AF1EE10FA03D20020FFF765FE0FE094ED060AF0EE040AB4EEE00AF1EE10FA03DD012017
:40AB4000FFF758FE02E00320FFF754FE94ED0C0AB5EEC00AF1EE10FA02D21FED4A8A01E094ED068AB848007819F05EF800EE100AF8EE400A1FED4D1A1FED4D0A10EE810A3B
:40AB800084ED220AD4ED220AB0EE600A0A2104F1700009F0F1FB94ED1C0A5FED540AB4EEE00AF1EE10FA03D20020FFF71FFE0FE094ED1C0AF0EE040AB4EEE00AF1EE10FAC9
:40ABC00003DD0120FFF712FE02E00320FFF70EFE94ED220AB5EEC00AF1EE10FA02D25FED6B8A01E0D4ED1C8AB0EE480AFFF706FEB0EE401AB0EE680AFFF700FE31EE400A98
:40AC000010EE105A284625F0A5FA41EC1A0BB0EE4A0AF0EE6A0A21F077FEB0EE409AF0EE609A51EC190B24F059FC606060E18248007818F0F9FF00EE100AB8EE400A5FEDCD
:40AC40007F0A20EE200ADFED7D0A80EE201A84ED0C1AD4ED0C0AB0EE600A0A2104F1180009F08AFB94ED060ADFED750AB4EEE00AF1EE10FA03D20020FFF7BCFD0FE094ED87
:40AC8000060ADFED700AB4EEE00AF1EE10FA03DD0120FFF7AFFD02E00320FFF7ABFD6A48007818F0C1FF00EE100AB8EE400A5FED9B0A20EE200ADFED610A80EE201A84ED20
:40ACC000221AD4ED220AB0EE600A0A2104F1700009F052FB94ED1C0ADFED590AB4EEE00AF1EE10FA03D20020FFF780FD0FE094ED1C0ADFED540AB4EEE00AF1EE10FA03DD85
:40AD00000120FFF773FD02E00320FFF76FFD94ED060AD4ED1C0A30EE600A10EE101A084625F018FA41EC1B0BB0EE4B0AF0EE6B0A21F0EAFDB0EE40AAF0EE60AA51EC1A0B25
:40AD400024F0CCFB09EE100AB0EE490AFFF756FD84ED010ACCE06421E0681BF020F9002869D01BF016F9E06094ED0F0A84ED100A314800781DF0A2F800EE100AB8EEC00AA4
:40AD800084ED0F0A94ED0F0AD4ED100A30EE600A84ED0C0A94ED0C0ADFED2C0A80EE201A84ED0C1A94ED250A84ED260A284800781DF084F800EE100AB8EEC00A84ED250AD3
:40ADC00094ED250AD4ED260A30EE600A84ED220A94ED220ADFED1D0A80EE201A84ED221AD4ED0C0AB0EE600A032104F1180009F0C3FAD4ED220AB0EE600A032104F1700054
:40AE000009F0BAFA94ED060AD4ED1C0AB4EEE00AF1EE10FA04DD94ED060A84ED010A03E094ED1C0A84ED010AEFF758FB90B10020FFF7E0FC22E03CE0D60600200CAC233FE4
:40AE4000CDCCCC3C33339F40D9060020CDCCCC3DDA06002094ED1C0AD4ED060A30EE600AF3EE090AB4EEE00AF1EE10FA03DD0220FFF7C0FC02E00320FFF7BCFCEFF73BFB5F
:40AE800018B10020FFF7B2FC13E094ED060AD4ED1C0A30EE600AF3EE090AB4EEE00AF1EE10FA03DD0220FFF7A1FC02E00320FFF79DFC1DE09FEDFE0A84ED0C0A9FEDFC0AD6
:40AEC00084ED010A0320FFF795FC0320FFF78EFC0EE09FEDF70A84ED0C0A9FEDF50A84ED010A0020FFF786FC0020FFF77FFC00BF00BFBDEC0A8B70BD10B518F0B8FCD0B16C
:40AF0000FAF7FAFEC4B22346FA22EA4900200BF0CBFC9FEDE70AE84880ED060A9FEDE40A80ED060A032180F8381080F890100020E249487242E0E048FFF767FCE048B0F883
:40AF4000BE0118B90220DB49087535E0DA4890F83800032804D1D84890F89000032809D0FAF7CAFEC4B22346FA22D24902200BF09BFC21E0D048D0ED010AD148B0F8BE0167
:40AF800000EE100AB8EE400AF4EEC00AF1EE10FA09DBFAF7B1FEC4B22346FA22C54901200BF082FC08E0FAF7A7FEC4B22346FA22C04900200BF078FCFFF7A3FB10BDBF4963
:40AFC0004872704731B50024BDF80000C82803DDC8200090022406E0BDF80000012802DA01200090032400BF02226946B548006800F5DF70FEF7C4F920B9BDF80000B049C7
:40B00000A1F8BE0100BF204638BD31B50024BDF80000B0F5FA7F04DD4FF4FA700090022406E0BDF80000012802DA01200090032400BF02226946A348006800F5DF70FEF7E7
:40B040009FF920B9BDF800009D49A1F8BE0100BF204638BD31B50024BDF80000322803DD32200090022406E0BDF80000012802DA01200090032400BF022269469148006806
:40B0800000F5DF70FEF77CF920B9BDF800008C49A1F8BE0100BF204638BD31B50024BDF80000C82803DDC8200090022406E0BDF80000012802DA01200090032400BF022285
:40B0C00069468048006800F5DF70FEF759F920B9BDF800007A49A1F8BE0100BF204638BD31B50024BDF8000040F26351884203DD08460090022406E0BDF80000012802DA30
:40B1000001200090032400BF022269466D48006800F5DF70FEF734F920B9BDF800006849A1F8BE0100BF204638BD31B50024BDF8000045F2CC01884203DD08460090022400
:40B1400006E0BDF80000012802DA01200090032400BF022269465B48006800F5DF70FEF70FF920B9BDF800005549A1F8BE0100BF204638BD10B52DED028BB0EE408A0024E3
:40B180004F4890F8BD010B2839D2DFE800F0061B07111C081226381D2F0000BF00BFBCEEC80A10EE101A88B2FFF7BFFF04462FE000BFBCEEC80A10EE101A88B2FFF790FF19
:40B1C000044625E000BF00BFBCEEC80A10EE101A88B2FFF762FF04461AE0BCEEC80A10EE101A88B2FFF736FF044611E0BCEEC80A10EE101A88B2FFF708FF044608E0BCEE0E
:40B20000C80A10EE101A88B2FFF7DCFE044600BF00BF3F20F1F776FF0020FFF7D0FE2046BDEC028B10BD10B52DED020B00BF042269462448006800F5E670FEF7A1F820B933
:40B240009DED000A1E4880ED730A00BF1E48016D0120DFF878C000DF1CBD10B52DED020B00BF042269461748006800F5E470FEF787F820B99DED000A114880ED720A00BFFD
:40B280001148016D0120DFF844C000DF1CBD10B52DED020B00BF042269460A48006800F5E270FEF76DF8A8B99DED000A04480FE000000000E82700202C2700200827002017
:40B2C000081F0020A4030020D03F002089E7030880ED710A00BFFE48016D0120DFF8F4C300DF1CBD10B52DED020B00BF04226946F948006800F5E070FEF742F820B99DEDD4
:40B30000000AF64880ED700A00BFF148016D0120DFF8C0C300DF1CBD10B5F04890F830000A2818D1ED4890F8BD010A2813D19FEDEC0AFFF71FFF9FEDEB0AFFF7D3FF9FED79
:40B34000EA0AFFF7A4FF9FEDE90AFFF786FF9FEDE80AFFF768FFE14890F83000702819D1DE4890F8BD010A2814D19FEDE20AFFF701FF9FEDE10AFFF7B5FF9FEDE00AFFF78A
:40B3800086FF9FEDDF0AFFF768FF9FEDDE0AFFF74AFF18E0D14890F8BD010A2813D19FEDD50AFFF7E7FE9FEDCF0AFFF79BFF9FEDCE0AFFF76CFF9FEDD40AFFF74EFFBBEEC0
:40B3C000040AFFF730FFC54890F8BD01012804D1B7EE000AFFF7CEFE44E0C04890F8BD01022804D19FEDC90AFFF7C4FE3AE0BB4890F8BD01032804D1B3EE040AFFF7BAFE10
:40B4000030E0B64890F8BD01042804D11FED580AFFF7B0FE26E0B14890F8BD01052804D19FEDBB0AFFF7A6FE1CE0AC4890F8BD01062804D19FEDB70AFFF79CFE12E0A7487C
:40B4400090F8BD01072804D1B1EE040AFFF792FE08E0A24890F8BD01092803D19FEDAD0AFFF788FE10BD10B59C4890F8BD010A280DD19A4890F830000A2803D1FA20FFF7F7
:40B48000C4FD03E04FF49670FFF7BFFD00E000BF00BF10BD00B589B018F0D6F9002878D08E4890F8BD010C2874D2DFE800F07306292A4D74759873FEFDEB0020009001900C
:40B4C000029003460246944903900846007818F0BCFA0020009001900290034602468F4903900846007818F0B0FA01218A48007818F059FE01218948007818F054FE6DE110
:40B5000000BF002000900190029003460322824903900846007818F098FA0020009001900290034603227D4903900846007818F08CFA03217848007818F035FE03217748E5
:40B54000007818F030FE49E101200021009101910B460A46CDE902106F490846007818F074FA01200021009101910B460A46CDE902106A490846007818F067FA01216648B1
:40B58000007818F010FE01216448007818F00BFE24E124E1FDE000BF0020009001900290034603225C4903900846007818F04DFA00200090019002900346032257490390FE
:40B5C0000846007818F041FA00215348007818F0EAFD00215148007818F0E5FDFEE00020009001900290034602224B4903900846007818F02AFA00200090019002900346B0
:40B600000322464903900846007818F01EFA002000900190029003460222414903900846007818F012FA02213B48007818F0BBFD02213B48007818F0B6FD002000900190AE
:40B64000034614220121029004A81CF053FA04A85FEDE90A9FED330A02230022324900902D4800781CF02EF904A85FEDEF0A9FED2D0A022303222D490090294800781CF073
:40B6800021F9ABE0002000900190029003460222214903900846007818F0D7F90020009001900290034601E075E073E003221B4903900846007818F0C8F900200090019079
:40B6C00002900346022216490390084600782FE0D03F002089E70308A4030020081F002000007A43C6DCB53DB8AF833E52B8444114AE4740000096436744293EE5F25F3E1C
:40B7000052B862416666E6C133331B41000016430080BB440000C842D6060020D9060020DA06002000504347000400400000014018F08BF90621FA48007818F034FD06211E
:40B74000F848007818F02FFD002000900190034614220121029004A81CF0CCF904A8DFEDF20A1FED100A02230022F0490090EC4800781CF0A7F804A8DFEDEB0A1FED170A51
:40B7800002230322EA490090E64800781CF09AF824E000BF00BF002000900190029003460322DF4903900846007818F04EF9002000900190029003460322DE49039008465C
:40B7C000007818F042F90121D548007818F0EBFC0121D848007818F0E6FC00BF00BFD64890F8BD01D54908700020FFF7E8FB0020D349087209B000BDD249097D012900D10B
:40B8000000E0002108467047CE48407D7047CD48007D08B9012070470020FCE7CA4909880143C94A11807047F7EE000AB0EE600A7C220270C04A92F8BD210B2A1DD2DFE8A3
:40B8400002F00611070812090A161C13190000BF00BF00BF00BF01224270DFEDBC0AB0EE600A0BE000BF00BF0222427006E00422427003E00522427000E000BF00BFAF4AB2
:40B88000D2ED060A60EE800AFCEEE00A10EE902A91B281700A0AC270A84AD2ED1C0A60EE800AFCEEE00A10EE902A91B201710A0A4271A14AB2F8BE1181710A0AC2717047D0
:40B8C0009E4890ED010A704701B500BF012269469F48006800F2BD10FDF752FD20B99DF80000954981F8BD0100BFFFF715FD012000F07EFC1D20F1F705FC08BD01B500BF56
:40B90000022269469248006800F5E870FDF738FD20B9BDF800008849A1F8D00100BF08BD0020854991F8BD110B2916D2DFE801F0160C09060D0A070F1117130000BF01209D
:40B940000EE000BF01200BE000BF012008E0012006E0012004E0012002E000BF00BF00BF00BF70470020744991F8BD110B2919D2DFE801F0190E0A060F0B0711131A1500CE
:40B9800000BF40F2635010E000BF45F2CC000CE000BFC82009E0322007E0C82005E04FF4FA7002E000BF00BF00BF00BF70470020624991F8381009B9142012E05F4991F8B8
:40B9C0003810012901D116200BE05C4991F8901009B9152005E0594991F89010012900D11720704770B504245A4880780A2876D2DFE800F0051376E1E1E1E1DBDDDF0020A3
:40BA000054490870C8808860FFF778FF514880785049487001208870CEE0FFF7C8FF4D4908700846007810B10720887056E04948806820B91AF0ADFA464988604EE04549CE
:40BA400088684FF47A711AF0AAFA002846D0FFF737FFBCEEC00A10EE100A85B22846FFF74DFF3548B0F8AC0068B13348B0F8AC003149B1F8D011884205DD2F48B0F8AC00E9
:40BA80003449C88021E02C48B0F8D001002803DC01203049C88018E0274890F8BD01032804D0254890F8BD01062805D12248B0F8D00100F5FA7006E01F48B0F8D0018000FF
:40BAC000032190FBF1F02349C8800220214988701AF05FFA1F498860002008736CE06AE0FFF7EEFE1B48C08800EE900AF8EE600AB4EEE00AF1EE10FA05DB1648007B401CAB
:40BB00001449087302E0002012490873FFF74FFF1049087008460078F0B10720887043E0D6060020DA060020000000000004004000000140D9060020081F00202C2700205D
:40BB400008270020E8270020B0030020C0A90646A4030020002800206848007B04280DDB6648C08800EE900AF8EE600AB0EE600AFFF700FB09206149887015E05F49886852
:40BB800041F288311AF00BFA70B15C48C08800EE900AF8EE600AB0EE600AFFF7EBFA0720564988701820087006E0012404E0022402E0032400E000BF00BF5048007818B1FF
:40BBC0004E490878F8F778FE204670BD4B48807870474A4800787047002048498870C870704701B500BF0222694645480068AC30FDF7C6FB20B9BDF800004249A1F8AC006F
:40BC000000BF08BD10B52DED028B3E4890F8BD0103280ED03B4890F8BD01062809D0394890F8BD01022804D0364890F8BD0105280CD113F004FB10B1012806D102E0B7EE92
:40BC4000008A02E09FED308A00BF01E0B7EE008AB0EE480ABDEC028B10BDB7EE000AF0EE400A284890F8BD010B2815D2DFE800F0060F070810090A121411130000BF00BFE3
:40BC800000BF00BF1FED4F0AF0EE400A05E000BF00BF00BF00BF00E000BF00BF1B4890ED060A20EE200A7047B7EE000AF0EE400A144890F8BD010B2815D2DFE800F0060FFC
:40BCC000070810090A121411130000BF00BF00BF00BF1FED620AF0EE400A05E000BF00BF00BF00BF00E000BF00BF084890ED1C0A20EE200A70470648407A70470028002004
:40BD0000A4030020081F0020D7A3DC402C2700200827002010B517F0AAFD18B1FB4890F8860348B9F9F7E8FFC4B22346FA22F84903200AF0B9FD17E0F648007818F0B0F9C8
:40BD400048B1F9F7D9FFC4B22346FA22F04901200AF0AAFD08E0F9F7CFFFC4B22346FA22EB4900200AF0A0FD10BD10B517F07FFD48B9F9F7C1FFC4B22346FA22E64903206D
:40BD80000AF092FD17E0E548007818F089F948B1F9F7B2FFC4B22346FA22DF4901200AF083FD08E0F9F7A8FFC4B223464122DA4900200AF079FD10BDD948007D704710B521
:40BDC000D8480AF0D5FD17F052FD48B1F9F794FFC4B223464122D24903200AF065FD1BE0D148007818F05CF918B9CE48407A012809D1F9F781FFC4B223464122C849012038
:40BE00000AF052FD08E0F9F777FFC4B223464122C34900200AF048FDC4484078002866D0C348007800F0010070B9FFF7C5FF012800D100E000204000BD49087008460078C7
:40BE400040F0010008703EE0B9480078C0F34000D0B1FFF7B1FF012806D0B548007840F00800B34908702EE0FFF7A6FF01282AD1AF48007800F0080028B3AD48007840F09C
:40BE80000400AB4908701EE0A9480078C0F34000C8B9FFF791FF012806D1A548007840F00400A34908700EE0FFF786FF01280AD09F48007800F0040028B19D48007840F08F
:40BEC00008009B4908709A48007800F0040070B19748007800F0080048B10020944908709448D0F818111020DFF84CC200DF10BD10B5032417F0A8FC40B19048007818F044
:40BF0000CFF808B101243EE000243CE017F084FC002838D08A48007818F0C2F8002832D08848007818F0BCF840B18448007818F0B7F808B1012426E0002424E082480078D3
:40BF400018F0AEF830B17D48007818F0A9F808B1012418E07C48007818F0A2F830B97748007818F09DF808B901240CE07648007818F096F830B17148007818F091F808B9D9
:40BF8000002400E00124204610BD70B5044617F06EFC48B1F9F7B0FEC5B22B46FA226B4901200AF081FC59E06078022824D1FFF79FFF012809D1F9F79FFEC5B22B46FA2206
:40BFC000624901200AF070FC48E0FFF791FF48B9F9F792FEC5B22B46FA225C4900200AF063FC3BE0F9F788FEC5B22B46FA22574903200AF059FC31E06078012817D1FFF727
:40C0000077FF012809D1F9F777FEC5B22B46FA224E4901200AF048FC20E0F9F76DFEC5B22B46FA22494900200AF03EFC16E0607803280AD1F9F760FEC5B24549487A2B4689
:40C04000FA2242490AF030FC08E0F9F755FEC5B22B46FA223D4903200AF026FC70BD01B500BF042269463B4800689830FDF788F918B926490098C1F8980000BF08BD10B5EE
:40C080002DED028B17F0C8FB40B13348007818F007F808B1012463E0002461E017F0E7FB08B103245CE02C48007803F075FAB0EE408A1648B0F8800300EE100AB8EE400A62
:40C0C000B4EEC80AF1EE10FA0DD81048B0F8820300EE100AB8EE400AB4EEC80AF1EE10FA01DB01243BE00948B0F8800300EE100AB8EE400AB4EEC80AF1EE10FA2EDD0348E1
:40C1000090F8BC01022829D1032428E0081F002058280020A406002070280020A90600201028002088280020A806002000FF0020BC030020D03F002089E70308A1060020CA
:40C14000A0060020AC060020D106002040280020A0280020A4030020A5060020002400BF2046BDEC028B10BD70B50446A078022802D0A07801280CD1F9F7BEFDC5B2FFF729
:40C180007EFF06462B464FF41672F8490AF08CFB18E0A07803280BD1F9F7AEFDC5B2F449487A2B464FF41672F0490AF07DFB09E0F9F7A2FDC5B22B464FF41672EB49032027
:40C1C0000AF072FBE948007D58B9EA48007840B1E949D1F8B400FFF742FF0020E549087005E0E248007D012801D1E249087070BD10B50446E148D0F82C112046DFF880C3BE
:40C2000000DF10BD01B500BF02226946DD48006800F28230FDF7B4F820B9BDF80000D649A1F8820300BF3320F0F76CFF08BD01B500BF02226946D348006800F56070FDF7C1
:40C240009FF820B9BDF80000CB49A1F8800300BF3220F0F757FF08BD13B50C4640F6C410FFF7E5FF4FF47A50FFF7CCFF00BF01226946C448006800F5DE70FDF781F820B9FC
:40C280009DF80000BC4981F8BC0100BF14B10120FFF7AEFF2D20F0F735FF1CBD10B50446B948007820B1B44890F8BC01A07005E00020A070A0780021FFF7CEFF0120607079
:40C2C0002070FFF7E7F82D20F0F71CFF10BD08B50321AA4880F83011DFF8B0C200DF064631460120DFF898C200DF17F095FA20B10121A748007817F0D1FA00BF002214213D
:40C300000120DFF890C200DF85B2012D0AD0DFF888C200DF044604F0010088B16846FFF7BDFF0DE0FEF7E8FD6846FFF71DFF6846FFF72BFEFFF743FDFFF717FDFFF7EAFC4D
:40C340002B20F0F7DFFE2C20F0F7DCFE2A20F0F7D9FE4720F0F7D6FED0E79048007D70478F48007D70478F48407D70478E48407D70477E48407D704710B517F04DFA08B10E
:40C38000022405E017F060FA08B1012400E00024204610BD10B517F03FFA10B917F054FA08B1012400E00024204610BD7047704710B5029C10BD2DE9F04105460C461746E5
:40C3C0009846069EB5F56F4F0DD12078B1280AD16078362807D1A078012804D18222012172480AF0B8FA4FF6467085420FD1207868B96078042805D1822201216B480AF031
:40C40000AAFA04E00022114668480AF0A4FABDE8F0812DE9F04104460D4617469846069E4FF6B07084420FD1A87800F01000102805D1822201215D480AF08DFA04E00022AF
:40C4400011465A480AF087FABDE8F0812DE9F04106460C4617469846069D607800F00300534908706078032101EAA000504948706078032101EA20104D4988706078032117
:40C4800001EAA0104A49C870A078888008468088E1784FF47F4202EA0121084344498880207900F0030088712079032101EAA0003F49C8712079032101EA20103C490872F0
:40C4C000A0794872E079887208464178002237480AF041FA3648C179002225480AF03BFABDE8F0812DE9F84305460E4617469846089C214991F83000FAF7A9FC38B14346B3
:40C500003A46314628460094FFF7A0FF1AE01A4991F83000FAF7A3FC38B143463A46314628460094FFF775FF0CE0134991F83000FAF76BFC30B143463A4631462846009436
:40C54000FFF739FFBDE8F88310B51A48007817F0A7FDA8BB1848007817F0A2FD80BB1748007817F09DFD58BB01202BE02828002094280020B4030020081F0020D03F0020B7
:40C5800089E70308A4030020A2030020C9F30308BD060020E9E7030831E703085828002070280020402800201028002088280020AC280020F2060020F9060020E306002090
:40C5C000FFE700200446204610BD10B52448D0F8B4002349D1F89810401AB0F5B46F08D91F4890F8BC0120B1F9F786FB08B9012010BD0020FCE710B501241A48007D58B9B1
:40C6000041F658311848006819F0C9FC10B9F9F773FB68B900240BE0FFF7D7FF20B1F9F76BFB08B9002403E019F0B3FC0E490860204610BD01B500BF012269460B480068E6
:40C6400000F28630FCF79CFE20B99DF80000044981F8860300BF3120F0F754FD08BD0000081F002028280020B8030020A4030020B5EEC00AF1EE10FA04DDF4EEE10AF1EE7F
:40C6800010FA09DAB5EEC00AF1EE10FA06D2F4EEC10AF1EE10FA01D8012070470020FCE7FD480078704710B52DED028B0446B0EE408AB7EE000AF0EE408AFFF7F1FF80B313
:40C6C000F8F726FE68BBF2EE0A0AB4EEE08AF1EE10FA03DBDFEDF10AB0EE608AFDEEC80A10EE901A08B200EE900AF8EEE00A38EE600A04F1140101EB8001D1ED000AB7EE03
:40C70000001A31EE401A60EE810A04F11401421C01EB820191ED001A41EE000AF0EE608A00BFB0EE680ABDEC028B10BD70B52DED028B04460D46B7EE000AB0EE408AF8F7DC
:40C74000E7FD40B9D64800EBC40000EB850090ED000AB0EE408AB0EE480ABDEC028B70BDD0ED000A91ED001A60EE810A90ED011AD1ED011A41EE210A90ED021AD1ED021AE7
:40C7800041EE210A90ED031A60EE810AB0EE600A704710B52DED068B04469FEDC20AF0EE409A94F8C200012804D194ED210A84ED220A87E004F1900104F14C00FFF7D0FF9B
:40C7C000B0EE408AB64A4C3A92F8421092F84100FFF7ACFF20EE080AB0EE408A10F07CFDB0EE40AA2046FFF75EFF20EE080AB0EE408AB5EEC08AF1EE10FA06DD94ED1B0ADA
:40C8000020EE080AB0EE408A05E094ED170A20EE080AB0EE408A94F87C0001283AD194ED220A30EE080A84ED220A94ED220AD4ED180AB4EEE00AF1EE10FA43DD94ED220AD9
:40C84000D4ED1C0AB4EEE00AF1EE10FA3AD2B5EEC08AF1EE10FA0ED294ED220AD4ED1C0A30EE600AB0EE408A94ED180A30EE080AB0EE408A26E094ED220AD4ED180A30EE27
:40C88000600AB0EE408A94ED1C0A30EE080AB0EE408A17E084ED228AB5EEC08AF1EE10FA08DD94ED220AD4ED1C0A30EE200A84ED220A07E094ED220AD4ED180A30EE200A60
:40C8C00084ED220A94ED220AD4ED1D0AB4EEE00AF1EE10FA04DD94ED1D0A84ED220A0CE094ED220AD4ED190AB4EEE00AF1EE10FA03D294ED190A84ED220AA06819F071FBE6
:40C9000000EE100AB8EE409A94ED030A60EE098A94ED220AD4ED1C0AB4EEE00AF1EE10FA08DB94ED230AD4ED1C0AB4EEE00AF1EE10FA11D394ED220AD4ED180AB4EEE00A0A
:40C94000F1EE10FA14D894ED230AD4ED180AB4EEE00AF1EE10FA0BDD94ED180AB0EEC00AD4ED1C0A30EE200A30EE280AF0EE408A94ED220AD4ED230A30EE600AB4EEE80A0B
:40C98000F1EE10FA06DD94ED230A30EE280A84ED220A12E094ED220AD4ED230A30EE600AF1EE680AB4EEE00AF1EE10FA05D294ED230A30EE680A84ED220A19F0EAFAA06096
:40C9C00094ED220A84ED230A35484C3890F830000A2806D1FAF731FB18B1B7EE000AF0EE409AF9F7FBF9B8B1F5EEC09AF1EE10FA1ED094ED1E2AF0EE421A94ED1A2AB0EE16
:40CA0000421A94ED202AF0EE420A94ED232AB0EE420AFFF72DFE58B1F8F77CFD102807D09FED200A84ED220A9FED1E0A84ED230A0120BDEC068B10BD70B52DED088B054662
:40CA40000C46B0EE408A94ED010AD4ED000A30EE600A84ED040A18EE100A23F07BFB41EC190B94ED040A10EE101A084623F072FB41EC1B0BB0EE4B0AF0EE6B0A1FF044FF34
:40CA8000B0EE40AAF0EE60AA53EC192B51EC1A0B23F02EF80CD207E0D80300200AD74F41541F0020000000001FED020A84ED040A94ED040AD5ED040A30EE600A84ED060A25
:40CAC00094ED070A10EE101A084623F043FB41EC190B94ED060A10EE101A084623F03AFB41EC1B0BB0EE4B0AF0EE6B0A1FF00CFFB0EE40AAF0EE60AA53EC192B51EC1A0B35
:40CB000023F030F904D21FED190A84ED050A12E0F9F764F978B194ED040AD5ED040A30EE200AF0EE000AC0EE208A94ED050A30EE280A84ED050ABDEC088B70BDFD4A92F84B
:40CB4000281092F83020702A38D19FEDFB0A80ED030A9FEDFA0A80ED040A9FEDF90A80ED050A9FEDF80A80ED060A9FEDF70A80ED070A9FEDF60A80ED080A9FEDF50A80EDC6
:40CB8000090A9FEDF40A80ED0A0A9FEDF30A80ED0B0A9FEDF20A80ED0C0A9FEDF10A80ED0D0A9FEDF00A80ED0E0A9FEDEF0A80ED0F0AB7EE000A80ED100A0AE3DD4A92F84C
:40CBC00030200A2A38D19FEDDF0A80ED030A9FEDE70A80ED040A9FEDE60A80ED050AB6EE080A80ED060A9FEDDC0A80ED070A9FEDE10A80ED080A9FEDE00A80ED090A9FED2E
:40CC0000DF0A80ED0A0AB7EE000A80ED0B0A9FEDDC0A80ED0C0A9FEDDB0A80ED0D0A9FEDDA0A80ED0E0A9FEDD90A80ED0F0AB7EE040A80ED100ACCE2BE4A92F84A20032A74
:40CC40007CD10E297CD2DFE801F07B077C7B407F80817B7B7B7B7E7D9FEDBA0A80ED030A9FEDC20A80ED040A9FEDC10A80ED050AB6EE080A80ED060A9FEDB70A80ED070A9C
:40CC80009FEDBC0A80ED080A9FEDBB0A80ED090A9FEDBA0A80ED0A0AB7EE000A80ED0B0A9FEDB70A80ED0C0A9FEDB60A80ED0D0A9FEDB50A80ED0E0A9FEDB40A80ED0F0A90
:40CCC000B7EE040A80ED100A79E09FEDB10A80ED030A9FEDB00A80ED040A9FEDAF0A80ED050A9FEDAE0A80ED060A9FEDAD0A80ED070A9FEDAC0A80ED080A9FEDAB0A80ED6D
:40CD0000090A9FEDAA0A80ED0A0A9FEDA90A80ED0B0A9FEDA80A80ED0C0A9FEDA70A80ED0D0A9FEDA60A80ED0E0A9FEDA50A80ED0F0A9FEDA40A80ED100A40E040E0FFE773
:40CD400000BF00BF00BF00BF00BF00BFB7EE000A80ED030AB7EE000A80ED040AB7EE000A80ED050AB7EE000A80ED060AB7EE000A80ED070AB7EE000A80ED080AB7EE000A85
:40CD800080ED090AB7EE000A80ED0A0AB7EE000A80ED0B0AB7EE000A80ED0C0AB7EE000A80ED0D0AB7EE000A80ED0E0AB7EE000A80ED0F0AB7EE000A80ED100A00BF08E2E5
:40CDC0000E297AD2DFE801F079077A40B4B3B2B179797979B0AFB6EE000A80ED030A9FED660A80ED040AB7EE040A80ED050A9FED760A80ED060AB0EE000A80ED070AB0EE96
:40CE0000020A80ED080A9FED710A80ED090A9FED700A80ED0A0A9FED6F0A80ED0B0A9FED6D0A80ED0C0A9FED6B0A80ED0D0A9FED690A80ED0E0A9FED670A80ED0F0A9FED34
:40CE4000650A80ED100AC3E19FED630A80ED030A9FED620A80ED040A9FED610A80ED050A9FED600A80ED060A9FED5F0A80ED070A9FED390A80ED080A9FED5C0A80ED090A19
:40CE80009FED400A80ED0A0AB7EE040A80ED0B0A9FED570A80ED0C0AB7EE080A80ED0D0A9FED490A80ED0E0A9FED520A80ED0F0AB0EE000A80ED100A8AE14DE19FED480AC3
:40CEC00080ED030A9FED460A80ED040A9FED440A80ED050A9FED430A80ED060A9FED420A80ED070A9FED1C0A80ED080A9FED3F0A80ED090A9FED230A80ED0A0AB7EE040AEC
:40CF000080ED0B0A9FED3A0A80ED0C0AB7EE080A80ED0D0A9FED2C0A80ED0E0A9FED2A0A80ED0F0A68E06CE0A4E018E116E114E1D9E00000081F00208FC2F53EB81E053FB9
:40CF4000295C0F3F9A99193F0AD7233F7B142E3FEC51383F5C8F423FCDCC4C3F3D0A573FAE47613F1F856B3F8FC2753F6666263F3333333F9A99593F6666663F3333733FAE
:40CF80006666863FCDCC8C3F3333933F9A99993FA69B443D6F12833D6F12033EF4FD543E6F12833E96438B3EBC74933EE3A59B3E0AD7A33E3108AC3E5839B43E7F6ABC3E60
:40CFC000A69BC43ECDCCCC3E3333D33FCDCC1C400AD7234066662640CDCCCC3DCDCC4C3E9A99993E7B14EE3EAE47213F48E17A3F3333B33F6666E63F1FED0D0A80ED100AB4
:40D00000E6E01FED2B0A80ED030A1FED2D0A80ED040A1FED2F0A80ED050A9FEDFE0A80ED060A1FED330A80ED070A1FED350A80ED080A1FED370A80ED090A1FED310A80EDCD
:40D040000A0AB7EE000A80ED0B0A1FED320A80ED0C0A1FED330A80ED0D0A1FED340A80ED0E0A1FED360A80ED0F0A1FED380A80ED100AADE01FED4D0A80ED030A9FEDE60A77
:40D0800080ED040A9FEDE50A80ED050A9FEDE40A80ED060A9FEDE30A80ED070A9FEDE20A80ED080A9FEDE10A80ED090A9FEDE00A80ED0A0A9FEDDF0A80ED0B0A9FEDDE0AC0
:40D0C00080ED0C0A9FEDDD0A80ED0D0A9FEDDC0A80ED0E0A9FEDDB0A80ED0F0A9FEDDA0A80ED100A74E09FEDD90A80ED030A1FED6E0A80ED040A9FEDD60A80ED050A1FEDA1
:40D10000620A80ED060A1FED610A80ED070AB7EE040A80ED080A9FEDCF0A80ED090A9FEDCD0A80ED0A0A9FEDCB0A80ED0B0A9FEDC90A80ED0C0A9FEDC70A80ED0D0A9FEDE4
:40D14000C50A80ED0E0A9FEDC30A80ED0F0A9FEDC10A80ED100A3BE000BF00BF00BFB7EE000A80ED030AB7EE000A80ED040AB7EE000A80ED050AB7EE000A80ED060AB7EEF7
:40D18000000A80ED070AB7EE000A80ED080AB7EE000A80ED090AB7EE000A80ED0A0AB7EE000A80ED0B0AB7EE000A80ED0C0AB7EE000A80ED0D0AB7EE000A80ED0E0AB7EEEB
:40D1C000000A80ED0F0AB7EE000A80ED100A00BF00BF7047A0490870704710B504469F4890F842106830405C00EE100AB8EE400ADFED9B0A80EE201A84ED151A974890F800
:40D2000042106C3000EB810090ED000A84ED160A924890F842107C3000EB810090ED000A84ED170AF9F7FBFE20B19FED8E0A84ED180A07E006F0A8F85FEDB20A20EE200A69
:40D2400084ED180A854890F842106A30405C00EE100AB8EE400ADFED820A80EE201A84ED191A7E4890F84210743000EB810090ED000A84ED1A0A794890F84210843000EB9C
:40D28000810090ED000A84ED1B0AF9F7C8FE20B19FED730A84ED1C0A07E006F0B3F85FEDCB0A20EE200A84ED1C0A6C4890F841105C3000EB4100694991F84210405C00EED5
:40D2C000100AB8EE400ADFED660A80EE201A84ED111A624890F84110603000EB41005F4991F84210405C00EE100AB8EE400ADFED5C0A80EE201A84ED121A584890F841105E
:40D30000643000EB4100554991F84210405C00EE100AB8EE400ADFED520A80EE201A84ED131AF9F754FE50B14C4890F830000A2800D004E09FED4C0A84ED140A0EE0F9F7EE
:40D340006EFE38B116F093FA20B1B1EE040A84ED140A03E09FED450A84ED140A3F4890ED7E0A84ED010A9FED420A84ED020A0120FFF730FF394890F82800072806D116F08B
:40D3800063FA18B1012084F8740002E0002084F874002046FFF7D2FB0A20EFF7B3FE0B20EFF7B0FE0C20EFF7ADFE0E20EFF7AAFE0D20EFF7A7FE1120EFF7A4FE1020EFF79B
:40D3C000A1FE012010BD2DED028B302629482A490860001D29490860001D294908600C3828490860343028490860401C27490860B93827490860FFF7F0FE184890F828001E
:40D400001C4990390870154890ED0F0A084680ED010A3FE07B144E3F3789213F4C37293FE926313F8716393F2506413F39B4483FD7A3503F7593583F8941603F2731683F84
:40D44000C520703FD9CE773F77BE7F3F3333B33ED7A3303F6666A63FD8030020081F00200000C8420000C8C20000FA4300C05A4500000000B4290020C0030020C40300209E
:40D48000C8030020CC030020D0030020D4030020DC0300209FEDFE0A80ED270A90ED1E0AFC4880ED190A084690ED1A0AF94880ED1A0ADFF8E4C300DFDFF8E0C300DF8046C1
:40D4C0003022012118F06FFEDFF8D0C300DF8046012118F097FE0321F14880F8401000BF002231464CF20300DFF8B8C300DF0446012C17D100BFEA4890F8410040F001013B
:40D50000E74880F84110B0F84C004FF6FF71884207DAE348B0F84C00401C81B2E048A0F84C10DDE7022CDBD1DFF87CC300DF054605F0020030B3DD48FFF74FFEDC4890F809
:40D540002800DA4908390870D94890ED0F0A084680ED010A1021CF48DFF858C300DF012810D0D248083890ED1E0ACA4880ED190ACE48083890ED1A0AC64880ED1A0ADFF8FA
:40D5800038C300DF05F001000028A9D01021C148DFF820C300DF01287DD02022C349783101F120001DF0F3FF18F0F3FC0746BF48083890F8C00006286ED2DFE800F0037F2F
:40D5C0008596ADC2B34890F84100012812D1B148816B384618F014FDFA280BD20320B349083981F8C000012081F8C100002081F8C20062E003F054FBD0B1F8F77DFBB8B132
:40D60000A44890F85900012812D1A248016D384618F0F6FCFA280BD20520A449083981F8C000012081F8C100002081F8C20044E003F036FBC8B1F8F75FFBB0B1954890F830
:40D640004D00012811D19348416C384618F0D8FCFA280AD204209549083981F8C000012081F8C10081F8C20027E003F019FBE8B1F8F742FBD0B1874890F83500012815D171
:40D680008448C16A384618F0BBFCFA280ED202208649083901E08CE064E081F8C000012081F8C100002081F8C20006E000207F49083981F8C10081F8C20059E000207B49E1
:40D6C000083981F8C00053E0F8F716FB28B101207649083981F8C10006E000207349083981F8C10081F8C00042E06A4890F8410030B16848816B384618F082FCFA2805D9B5
:40D7000000206A49083981F8C00004E001206749083981F8C1002BE0F8F7EEFA38B101206249083981F8C10081F8C20008E000205E49083981F8C10081F8C20081F8C00081
:40D7400016E0F8F7D9FA28B101205849083981F8C10006E000205549083981F8C10081F8C00005E000205149083981F8C10000BF00BF4E48083890F8C10080B14B480838C8
:40D7800090F8C00000EB40014248143000EB810090ED010A4548083880ED210A05E01FEDCC0A4248083880ED210A3A48DFF808C100DF3E48083890F8C10001287ED1F9F72D
:40D7C00006FC38B305F0BBFD324880ED040A37490839087891ED011AF0EE410A2D4991ED041AB0EE410A05F0C1FC3048083880ED200A0146087891ED011AF0EE410A91ED94
:40D80000211AB0EE410A05F0B1FC2848083880ED210A34E0F9F703FC30B1F8F772F82348083880ED200A2AE0F9F7F0FB38B305F086FD184880ED040A0FF04AFDB0EE408A8A
:40D840001448D0ED040AB0EE600AF0EE480A05F04BFD1648083880ED200A0FF039FDB0EE408A12480838D0ED210AB0EE600AF0EE480A05F039FD0D48083880ED210A0B48D5
:40D880000838D0ED040AB0EE600A00F1800116E099A0063CB82800205DEB0308C9F30308D03F0020E9E7030831E703082C290020081F002051EC03086DEB030816E0A030FE
:40D8C000FFF7BAF8FE48FEF764FF50B1FC4890ED230AFC4880ED170A0120FA4981F860000DE00020F74981F8600008E09FEDF60AF44880ED170A0020F24981F860003E20EE
:40D90000EFF700FC4F20EFF7FDFBE9E510B5EF48C16B012018F0B0FCEC48C16B0120DFF8B0C300DF10BD10B5E848C16B012018F0C1FC0446204610BD70B52DED028BB0EE88
:40D94000408A04460D460026012C04D0022C03D0032C61D101E000BF00BFDA4890ED1A0AB4EEC80AF1EE10FA05DD90ED1A0AB0EE408A03260CE0D34890ED190AB4EEC80A09
:40D98000F1EE10FA04D290ED190AB0EE408A02261021CC48DFF83CC300DF01283AD004EB4401C848143000EB810080ED018A15F05EFF98B104EB4401C248143000EB8100C6
:40D9C00090ED010AFFEE000A20EE200A04EB4401BC48143000EB810080ED010A18F0D9FA04EB4402B749143141F82200012104EB4402B448143000EB8200017204EB4401B5
:40DA0000B048143000EB81004572AE48DFF8C8C200DF00E0062601E0062600BF00BF3046BDEC028B70BD70B52DED028BB0EE408A04460D460026012C04D0032C03D0042CB7
:40DA400047D100BF00BF9FEDA50AB4EEC08AF1EE10FA05D29FEDA10AB0EE408A03260BE09FED9F0AB4EEC08AF1EE10FA04DD9FED9C0AB0EE408A022610219248DFF854C2D1
:40DA800000DF012823D004EB44018E48143000EB810080ED018A18F07CFA04EB44028949143141F82200012104EB44028548143000EB8200017204EB44018248143000EB1F
:40DAC000810045727F48DFF810C200DF00E0062601E0062600BF00BF3046BDEC028B70BD70B52DED028BB0EE408A04460D460026012C04D0032C03D0052C47D100BF00BF6E
:40DB00009FED760AB4EEC08AF1EE10FA05D29FED730AB0EE408A03260BE09FED710AB4EEC08AF1EE10FA04DD9FED6D0AB0EE408A022610216348DFF89CC100DF012823D04D
:40DB400004EB44015F48143000EB810080ED018A18F01FFA04EB44025A49143141F82200012104EB44025748143000EB8200017204EB44015348143000EB810045725148A0
:40DB8000DFF854C100DF00E0062601E0062600BF00BF3046BDEC028B70BD4A4890ED170A7047484890F860007047454890ED210A7047434890ED200A704773B52DED020BF0
:40DBC00004460D4600269DED000ADFED460AB4EEE00AF1EE10FA05DD02269FED420A8DED000A0DE09DED000ADFED3F0AB4EEE00AF1EE10FA04D203269FED3B0A8DED000A78
:40DC000000BF3A4909684C3101EBC40101EB850004226946FBF7B4FB40B99DED000A344800EBC40000EB850080ED000A00BF30484C3890F84200A8420BD12D484C3890F8B1
:40DC40004100A04205D12148C16B0220DFF880C000DF1620EFF756FA304604B070BDF7B50C46154600269DF80000FF2803DD0226FF20009006E09DF80000012802DC03269E
:40DC80000120009000BF194909685C3101EB4401481901226946FBF773FB30B99DF800101348103000EB4400415500BF10484C3890F84200A84227D10D484C381AE00000C8
:40DCC00024290020B828002000000000D03F002089E7030851EC03086DEB03080000C8C20000C842333323400AD7233CA4030020541F002090F84100A04205D1FE48C16B78
:40DD00000220DFF8F8C300DF0A20EFF7FBF93046FEBDF7B50C46154600269DF80000FF2803DD0226FF20009006E09DF80000002802DC03260020009000BFF14909686031D4
:40DD400001EB4401481901226946FBF719FB28B99DF80010EB4800EB4400415500BFE948603890F84200A8420BD1E648603890F84100A04205D1E048C16B0220DFF87CC3D0
:40DD800000DF0B20EFF7BEF93046FEBDF7B50C46154600269DF80000FF2803DD0226FF20009006E09DF80000002802DC03260020009000BFD2490968643101EB44014819CD
:40DDC00001226946FBF7DCFA30B99DF80010CD48001D00EB4400415500BFCA48603890F84200A8420BD1C748603890F84100A04205D1C148C16B0220DFF800C300DF0C20E7
:40DE0000EFF780F93046FEBD73B50C4600259DF80000FF2803DD0225FF20009006E09DF80000012802DA03250120009000BFB44909686831081901226946FBF7A1FA20B9C9
:40DE40009DF80010AF480830015500BFAD48603890F84200A04205D1A748C16B0220DFF89CC200DF0F20EFF74DF928467CBD73B50C4600259DF80000FF2803DD0225FF20D6
:40DE8000009006E09DF80000012802DA03250120009000BF9A4909686A31081901226946FBF76EFA20B99DF8001096480A30015500BF9448603890F84200A04205D18E4807
:40DEC000C16B0220DFF834C200DF1220EFF71AF928467CBD31B52DED020B044600258948603890F842107C3000EB810090ED000ADDED000AB4EEE00AF1EE10FA0CDD8148FD
:40DF0000603890F842107C3000EB810090ED000A8DED000A02250DE09DED000ADFED7A0AB4EEE00AF1EE10FA04DD9FED770A8DED000A032500BF724909686C3101EB84004D
:40DF400004226946FBF71CFA38B99DED000A6D480C3000EB840080ED000A00BF6948603890F84200A0420BD16348C16B0220DFF88CC100DF6048016D0120DFF880C100DFAE
:40DF80004D20EFF7BFF80E20EFF7BCF828463EBD31B52DED020B044600259DED000AB5EEC00AF1EE10FA05D21FEDB90A8DED000A03251BE05348603890F84210843000EBC7
:40DFC000810090ED000ADDED000AB4EEE00AF1EE10FA0BD24B48603890F84210843000EB810090ED000A8DED000A022500BF44490968743101EB840004226946FBF7C0F94A
:40E0000038B99DED000A3F48143000EB840080ED000A00BF3B48603890F84200A0420BD13548C16B0220DFF8D4C000DF3248016D0120DFF8C8C000DF4D20EFF763F811200D
:40E04000EFF760F828463EBD31B52DED020B044600259DED000A5FEDDF0AB4EEE00AF1EE10FA05D21FEDE30A8DED000A02251BE02448603890F842106C3000EB810090ED66
:40E08000000ADDED000AB4EEE00AF1EE10FA0BD21C48603890F842106C3000EB810090ED000A8DED000A032500BF154909687C3101EB840004226946FBF762F938B99DEDD7
:40E0C000000A10481C3000EB840080ED000A00BF0C48603890F84200A0420BD10648C16B0220DFF818C000DF0348016D0120DFF80CC000DF4D2009E0D03F002089E70308D3
:40E10000A4030020681F002000000080EEF7FAFF0D20EEF7F7FF28463EBD31B52DED020B044600259DED000ADFEDF90AB4EEE00AF1EE10FA05DD9FEDF60A8DED000A022535
:40E1400019E0F44890F84210743000EB810090ED000ADDED000AB4EEE00AF1EE10FA0ADDEC4890F84210743000EB810090ED000A8DED000A032500BFE7490968843101EB77
:40E18000840004226946FBF7FBF838B99DED000AE048843000EB840080ED000A00BFDD4890F84200A0420BD1DC48C16B0220DFF870C300DFD948016D0120DFF864C300DF86
:40E1C0004D20EEF79FFF1020EEF79CFF28463EBD01B500BF02226946CF4800689230FBF7CFF820B9BDF90000CA49A1F8920000BFCA48C16B0220DFF828C300DF08BD01B5CC
:40E2000000BF02226946C44800689430FBF7B8F820B9BDF90000BF49A1F8940000BFBF48C16B0220DFF8F8C200DF08BD10B52DED020B00249DED000AF2EE040AB4EEE00A47
:40E24000F1EE10FA05DD0224B2EE040A8DED000A0DE09DED000ADFEDB30AB4EEE00AF1EE10FA04D203249FEDAF0A8DED000A00BF04226946A848006800F5FC70FBF780F87F
:40E2800020B99DED000AA34880ED7E0A00BFA348C16B0220DFF888C200DF1720EEF732FF20461CBD31B52DED020B044600BF9A490968C03101EB840004226946FBF760F8A3
:40E2C00038B99DED000A9348C03000EB840080ED000A00BF8F4890F84200A04205D18F48C16B0220DFF838C200DF3EBD31B52DED020B044600BF88490968C83101EB84003F
:40E3000004226946FBF73CF838B99DED000A8148C83000EB840080ED000A00BF7D4890F84200A04205D17D48C16B0220DFF8F0C100DF3EBD31B52DED020B044600BF764966
:40E340000968D03101EB840004226946FBF718F838B99DED000A6F48D03000EB840080ED000A00BF6B4890F84200A04205D16B48C16B0220DFF8A8C100DF3EBD31B52DEDB3
:40E38000020B044600BF64490968D83101EB840004226946FAF7F4FF38B99DED000A5D48D83000EB840080ED000A00BF594890F84200A04205D15948C16B0220DFF860C116
:40E3C00000DF3EBD13B50C4600BF53490968E031081901226946FAF7D3FF20B99DF800104C48E030015500BF4A4890F84200A04205D14A48C16B0220DFF824C100DF1CBDF7
:40E4000013B50C4600BF44490968E231081901226946FAF7B5FF20B99DF800103D48E230015500BF3B4890F84200A04205D13B48C16B0220DFF8E8C000DF1CBD31B52DED23
:40E44000020B044600BF3449096801F5F27101EB840004226946FAF793FF30B99DED000A314800EB840080ED000A00BF3EBD13B50C4600BF2849096801F5F6710819012285
